:020000040000FA
:1000000000020400000000007A8E00007A8E0000DA
:100010007A8E00007A8E00007A8E00007A8E0000C0
:100020007A8E00007A8E00007A8E00007A8E0000B0
:100030007A8E00007A8E00007A8E00007A8E0000A0
:100040007A8E00007A8E00007A8E00007A8E000090
:100050007A8E0000587100007A7100007A8E0000DC
:100060007A8E00007A8E00007A8E00007A8E000070
:100070007A8E00007A8E00007A8E00007A8E000060
:100080007A8E00007A8E00007A8E00007A8E000050
:100090007A8E00007A8E00007A8E00007A8E000040
:1000A0007A8E00007A8E00007A8E00007A8E000030
:1000B0007A8E00007A8E00007A8E00007A8E000020
:1000C0007A8E00007A8E00007A8E00007A8E000010
:1000D0007A8E00007A8E00007A8E00007A8E000000
:1000E0007A8E00007A8E00007A8E00007A8E0000F0
:1000F0007A8E00007A8E00007A8E00007A8E0000E0
:100100007A8E00007A8E00007A8E00007A8E0000CF
:100110007A8E00007A8E00007A8E00007A8E0000BF
:100120007A8E00007A8E00007A8E00007A8E0000AF
:100130007A8E00007A8E00007A8E00007A8E00009F
:100140007A8E00007A8E00007A8E00007A8E00008F
:100150007A8E00007A8E00007A8E00007A8E00007F
:100160007A8E00007A8E00007A8E00007A8E00006F
:100170007A8E00007A8E00007A8E00007A8E00005F
:100180007A8E00007A8E00007A8E00007A8E00004F
:100190007A8E00007A8E00007A8E00007A8E00003F
:1001A0007A8E00007A8E00007A8E00007A8E00002F
:1001B0007A8E00007A8E00007A8E00007A8E00001F
:1001C0007A8E00007A8E00007A8E00007A8E00000F
:1001D0007A8E00007A8E00007A8E00007A8E0000FF
:1001E0007A8E00007A8E00007A8E00007A8E0000EF
:1001F0007A8E00007A8E00007A8E00007A8E0000DF
:10020000FFFFFF00FFFFFF007A8E00007A8E0000E4
:100210007A8E00007A8E00007A8E00007A8E0000BE
:100220007A8E00007A8E00007A8E00007A8E0000AE
:100230007A8E00007A8E00007A8E00007A8E00009E
:100240007A8E00007A8E00007A8E00007A8E00008E
:100250007A8E0000587100007A7100007A8E0000DA
:100260007A8E00007A8E00007A8E00007A8E00006E
:100270007A8E00007A8E00007A8E00007A8E00005E
:100280007A8E00007A8E00007A8E00007A8E00004E
:100290007A8E00007A8E00007A8E00007A8E00003E
:1002A0007A8E00007A8E00007A8E00007A8E00002E
:1002B0007A8E00007A8E00007A8E00007A8E00001E
:1002C0007A8E00007A8E00007A8E00007A8E00000E
:1002D0007A8E00007A8E00007A8E00007A8E0000FE
:1002E0007A8E00007A8E00007A8E00007A8E0000EE
:1002F0007A8E00007A8E00007A8E00007A8E0000DE
:100300007A8E00007A8E00007A8E00007A8E0000CD
:100310007A8E00007A8E00007A8E00007A8E0000BD
:100320007A8E00007A8E00007A8E00007A8E0000AD
:100330007A8E00007A8E00007A8E00007A8E00009D
:100340007A8E00007A8E00007A8E00007A8E00008D
:100350007A8E00007A8E00007A8E00007A8E00007D
:100360007A8E00007A8E00007A8E00007A8E00006D
:100370007A8E00007A8E00007A8E00007A8E00005D
:100380007A8E00007A8E00007A8E00007A8E00004D
:100390007A8E00007A8E00007A8E00007A8E00003D
:1003A0007A8E00007A8E00007A8E00007A8E00002D
:1003B0007A8E00007A8E00007A8E00007A8E00001D
:1003C0007A8E00007A8E00007A8E00007A8E00000D
:1003D0007A8E00007A8E00007A8E00007A8E0000FD
:1003E0007A8E00007A8E00007A8E00007A8E0000ED
:1003F0007A8E00007A8E00007A8E00007A8E0000DD
:100400002F2422000E7F22000E0188000000000031
:100410000C000700C04D270001002000110007005C
:10042000000020000000E000020032000000020096
:1004300000000000368B0200000000000040DA00DF
:100440000000FE004440A900403220000000E0000F
:100450000300320000002000A00188004440A800F2
:100460000000060091018800800078000000EB0089
:1004700015003700E280400032A0B4009101BA00BC
:10048000E280400032A0B4009102BA00E280400055
:1004900032A0B4000002EB00472BDE00F507B200EB
:1004A000602CE10004003A000059EB008301E900F0
:1004B000FDFF3E00040037006128E100010032002A
:1004C0000082EB00040007001101BA000200E00006
:1004D000E8FF3A00000006003159BA008301E90044
:1004E0000C0032002159BA008301E90008003200F3
:1004F0000400E00003003A00E280400032A0B400B3
:10050000F5FF370011D9BA008301E900FAFF3A007C
:100510008100E800E180400032A0B4000000060045
:1005200000000000000000000000000000000000CB
:1005300000000000000000000000000000000000BB
:1005400000000000000000000000000000000000AB
:10055000000000000000000000000000000000009B
:10080000889FBE008A9FBE00010578000100E000BD
:100810000400350008003C000000E0002000320029
:100820000500370060001000E080180002003B0067
:1008300001F02C001A0037000004BE006011B8005F
:100840006B0920000982CF00020039000882CF0026
:100850000441B000694252000E00320008003B0023
:1008600082817100610164008904D1000884D30091
:100870008B05E8000442E800F9FF3A000500370064
:100880000804440089844C008B05E9000442E90017
:10089000FBFF3A00730207000AF0A70001F0A00076
:1008A0004F05BE004F04BE0000000600F4FF2F00FD
:1008B000920237001400200090023700889FBE008B
:1008C0008A9FBE008C1F7800A7020700AE0233008B
:1008D00003866C006450E1002E0032006420E100C9
:1008E000330032006150E1002F0032006120E1004E
:1008F0003100320085855500EB07B000090020006B
:1009000008042000050037000804440089844C00D6
:100910000A0031000603430087834B0000015300A7
:1009200081815B00F8FF33000203BE000800A000D5
:100930000804440089844C00F6FF3900C639DD0004
:100940008301730001003200130020008904D100EC
:100950000884D3000998A300050032000800A7000E
:100960000300A0008904D1000884D3008B05E800AF
:100970008904D1000884D3000001EB000281D20079
:100980003802070001F0A1000CF0A70001F0A00060
:10099000860237006420E100880232000801BE00B0
:1009A0000200BE00F7FF37006120E1008302320041
:1009B0006000B800F3FF37000000200001F82700B6
:1009C000F0FF370003F0A200889FBE008A9FBE00A0
:1009D0008C1F7800640207006B0233006450E10052
:1009E0004F0032006420E1005200320003826C00AC
:1009F00007003B000905D0000306D000820F540019
:100A00000C065D0002003900020032008901780006
:100A1000030678008582550004003D000003FD00B8
:100A20008103FD008502EA008B854200840F72007D
:100A300002003B0060001000E08018006011B80068
:100A40000005EB007A28E1000A0039000600780072
:100A5000C75DDD00F707B200878075002D00370005
:100A6000828171000A017800610560008180D100F7
:100A70000080D3008502E900F9FF3B000604400036
:100A80008784480002003B0060041400E0841C00DE
:100A90000988A300070032008A81710082817100F9
:100AA000610164008904D1000884D3008B05E8004B
:100AB000170037000978A30013003A000B00E0008C
:100AC000130034008B05E9000804440089844C00BD
:100AD0000A4474000978A3000D003A000B00E000FE
:100AE000070034008B05E9000804440089844C00A9
:100AF00001003A000B0020000978A300F7FF320044
:100B00000001EB0002003700828171000A017800C9
:100B1000D40107000CF0A70001F0A0002302370069
:100B20006420E10002003A00838F6C00230233004E
:100B30000801BE000200BE001C023700889FBE00F4
:100B40008A9FBE008C1F7800070207000E02330048
:100B500003866C006450E100240032006420E10050
:100B6000270032006150E100220032006120E100E4
:100B7000210032008B854200EB07B1000134B80040
:100B8000003AB8000804420089844A00013AB800DB
:100B90000030B8008880400009014A00040033009A
:100BA0000000400081804800020149008B05E900F7
:100BB000C909DD008301700001003200130020002C
:100BC000C814DE004814DD004709DE001200B20040
:100BD000C808DE0008847000A201070001F0A1002F
:100BE0000CF0A70001F0A000F00137006120E10047
:100BF000F20132000801BE000200BE00F7FF37001C
:100C00006150E100FCFF3A00EC0137000001BE003A
:100C1000ED0107000470A70003F0A10003F8A30092
:100C200013003A006509B1001000320009003500D8
:100C30006928E100020035000100280000000500DD
:100C400000004000818048008502E900FCFF3A0076
:100C500000000600F88F4200050035008100D10039
:100C60000080D3008502E800FCFF3A000000060087
:100C70008000EB0000000500889FBE008A9FBE0038
:100C8000030578000300E000050035000B003C0080
:100C9000008270000402710030003200070037004B
:100CA00060001000E080180060011900E081190068
:100CB00002003B0001F02D00280037000004BE00B8
:100CC0000200BE006011B8006B09200095022000F0
:100CD0000182CF000A0039000541B1000082CF0037
:100CE000070039000541B1000982CF000400390036
:100CF0000541B1000882CF00010039000541B10073
:100D000005425200120032000A003B00828171004D
:100D1000610164008100D1000080D3008984D30088
:100D20000884D3008B05E8000442E800F7FF3A008E
:100D3000070037000804440089844C000000480084
:100D4000818048008B05E9000442E900F9FF3A0080
:100D5000440107000AF0A70001F0A0004F05BE0003
:100D60004F04BE00000006000003BE00960107000D
:100D70006011B8000470A70007F0A10007F8A300F5
:100D800017003A006509B1000D0032000D00350072
:100D9000860220000628E100030035000300280039
:100DA0006000B8000200050000004000818048009B
:100DB00002014900838149008502E900FAFF3A00F7
:100DC00000000600F88F4200050034008100D100C9
:100DD0000080D3008502E800FCFF3A000000060016
:100DE0006011B8008000EB0000000500881F78004B
:100DF000000478005001BE004000BE000400400026
:100E0000858048000601490087814900009CBE009A
:100E10000294BE000400E1000588E1000690E100B4
:100E20000798E10002003100680044001008E80063
:100E30004F04780000000600F4874700889FBE003A
:100E40008A9FBE008C9FBE008E1F78000205BE00E8
:100E50000004BE00D4B79F00E5B79F00F6B79F001F
:100E600087BF9F000000EB00C0B79F00B0B79F0096
:100E7000A0B79F0090B79F0080B79F000D0420008F
:100E8000BFB097004FB09700000140000000E000A5
:100E90000F003D004F08DE0000007100C0B79F004A
:100EA0009E00070001003D0012002000A100070085
:100EB00001003D0012002000A6000700B10007005D
:100EC000B60007000F004000C8FF070022003700EF
:100ED0004F08DE0000067100CCB79F008F000700AE
:100EE00001003D00120020009200070001003D00BB
:100EF0001200200097000700A20007000FB2970021
:100F00009FB297002FB39700BFB39700A9000700C7
:100F10000000520081805A0002015B0083815B0067
:100F200080B79F0091B79F00A2B79F00B3B79F0003
:100F30000007EB009F0007000020E10001A8E1008E
:100F400002B0E10003B8E100010031001E00200002
:100F50000E005600C0B79F004FB297000400E0009B
:100F60000700350010002000010020006011B800CB
:100F700008047000898470000A0571008B85710077
:100F80008D06E900BEFF3A000400E00003003D00CA
:100F9000820007000F00400094FF07004FA8970051
:100FA0000000E00004003A000FB497009FB49700DF
:100FB0002FB59700BFB59700940007004F07780042
:100FC0004F06BE004F05BE004F04BE004F01B100EA
:100FD00000000600881F780018002000881F780095
:100FE00095FF07008F87E9004F0478000000060096
:100FF000801FEB0090FF07008F87E90000000600CC
:10100000889FBE008A9FBE008C1F78006E0007007C
:1010100007003D0073000700E00F5B00E08F5B00FE
:1010200007003D00320007000006EB000400370017
:101030003400070002003D002A0007001C002000C9
:1010400072000700E3FF07000203BE000002BE00BB
:101050000C00E00001003200220007000400BE0086
:101060000601BE004F0678004F05BE004F04BE00CB
:1010700000000600889FBE008A9FBE008C1F78007B
:101080005100070005003D0056000700E00F5B001F
:10109000E08F5B0006003D000400370019000700E8
:1010A00003003D006000B8006011B80010000700A8
:1010B00056000700CEFF07000203BE000002BE007C
:1010C0000C00E00001003200060007000400BE0032
:1010D0000601BE004F0678004F05BE004F04BE005B
:1010E000000006006000B8006011B8000000370082
:1010F0000402500085825800060359008783590076
:10110000000006000006EB00E00F5200E08F5A00DE
:10111000E00F5B00E08F5B000000060001804000F4
:1011200090B79F000001EB008FB097000100E00036
:10113000000006000200700090B79F000180400090
:1011400080B79F000001EB00FFA897000100E000BE
:10115000000006000200700080B79F000180400080
:101160006FAA9700CF20DE0001007000F0AF9F0053
:1011700004024200250007004F18DE000002720042
:1011800000000600E4AF9F000804440089844C007E
:101190000A054D008B854D00000006003FB2970008
:1011A000CFB297005FB39700EFB3970000FE2F0018
:1011B000000006003FB09700CFB097005FB19700E6
:1011C000EFB19700000006000205BE000004BE005B
:1011D000E00F5000E08F5800E00F5900E08F5900F9
:1011E000000006006000B8006011B800080450005C
:1011F000898458000A0559008B8559001C0020007D
:10120000E00F5200E08F5A00000006000800BE0008
:101210000A01BE00000006006022B800060220009D
:101220000000D0008180D2000482D2008582D200EA
:101230000000A0000202520083825A000300310025
:101240000202420083824A000000A1000603E90076
:10125000F3FF3A0000000600EFFF07000400BE00A5
:101260000000060081002000618055000B003D0059
:101270000B00200061FE2F000100E1001D00340082
:1012800082817100610164008904D1000884D30067
:101290000000E800FAFF3A007100200061006400DD
:1012A0000300700002006000090032006104440085
:1012B000E0844C000988A500050032008B05E80099
:1012C0006808E10002003A008904D1000884D300D4
:1012D000F20F20000258E10005003D00C75DDD006F
:1012E000F907B20089807500080078000000060048
:1012F0000BF827008B00780000000500889FBE00D7
:101300008A9FBE00841F7800170007004F007800F6
:1013100011003300F0FF2F00838F6C0006003B00AC
:10132000040565000A00A7000800370009F0A600C0
:101330001000200008003700820F5400838F5C00EB
:10134000030039001000200001003E0000002000D2
:1013500009F0A7000000EA004F05BE004F04BE00E0
:101360000000E000000006000004BE0016000700B8
:101370000003BE000405BE000200BE00120007000C
:10138000844F7500000006000200BE006450E100BA
:10139000050036006420E100020036000968A30061
:1013A00001003A000800BE000160A0004F0678006E
:1013B0004F05BE004F04BE0000000600F0FF2F00E6
:1013C000F1FF2700F9FF3700C70ADE00F107B2007E
:1013D000F50FB20008003200E1CF420002003200F7
:1013E0000170A00024000500810F70000100320090
:1013F0000408050044000500810F700002003A0057
:10140000140005008502E9000000400081C048008A
:10141000FCFF3B000170A000240005003E0000001E
:1014200008200000080000001B5B000044000000D2
:101430001B5B000000440000001B00005B43000039
:10144000001B00005B3200004B0D00000043000059
:10145000000000001B5B0000324400000057000049
:10146000617200006E6900006E6700003A200000A3
:101470006E6F0000207600006F6C00007461000049
:1014800067650000206F00006E20000056700000AD
:10149000756C00006C750000702000007069000021
:1014A0006E000000203D000020000000436C0000A2
:1014B0007574000063680000206500006E6700001E
:1014C0006167000065640000212100002100000028
:1014D0005652000045470000207400006F6F000066
:1014E000206C00006F7700002C2000006973000062
:1014F0002074000068650000726500002061000033
:1015000020730000686F0000727400003F0000004C
:10151000436C0000757400006368000020640000E4
:1015200069730000656E0000676100006765000078
:101530006421000021210000002E0000203C00005A
:10154000002E000020000000546F00002066000004
:10155000696E000069730000682000007365000078
:1015600074750000702C000020730000746100008E
:101570007274000020750000702000007468000084
:1015800065200000706F0000776500007220000089
:1015900073750000707000006C69000065730000D6
:1015A000207700006974000068200000636F00006D
:1015B0006D6D0000616E0000642000002757000080
:1015C000270D00000A0000000D0A0000280000009E
:1015D00078000000293E0000004200007573000002
:1015E0002050000069720000617400006520000056
:1015F0007633000000200000636C00006F6E000076
:1016000065200000772F0000646900006666000016
:1016100065720000656E00007420000050490000F3
:101620004300000046690000726D00007761000011
:101630007265000020760000362E0000332D000079
:101640006265000074610000312000007232000009
:101650003135000031200000002000002832000059
:10166000344600004A360000344700004130000094
:101670003000000034200000003200002000000094
:1016800041330000004200003400000042350000F9
:101690000042000038000000554E00004B000000E2
:1016A0002900000049090000004F00000900000067
:1016B00048090000004C000009000000456E0000D1
:1016C0007465000072200000726100007720000045
:1016D000766100006C75000065200000666F0000F8
:1016E0007220000042520000470000004C450000FC
:1016F0005400000049460000005400004845000026
:101700004E000000454C000053450000004700001B
:101710004F5400004F000000474F00005355000099
:10172000420000005245000054550000524E000097
:1017300000520000454D00000050000052490000DA
:101740004E540000004900004E5000005554000067
:10175000004600004F520000005400004F000000FF
:101760004E45000058540000005200004541000062
:1017700044000000444100005441000000530000B8
:101780005441000052540000520000005354000025
:101790004152000054000000535400004F5000001C
:1017A00052000000535400004F500000005300004E
:1017B000454E000044000000524500004345000033
:1017C0004956000045000000434C00004B0000005B
:1017D00044410000540000004249000054520000FF
:1017E0004541000044000000414400004300000067
:1017F0004155000058500000494E000000500000C4
:101800005355000000500000554C00004C5500009E
:1018100050000000444500004C4100005900000009
:10182000415500005800000046520000455100009C
:101830000044000055540000590000004D410000D4
:10184000435200004F000000454E000044000000DD
:1018500000520000554E0000004C000049530000AB
:1018600054000000455800004954000000440000A6
:101870004542000055470000004E0000455700005B
:101880000000000000000000000000000000000058
:101890002C010000000000005802000000000000C1
:1018A000B00400000000000060090000000000001B
:1018B000C0120000000000008025000000000000B1
:1018C0004038000000000000004B00000000000055
:1018D0008070000000000000009600000000000082
:1018E000C0DA00000000000000E10000000000007D
:1018F00000C200000100000000F400000100000030
:1019000000E80000030000004152000054310000D4
:1019100000000000204800007A000000467200002D
:1019200065710000756500006E6300006965000068
:10193000732000003C200000314800007A200000A5
:1019400061720000652000006E6F000074200000CE
:1019500073750000707000006F7200007465000005
:10196000642E000000000000306200000030000023
:10197000303000002C00000030300000003000004B
:1019800031320000333400003536000037380000B3
:101990003941000042430000444500004630000049
:1019A00078000000436F0000756C0000646E00005A
:1019B00027740000206B00006565000070200000A7
:1019C0007570000000000000535000004931000015
:1019D0000000000000290000002000005700000067
:1019E0002052000000490000324300003100000096
:1019F0003A200000000000002E00000031570000D7
:101A00003031000000000000314100004C53000064
:101A1000004200005076000033000000080800007B
:101A2000080800000800000000000000424200001A
:101A3000494F0000310000005241000057310000C2
:101A4000000000004F43000044310000000000008F
:101A5000000000000000000029000000000000005D
:101A600000000000EE874700889FBE008A9FBE00EE
:101A70008C9FBE008E1F78000000EB0080678800FE
:101A800070678800A0408800906788000001780097
:101A900043CF20000042EB00050220004510DD008E
:101AA000030040008000EB00045878008100E8004B
:101AB000858F5000FCFF3A000201E800E50F51005D
:101AC000F6FF3A000000EB00A06C8800800678006A
:101AD000D0B79F00C0B79F000CB42000A140800089
:101AE000000320000089B90040952000000041005B
:101AF000826D020000000000A18120000020200073
:101B0000110060000400320071002000E056200047
:101B1000188A020000000000E0A02800826D020088
:101B2000000000000001EB00B2B79F000100370089
:101B3000BEB79F00A06C80000000E00044003200AF
:101B40000000E900A06C88004500DD0041CF2000C6
:101B5000E0C078000104E000130032000004EB0054
:101B6000E9BE20004ACF20007067800001F07C00B1
:101B7000014078000E7102000000000070678000D4
:101B80000000E8000804E800F00FB2007067880069
:101B9000A06C80004500DD0008004000E0407D00B2
:101BA0000104E000F0FF3A000000EB00A06C8800A8
:101BB000270037009C40780064C060002400320099
:101BC0004A8120001A007800090320000980B9002A
:101BD0007A004000C892200060007C0000000100F4
:101BE0000000E0001A0032001A0078000980B900F5
:101BF0008002B00008004000826D0200000000007A
:101C0000E0A02800826D02000000000080678000D4
:101C100071678000810F50000D00320000047800D1
:101C2000808F50000A003200E9BE200068C07C00AE
:101C30000E7102000000000008007800F00FB200F2
:101C40000004E80070678000800F5400F7FF3A003E
:101C500074700200000000000004E000D5FF3200B4
:101C60002A710200000000000004E00003003200BE
:101C70003271020000000000AEFF3700FA7002006F
:101C800000000000004578000080FB0001002000FB
:101C9000F2072000820F5000E08F580087023E00BC
:101CA000006001007D0237003F023700130137005A
:101CB00082023700BD0037004E0237002501370091
:101CC0007E023700770037007C0237005C02370065
:101CD0007A0237007902370059023700990137003C
:101CE000760237002901370074023700730237008B
:101CF0007202370071023700700237006F0237003E
:101D00006E0237006D0237006C0237006B0237003D
:101D1000D3003700690237006802370067023700D6
:101D2000660237006502370064023700630237003D
:101D30006202370061023700600237005F0237003D
:101D40005E0237005D0237005C0237005B0237003D
:101D50005A0237005902370058023700570237003D
:101D6000560237005502370054023700530237003D
:101D70005202370051023700500237004F0237003D
:101D80004E0237004D0237004C0237004B0237003D
:101D90004A0237004902370048023700470237003D
:101DA000460237004502370044023700430237003D
:101DB0004202370041023700400237003F0237003D
:101DC0003E0237003D0237003C0237003B0237003D
:101DD0003A0237003902370038023700370237003D
:101DE000360237003502370034023700330237003D
:101DF0003202370031023700300237002F0237003D
:101E00002E0237002D0237002C0237002B0237003C
:101E10002A0237002902370028023700270237003C
:101E2000260237002502370024023700230237003C
:101E30002202370021023700200237001F0237003C
:101E40001E0237001D0237001C0237001B0237003C
:101E50001A0237001902370018023700170237003C
:101E6000160237001502370014023700130237003C
:101E70001202370011023700100237000F0237003C
:101E80000E0237000D0237000C0237000B0237003C
:101E90000A0237000902370008023700070237003C
:101EA0004200370080678000808F56003B00320080
:101EB00070678000808F56000B003A000D00E9002B
:101EC00080067800FD0FB2007D6788000040EB00BF
:101ED000E3BE200080F6790000A12800826D020098
:101EE0000000000013FF37000D00E90080067800B5
:101EF000FD0FB20040A12800826D0200000000002A
:101F00000D0178008D0078008004EB007067800080
:101F10008D0F5000140032008004EB00EABE200058
:101F20000204E80068407D0000717D000004E000CC
:101F3000030032000E7102000000000003003700B1
:101F400000C2B3000E710200000000008904E80026
:101F500008017800F20FB2008200780070678000FC
:101F6000820F5000EEFF3A000100E900F00FB200CE
:101F70007067880080A12800826D020000000000C8
:101F8000094078005E6F020000000000B0A1280048
:101F9000826D020000000000E6FE370070C0B30052
:101FA0000E71020000000000E2FE37007067800042
:101FB000808F5600260032008D0078000D017800D9
:101FC0000005EB008D0F5000140032000005EB00FF
:101FD000E9BE20000104E80068C07C0080F07C00BD
:101FE0000004E000030032000E7102000000000057
:101FF0000300370000C2B3000E71020000000000B1
:102000000A05E80088007800F10FB20001017800AD
:1020100070678000810F5000EEFF3A000200E90077
:10202000F00FB2007067880080A12800826D020066
:10203000000000000A4078005E6F0200000000000F
:10204000B0A12800826D020000000000B9FE370038
:1020500070C0B3000E71020000000000B5FE370032
:10206000FA70020000000000B1C5B300814F5000BB
:10207000B0FE3A00FA7002000000000080407800D4
:1020800010C4B30080CF50004000320007003E0073
:102090007040500080CF50000C0032006340400080
:1020A00080CF5000A3FE3A000E00370030C4B300CA
:1020B00080CF500027003200A20039000040E80025
:1020C00080CF50009BFE3A000C003700FA700200EF
:1020D00000000000E1C7B300814F500095FE3A00B8
:1020E00031013700FA70020000000000E1C7B300C0
:1020F000814F50008FFE3A003E0137004FB09700ED
:10210000E40F500005003400F07C020000000000E5
:102110008000EB00C1B79F0086FE3700806780001B
:10212000808F5600070032000D00E900800678001D
:10213000FD0FB20040A12800826D020000000000E7
:102140007CFE370070C0B3000E710200000000007A
:1021500078FE370070678000808F560007003200DD
:102160000D00E80080067800FD0FB200D0A1280025
:10217000826D0200000000006EFE370070C0B300E8
:102180000E710200000000006AFE370084678000C4
:102190000400E90000047800F80FB2000805780098
:1021A00071678000888F5000620032008002EB006F
:1021B000E3BE200068C079000004E00057003A0048
:1021C0000800E90000017800F20FB20062C0790057
:1021D0000004E000510032008502E800BFB1970022
:1021E000858F51004D0031008301E800B3B79F0097
:1021F000810F52000A003200E3BE20008042EB0053
:10220000F60F200085F079000100E90086006000EB
:10221000810F5200FBFF3A007167880085F079005A
:1022200071678000828F5000DD053A000D00370095
:10223000E3BE200062C079000004E00004003A0020
:102240000200E800F00FB200D0B79F000500370091
:102250000200E90000017800F20FB200828F500006
:10226000F3FF3A0010A22800826D02000000000077
:10227000A1408000000320000089B90040952000A3
:1022800000004100826D020000000000A1812000DA
:1022900000202000110060000400320071002000C6
:1022A000E0562000188A020000000000E0A028008C
:1022B000826D0200000000005FB09700880F5000A0
:1022C0000F00320080047800EBBE2000FD0F2000DC
:1022D00069C07D000E710200000000007067800080
:1022E00069F07D000000E8000D0060007067880064
:1022F0000900E8008D046000888F5400F4FF3A0064
:102300007D6780000040EB00E2BE2000807679000F
:102310008A8F560007FE3A00060037000800E900E1
:1023200000047800F80FB20008057800888F50008C
:102330009FFF3A0070C0B3000E7102000000000061
:10234000FCFD3700846780000400E9008004780009
:10235000F90FB2000905780071678000818F540081
:10236000620032000007EB00E3BE200069C0790084
:102370000004E00057003A000900E900000178007D
:10238000F20FB20062C079000004E0005100320098
:102390000E07E800BFB197000300E9008E0F500060
:1023A0004C003A00810F52000A003200E3BE2000C8
:1023B0008042EB00F60F200085F079000100E90073
:1023C00086006000810F5200FBFF3A0071678800B1
:1023D00085F0790071678000828F500075053A00A2
:1023E0000D003700E3BE200062C079000004E00069
:1023F00004003A000200E800F00FB200D0B79F00DE
:10240000050037000200E90000017800F20FB20079
:10241000828F5000F3FF3A0010A22800826D020064
:1024200000000000A1408000000320000089B900E6
:102430004095200000004100826D02000000000075
:10244000A181200000202000110060000400320063
:1024500071002000E0562000188A020000000000F1
:10246000E0A02800826D0200000000005FB097002D
:10247000890F50000F00320000047800EBBE2000EE
:10248000FD0F200068C07D000E71020000000000FA
:102490007067800068F07D000000E8000D006000BB
:1024A000706788000800E8000D046000890F540080
:1024B000F4FF3A007D6780000040EB00E2BE2000A0
:1024C000807679008A8F560099FD3A00BEB79F004A
:1024D000060037000900E90080047800F90FB20017
:1024E00009057800898F50009FFF3A003FB09700A0
:1024F000E10F500028003A0010A22800826D02006F
:1025000000000000A1408000000320000089B90005
:102510004095200000004100826D02000000000094
:10252000A181200000202000110060000400320082
:1025300071002000E0562000188A02000000000010
:10254000E0A02800826D0200000000007D6780008E
:1025500081678000818F560009003200E2BE2000B2
:102560008041EB00F40F2000837679000D00E90034
:1025700084066000818F5600FBFF3A007D6788006B
:102580000040EB00E1BE200080F678000001EB0087
:10259000B2B79F0067FD370070C0B3000E71020034
:1025A0000000000063FD370088678000888F5600B8
:1025B0000C00320080A12800826D020000000000A3
:1025C00008805600F00FB2005E6F020000000000AD
:1025D000B0A12800826D0200000000008D6780001D
:1025E00054FD370070C0B3000E71020000000000FF
:1025F00050FD370078678000888F56000C0032004D
:1026000080A12800826D0200000000000D0054002F
:10261000F00FB2005E6F02000000000070A2280000
:10262000826D0200000000007D67800041FD3700E0
:1026300070C0B3000E710200000000003DFD3700C5
:10264000706780008040EB00E3BE200001F079005D
:102650000000E80080067800FD0FB2007D6788006A
:1026600090A228009A6D02000000000070678000B0
:10267000F0B79F0081678000E1B79F000000EB008A
:1026800090678800A18120000020200011006000D8
:102690000047EB005B003200530037004FB197005A
:1026A0000201E800C2B79F00F40F510021FD3A007B
:1026B000A2710200000000001EFD37007867800054
:1026C0000800E800F90F2000090060008167800021
:1026D000810F500040003200FF4F55003E00360091
:1026E000E0C7B300804F55003B003E008D0F540003
:1026F0000C003A000A4078000E7102000000000051
:1027000070678000E3BE20000AF079000000E80056
:10271000890660007D6788000040EB0080F6790044
:1027200004FD370080A12800826D02000000000037
:102730000D005400F80F2000080060005E6F0200DA
:102740000000000070A22800826D0200000000005E
:10275000796780000D00E90088056000898F5500C9
:1027600010003200E8BE20000900E80069707C001B
:1027700069407C000004E000050032000E71020098
:1027800000000000A0A22800826D020000000000EE
:102790000900E90080047800F90FB200898F550024
:1027A000F1FF3A000A4078000E71020000000000BC
:1027B000E2BE20008A7679000D00E800F10F2000CB
:1027C00081066000706780000000E8000100600082
:1027D00070678800D7FC370070C0B3000E7102002C
:1027E00000000000D3FC3700803D02000000000024
:1027F0005100200050572000728A020000000000A3
:102800006304370082678000E3BE200062C0790065
:102810000080FB0001002000E3072000830F500030
:10282000E08F580033043E0000600100330437009D
:10283000300437002F0437002E0437002D043700F2
:102840002C0437002B0437002A04370029043700F2
:1028500028043700290437002604370025043700F0
:1028600026043700230437002204370021043700F0
:10287000200437001F0437001E0437001D043700F2
:102880001C0437001B0437001A04370019043700F2
:1028900018043700170437001604370015043700F2
:1028A00014043700130437001204370013043700F0
:1028B000F303370075023700120137001B013700A0
:1028C000CF013700BD0137000A043700520237003C
:1028D00008043700070437000804370007043700EE
:1028E000A7033700BE0337008D033700D802370037
:1028F000D7023700D6023700D5023700D40237009E
:10290000D3023700D2023700D1023700D00237009D
:10291000CF023700F7033700F6033700D70137003F
:10292000B8003700F30337003F00370029013700B4
:102930001D013700EF033700610037009C013700AD
:10294000EC033700EB033700EA033700E9033700F5
:10295000E8033700E7033700E6033700610037007C
:10296000E4033700E3033700E20337008100370058
:10297000E0033700DF033700B5013700DD03370020
:10298000DC033700DB03370026013700D9033700AB
:10299000D8033700D70337008E0237006C033700A7
:1029A0009B0237009C03370081033700D1033700B7
:1029B000F2003700270037003A0037006E01370079
:1029C000CC033700290037002B003700CB0337003A
:1029D00018003700C7033700C60337004A00370026
:1029E0001A003700C30337001C0037004F003700C0
:1029F000C0033700F902370092013700BD033700EA
:102A0000BC0337001700370040013700B903370017
:102A1000B8033700B703370075023700910037005D
:102A200083023700AA0037007C8A02000000000001
:102A3000B2033700E9050700408120001000E000E4
:102A4000AE0332005A060700AC033700E10407006A
:102A5000AA03370078070700A803370057070700C5
:102A6000A6033700D7060700A40337005E41020023
:102A700000000000A1033700408120001000E000AA
:102A800005003A00D1012000505A2000728A02004D
:102A900000000000990337000C4002000000000015
:102AA00096033700C0CFB3001C4E600061012000C8
:102AB000A0572000728A0200000000008F03370038
:102AC0001C4078000014A1000004A000004E780013
:102AD0005101200000592000728A0200000000000D
:102AE000860337001C34A000C1012000E07E2000D6
:102AF000188A02000000000090A228009A6D0200CF
:102B0000000000007D0337001C34A100B10120004B
:102B1000307D2000188A02000000000090A22800EA
:102B20009A6D02000000000074033700408120000D
:102B30001000E00005003A00D1012000505A2000AA
:102B4000728A0200000000006C033700CB62A9000B
:102B5000C962A90051012000205C2000188A0200EF
:102B60000000000090A228009A6D02000000000002
:102B700062033700408120001000E00005003A00A9
:102B8000D1012000505A2000728A0200000000008B
:102B90005A0337009C40780070C0600004003A007F
:102BA00021022000F0E92000728A020000000000EB
:102BB000C962A800CB62A90041012000705D20001D
:102BC000188A02000000000090A228009A6D0200FE
:102BD0000000000021E3A800B0C0B3009488020008
:102BE00000000000F1042000810F500003003E00AF
:102BF000F0A228009A6D02000000000021E3A90065
:102C00003E0337000200E800F00FB2008067880042
:102C1000600407007503070000047800A46F020039
:102C20000000000020A52800826D020000000000C6
:102C3000084078005E6F02000000000020A5280018
:102C4000826D02000000000008407800BA6D0200AA
:102C50000000000090A228009A6D02000000000011
:102C6000260337000200E800F00FB20080678800FA
:102C7000480407005D0307000080FB00F0890200A4
:102C80000000000000047800A46F020000000000B3
:102C900020A52800826D0200000000000840780096
:102CA0005E6F02000000000020A52800826D020077
:102CB0000000000008407800BA6D0200000000002B
:102CC00090A228009A6D0200000000000B0337005C
:102CD000408120001000E00005003A0011C0B30060
:102CE00001407800C88102000000000003033700A3
:102CF000A1012000B05E2000728A020000000000E6
:102D0000FE0237005100200050602000728A02004D
:102D1000000000006C700200000000000004E000F1
:102D2000FCFF32000000FE00F4023700088B0200B6
:102D3000000000000000E000F0023200A1002000CE
:102D4000A0602000728A02000000000040062000FF
:102D50009E8902000000000056880200000000006A
:102D60006C700200000000000004E000FCFF320074
:102D700081BF2A0001400100E0023700B8030700CC
:102D8000800478000000E000DC0232000004EB0068
:102D900044470200000000000804E800888F540047
:102DA000D6023200FAFF3700AD0307008004780036
:102DB0000000E000D10232000004EB0028470200CE
:102DC000000000000804E800888F5400CB023200A5
:102DD000FAFF3700A2030700800478000000E0003B
:102DE000C60232000004EB006101200040612000B7
:102DF000188A020000000000604702000000000086
:102E0000726D02000000000090A228009A6D02007E
:102E1000000000000804E800888F5400B702320068
:102E2000F1FF3700408120001000E00005003A006B
:102E3000D1012000505A2000728A020000000000D8
:102E4000AE023700C002A900C202A80021E3A80018
:102E5000200020009E89020000000000A0C0B300F6
:102E60009488020000000000011B2000810F500028
:102E70001800360090C0B3009488020000000000E3
:102E8000712B2000810F500012003600110120002C
:102E9000A0622000188A02000000000090A2280012
:102EA0009A6D020000000000A04080000203200094
:102EB0000280B9000002B000C292200060007900D8
:102EC0000000010060A528009A6D020000000000CB
:102ED0000C003700C002A900C202A90080A6280089
:102EE0009A6D02000000000021012000B063200064
:102EF000188A02000000000090A228009A6D0200CB
:102F00000000000021E3A9007C023700A1408000FE
:102F10000100E00005003A00D1012000505A2000D5
:102F2000728A0200000000007402370000032000D3
:102F30000088B9002002B000C29220006000790031
:102F40000000010080A828009A6D02000000000027
:102F5000C002A900C202A90021012000B063200024
:102F6000188A02000000000090A228009A6D02005A
:102F70000000000061023700F1002000C036200090
:102F8000188A020000000000A6880200000000006D
:102F900011002000B0372000188A02000000000055
:102FA00090A228009A6D0200000000005302370032
:102FB000B488020000000000500237002803070018
:102FC000000478006100200090652000188A02004B
:102FD0000000000008007800146F020000000000EC
:102FE00021002000F0652000728A0200000000002D
:102FF00008007800C2890200000000003F0237008C
:10300000170307000004780061002000906520008D
:10301000188A02000000000008007800146F020007
:10302000000000002100200030EE2000728A020023
:1030300000000000080078009E89020000000000E7
:103040002E023700A08120001090A0002B02370034
:10305000408120001000E00005003A00D10120006E
:10306000505A2000728A020000000000230237003C
:1030700086470200000000002002370011002000F7
:10308000916788000200E8008081FB00E0BE20001C
:10309000634078000004E000130032000102780071
:1030A000E6C3B300F70F2000E5BE2000864F5000B6
:1030B00001003A000002EB008100E800010041003D
:1030C0000700600060C07A000004E000F7FF3A00EB
:1030D0009467880020022000808F50000200340096
:1030E0001000200090678800996780000900E000C8
:1030F00002023A00836788003C020700000478005F
:1031000082678000F30F200083006100E0BE200092
:10311000E1407800D0C3B30080CF50001E003A00D9
:103120000802E900E40F520018003E000200E80027
:103130008301600083678800C520DD0040CF200048
:1031400080804000090078000041EB00050220006B
:10315000825878000000E800850F50001A02320003
:10316000FBFF3700825878000300E8008081FB00F5
:10317000E0BE200063417800E0C3B300804F5100FF
:10318000F8FF3A0083678800DC0137001000200058
:1031900090678800D90137000800E00013003A006A
:1031A00049CF200018002000084078005E6F020020
:1031B00000000000D0A92800826D0200000000007D
:1031C00009007800826D020000000000E0A02800E5
:1031D0009A6D0200000000000804E8000902B00037
:1031E000E60F5400C5013200EFFF37000800E90088
:1031F000E40F500005003E0090A228009A6D0200E6
:1032000000000000A86C8800BC01370010002000FE
:1032100090678800B90137000200E800F80F20002D
:103220000800600080678800F001070080047800D3
:10323000D80207008067800008006000E1BE20001F
:10324000E0C0780090C2B30080CF50000C003A007C
:10325000A0408000020320000280B9007C004000F2
:10326000C2922000E000790009007800010001000E
:1032700090A228009A6D0200000000009F01370014
:1032800010002000906788009C0137001300200088
:10329000936788000200E8000080FB00E1BE200088
:1032A00060C078000004E0000E0032008280E80078
:1032B0000301780025C2B300F30F2000E4BE200014
:1032C000854F500001003A000001EB0003806000D0
:1032D00060407A008100E8000004E000F8FF3A0056
:1032E00092678800906780000000E00083013A0048
:1032F0007100200010662000188A02000000000003
:1033000020C2B3000E710200000000008067800040
:103310000000E800806788000081FB00E0BE20001C
:10332000E240780020C2B30080CF5000210032007C
:10333000E8BE200082678800014078000E7102001C
:10334000000000008067800060407C008001FB007E
:1033500000B4200010407800684060000400320093
:1033600003007800F089020000000000800178006E
:10337000A0408000020320000280B90068004000E5
:10338000C2922000E00079000300780001000100F3
:10339000806780000000E8008067880000017800F6
:1033A000F20FB200E2407C0020C2B30080CF500098
:1033B000E0FF3A008267880020C2B3000E7102006D
:1033C0000000000090A228009A6D0200000000009A
:1033D0004A013700A0408000020320000280B900AB
:1033E000C292200062007800000001004301370013
:1033F000A0408000020320000280B9000080E800A5
:10340000C292200060007900000001003B013700FB
:10341000A0408000020320000280B9006400400048
:10342000C2922000600079000000010033013700E3
:10343000A0408000020320000280B9006600400026
:10344000C292200060007900000001002B013700CB
:103450007100200010662000188A020000000000A1
:103460006201070080047800806780000000E900A6
:103470000080FB0080678800F901070080BF9F0083
:103480000E020700800078000000E0000900320012
:10349000F0B2200001487800E88F500003003400AB
:1034A00000B420001054A0000200370000B4200037
:1034B0001054A1008005EB0041003700090078009E
:1034C000128902000000000003C2B30002B4200011
:1034D00012C0610005003A0081C0B300F0B22000C4
:1034E00090CF100005003A000B00370003C1B30075
:1034F000F2B2200092CF110007003200B0C3B30037
:103500000E71020000000000F1B2200011407800AE
:103510005E6F02000000000002B42000124178003B
:10352000684061000400320009007800F089020060
:103530000000000080047800A0408000020320000A
:103540000280B90068004000C2922000E0007900CB
:1035500009007800010001000004780000C2B300F7
:103560000E710200000000000AB4200003C4B30082
:103570001AC0610011003200610020008066200046
:10358000188A0200000000001A45780068406500B3
:103590000400320008007800F089020000000000FA
:1035A0000004780008007800128902000000000082
:1035B00000C2B3000E710200000000008B05E8009D
:1035C0000FB89700808F5500BCFF3A0090A22800EA
:1035D0009A6D020000000000C80037006100200062
:1035E00080662000188A020000000000CA0107005F
:1035F000804478009A01070080057800AF01070039
:10360000800078000000E00009003200F0B22000E5
:1036100001487800E88F50000300340000B4200017
:103620001054A0000200370000B420001054A10084
:103630000904E000040032002181200011477800D5
:103640000980FB008008E9000B00E0002C0032003C
:103650000004EB00FAB22000A0408000020320002A
:103660000280B9006A004000C29220006000790028
:10367000000001008000780002B4200012417800B0
:10368000684061000400320001007800F089020007
:10369000000000008000780001007800128902001C
:1036A0000000000001C2B30003B4200013C060009A
:1036B00004003A0082C0B3009A4F110004003A009F
:1036C0000900370003C1B3009ACF11000600320091
:1036D000B0C3B3000E710200000000001A40780071
:1036E0005E6F02000000000000C2B3000E71020015
:1036F000000000000804E800888F5500D6FF3A005B
:103700000904E000020032000E80FB0090408800B7
:1037100090A228009A6D0200000000007700370098
:1037200081002000E0662000728A02000000000094
:10373000A0408000020320000280B9006C0040001D
:10374000C292200060007900000001006B00370089
:103750008100200060672000728A020000000000E3
:10376000A0408000020320000280B9006E004000EB
:10377000C292200060007900000001005F00370065
:10378000E1002000E0672000728A020000000000D3
:10379000A0408000020320000280B90070004000B9
:1037A000C292200060007900000001005300370041
:1037B000E1002000C0682000728A020000000000C2
:1037C000A0408000020320000280B9007200400087
:1037D000C29220006000790000000100470037001D
:1037E000C1002000D0642000188A02000000000000
:1037F000A0408000020320000280B9007400400055
:10380000C29220006000790000000100726D020089
:1038100000000000390037001101070000047800A3
:10382000D1002000A06A2000188A020000000000D9
:103830000800780012890200000000000800E00083
:103840000B0032008004EB000A032000CB92200022
:10385000A04080000A80B9007600400060807D00B2
:10386000000001008904E800890F5400F8FF3A00C5
:1038700090A228009A6D0200000000001F0037008F
:10388000F700070080047800A1002000706B200082
:10389000188A0200000000000900E0001000320059
:1038A0000004EB000A032000CB922000A04080001F
:1038B0000A80B9007800400060807D0000000100AF
:1038C000726D02000000000000C2B3000E71020021
:1038D000000000000804E800888F5400F3FF3A005D
:1038E00001012000A0692000728A0200000000008F
:1038F0000200370010002000906788008067800079
:103900000000E8000080FB0080678800906780006E
:103910000000E00002003A000001780016003700C5
:1039200051012000106C2000188A020000000000E5
:1039300080678000EFB09700808F50000400310056
:10394000014050005E6F02000000000004003700DC
:103950004FE99700024050005E6F02000000000037
:103960000000EB009067880090A228009A6D02008A
:103970000000000012002000816780007067800056
:10398000808F5000020032000200E0009DFB3200F8
:10399000FFB1970083678800736788004FF837008E
:1039A000E0BE2000624078000004E00024FA32000B
:1039B00027FA3700E0BE2000624078000004E000F3
:1039C0008CFA32008FFA3700E0BE200063417800A5
:1039D000E0C3B300804F5100C8FF3200C520DD00B6
:1039E00040CF200080804000DEFD3700881F780037
:1039F00085678000F40F200004806200E3BE200091
:103A0000E0C07900F0CCB30000C04000E84F5000A7
:103A10001A003E000100FB0001FD2F0001014000E3
:103A20000500E8000400600060C2790081404200A7
:103A300016002000E9CF500077003E00160020005D
:103A400001FD2F00F80F2000E7BE20006A11B90029
:103A50000400FB0002004000010140000603E800F2
:103A6000068042000800600060C27B000140420006
:103A7000E94F500068003E00F4FF370000C3B30078
:103A800080CF500060003A000500E8000080FB0095
:103A9000E1BE200060C2780020C6B300804F520013
:103AA0006100320020C4B300804F520012003A007F
:103AB0005D003700260020000001EB0003FD2F0011
:103AC000F70F2000E4BE2000020041008100FB004F
:103AD00001004000030140000603E80006804200A8
:103AE00007006000E0407A0003C04000E14F500052
:103AF00049003E00F4FF370080C7B300804F5200FA
:103B00001600320080C5B300804F520026003A00F4
:103B1000120037004411DD00E9CF510005003E00DE
:103B20000100FB000000410001FD2F0001014000E9
:103B300008003700014078000054A000E1BE2000DA
:103B400000F278000000FB000000410091FA2F0015
:103B5000010140000603E8000200370026002000B3
:103B60000001EB00068042000082FB00E0BE200066
:103B7000E440780000CDB30080C14000E9CF51009F
:103B8000E4FF36007140500000C04000E54F500097
:103B9000E0FF3600F0C9B30000C04000E54F500020
:103BA000DCFF36001C00370000CDB30000404200AF
:103BB000160020000001EB00E94F500016003E0007
:103BC0008400FB0000FD2F00008140008000780091
:103BD000F80F2000E7BE20006A11B9000400FB00C6
:103BE00002004000010140000603E8000500430018
:103BF0000800600060C27B0001404200E94F5000B5
:103C000005003E00F4FF3700100020009067880098
:103C10000001EB000F003700068042000080FB002F
:103C2000806788000B0037000580E8000080FB00FB
:103C3000E1BE2000E0C0780000CDB30000C040002D
:103C4000260020000001EB00E14F5000F2FF3E0093
:103C500098FF3700020078004F047800000006004B
:103C6000881F7800826780000200E8000080FB0067
:103C7000E1BE2000E0C0780013002000A0C3B30024
:103C800080CF50000A003A000280E800F80F2000C0
:103C9000080060008067880054FF070080017800FA
:103CA000806780000000E9000800600080678800ED
:103CB000030078004F04780000000600881F780099
:103CC000826780000200E8000080FB00E1BE200067
:103CD000E0C078008001EB00B0C3B30080CF50009B
:103CE0000A003A000280E800F80F20000800600097
:103CF000806788003DFF07008001780080678000B2
:103D00000000E90008006000806788000300780078
:103D10004F04780000000600806780000000E80083
:103D20000081FB00E0BE2000E240780080C7B300C5
:103D300080CF500003003A00826788001300200003
:103D40001200370040C6B30080CF500003003A0095
:103D500082678800230020000C00370020C6B300D3
:103D600080CF500003003A008267880033002000B3
:103D7000060037008001EB0070C7B30080CF500011
:103D800002003A00826788004300200003007800A8
:103D90000000060082678000E0BE2000E24078005C
:103DA00000C2B30080CF500009003A00F40F200099
:103DB000E3BE2000804078000200E80004016000BB
:103DC00062C07900814F5000FBFF3200826788009B
:103DD00000000600889FBE008A9FBE008C1F7800EE
:103DE000806780000000E8000080FB00806788009A
:103DF000E8FF0700FDFE07000000E00042003A0077
:103E0000180020000B032000CA9220000840780010
:103E10005E6F02000000000010AA2800826D020000
:103E2000000000000BC0B900680050000A0040000C
:103E30009A6D0200000000000804E800E90F540039
:103E4000F2FF3A0071012000606D2000728A0200CA
:103E5000000000000000EB009067880013002000C5
:103E60008200200083007800030078004C000700E7
:103E70000006E9000000E800E10F500005003E00E8
:103E8000E1002000D06E2000728A020000000000D5
:103E90003B0037004B8120001B0078000803200006
:103EA0000880B9002002B000CA92200060007D00A6
:103EB0000000010056880200000000008C0D780010
:103EC00008E4B9007E04440068007D0000000100A1
:103ED00080A828009A6D0200000000000C00E0009D
:103EE00004003200C222A80040AA28009A6D0200F5
:103EF000000000005100200050572000728A02008C
:103F0000000000001E0037000006E900E70F560021
:103F100017003C004B8120001B00780008032000A4
:103F20000880B9002002B000CA92200060007D0025
:103F30000000010056880200000000008C0D78008F
:103F400008E4B9007E04440068007D000000010020
:103F50000C00E00001003200C222A8005100200045
:103F600050572000728A0200000000000400370051
:103F700051012000C0722000728A0200000000007F
:103F8000706780000000E9000080FB008067880007
:103F90004F0678004F05BE004F04BE00000006002B
:103FA000E8874700889FBE008A9FBE008C9FBE00A6
:103FB0008E1F78000005BE00820678000307780097
:103FC00040AE2800826D0200000000000A00E00000
:103FD00004003D0080AE2800826D02000000000059
:103FE000030037000A4078005E6F02000000000006
:103FF000A0AE2800826D0200000000008004EB00EB
:1040000009067800360037000900E000050032009C
:104010008904E90000A12800826D02000000000070
:104020002F0037000C00E0000600320000A128003D
:10403000826D0200000000008004EB000906780099
:104040002700370070C0B3000E71020000000000AE
:104050008004EB00220037000900E00005003A0070
:10406000D0C2B3000E710200000000001C0020004E
:104070001B00370070C0B3000E710200000000008A
:10408000170037000E00E00046003A0000CDB300F4
:1040900000404400E94F50000E003E00E38F540002
:1040A0000500340070C0B3000E7102000000000073
:1040B000490020000A003700084078000E71020015
:1040C000000000007480540008F07F008904E800BC
:1040D0000300370070C0B3000E7102000000000042
:1040E000FA7002000000000000447800ED4F50001C
:1040F0002E00320005003C00E84F5000C2FF3200A5
:10410000EA4F5000E1FF3A0028003700D0C2B30068
:10411000804F5400D0FF320080C7B300804F54005E
:10412000DAFF3A00D7FF37000901E9000000EB0091
:104130000D0033000000EB008000780005FD2F002B
:104140000202E8006A01B9007483570066C0780073
:104150000000FB0002004000050040008100E80074
:10416000848F5000F7FF3A00808F550008003C0014
:10417000808F5600060035000C00E00002003A0077
:10418000000578000E0037000005EA000C0037003B
:10419000B101200080EC2000728A020000000000C3
:1041A00087FF37000085EB000500370090A228004C
:1041B0009A6D0200000000000900E000DAFF3A00FA
:1041C0000A0078004F0778004F06BE004F05BE007A
:1041D0004F04BE008F00B10000000600881F780069
:1041E000D0AE2800826D020000000000E0C2B300E3
:1041F0000E71020000000000A08120001040780035
:104200000E7102000000000061812000F0442000D7
:10421000910F100003003A00B0AF2800826D020039
:104220000000000090A228009A6D0200000000002B
:1042300020B12800826D020000000000D1002000A3
:10424000A0802000188A020000000000A1BF2A0000
:104250000000EB0034700200000000000004780051
:104260004800DE005E6F020000000000E0C2B30004
:104270000E71020000000000084078005E6F02002E
:104280000000000090A228009A6D020000000000CB
:104290006100200030762000188A02000000000033
:1042A0006881200018007800E06F02000000000024
:1042B0007100200010EC2000188A020000000000AD
:1042C000C0408000E06F020000000000D0B2280073
:1042D000826D020000000000F0442000980F1000E2
:1042E00004003A00A0B32800826D02000000000024
:1042F00003003700D0B32800826D020000000000E8
:10430000C140800020042300808F50001000320044
:1043100004003E0030002300808F500018003A0057
:104320000700370030042300808F50000C0032005B
:1043300063004000808F500011003A000C003700ED
:1043400000B42800826D0200000000000F0037005A
:1043500030B42800826D0200000000000B0037001E
:1043600060B42800826D02000000000007003700E2
:1043700090B42800826D02000000000003003700A6
:10438000C0B42800826D02000000000000B52800C3
:104390009A6D020000000000E101200090762000EC
:1043A000728A0200000000004F047800000006003E
:1043B0005100200050922000188A020000000000E6
:1043C000C1BF2A000000EB003470020000000000B2
:1043D000E06F02000000000061002000A0922000B9
:1043E000188A020000000000E1BF2A000000EB0074
:1043F0003470020000000000E06F020000000000C6
:1044000090A228009A6D020000000000C100200068
:1044100070782000728A0200000000006900070026
:10442000C2C2BF000008A300050032001101200035
:10443000A0622000188A020000000000040037007B
:1044400021012000B0632000188A02000000000053
:10445000C0C2B3000E7102000000000000C2B30031
:104460000E71020000000000CBC2BF000038A300A4
:104470000500320041012000705D2000188A020012
:10448000000000000400370051012000205C2000E3
:10449000188A020000000000C0C2B3000E710200C2
:1044A0000000000000C2B3000E7102000000000016
:1044B00000B4200010407800704060000500320019
:1044C0002102200030792000728A020000000000E2
:1044D00004003700E1012000507B2000728A0200B6
:1044E0000000000000B42000104078006840600028
:1044F00005003A00B1012000307D2000188A02003A
:104500000000000004003700C1012000E07E200010
:10451000188A020000000000C0C2B3000E71020041
:104520000000000000C2B3000E7102000000000095
:10453000B1012000B01A2100188A0200000000001A
:10454000F0B22000104078005E6F02000000000012
:1045500090A228009A6D02000000000000B4200024
:104560001040780063406000E14F500005003A00C1
:104570005101200000592000728A02000000000052
:104580000400370061012000A0572000728A020059
:1045900000000000A0408000020320000280B9005B
:1045A0006002B000C29220006000790000000100AB
:1045B000C100200070782000728A02000000000014
:1045C00000000600A100200040072100728A0200BE
:1045D0000000000061042000C00C2100728A02006B
:1045E00000000000A1012000E0072100188A02005D
:1045F00000000000A0408000020320000280B900FB
:104600004002B000C292200060007900000001006A
:10461000A100200080092100188A0200000000008B
:10462000004020004F000700001020004D00070050
:10463000002020004B000700000420004900070074
:10464000000820004700070090A228009A6D020091
:10465000000000004100200020112100188A020003
:104660000000000021E3A800A0C0B300948802006D
:10467000000000000A70020000000000110020008D
:10468000B0372000188A02000000000090C0B3007C
:104690000E7102000000000090C0B3009488020078
:1046A000000000000A70020000000000110020005D
:1046B000B0372000188A02000000000090C0B3004C
:1046C0000E71020000000000C0C0B3009488020018
:1046D000000000000A70020000000000110020002D
:1046E000B0372000188A02000000000090C0B3001C
:1046F0000E71020000000000B0C0B30094880200F8
:10470000000000000A7002000000000011002000FC
:10471000B0372000188A02000000000090C0B300EB
:104720000E7102000000000021E3A90000402000FB
:1047300017000700001020001500070000202000CF
:1047400013000700000420001100070000082000EB
:104750000F00070090A228009A6D020000000000E0
:1047600000000600411680008080600004003200D6
:1047700020B52800826D0200000000000300370011
:1047800050B52800826D0200000000000000060005
:1047900051168000808060000400320080B528003F
:1047A000826D02000000000003003700B0B5280051
:1047B000826D02000000000000000600881F7800E3
:1047C000806780000000E8000080FB0080678800B0
:1047D00070FD070085FC07000000E900E30F5000B2
:1047E00002003E00904088000D0037000004EB00FE
:1047F000986788002102200070812000728A0200E0
:104800000000000088017800420020001100200014
:1048100010002000E2FD07000000E9009040880041
:104820002101200090832000728A02000000000015
:104830004F04780000000600881F78008067800021
:104840000000E8000080FB008067880051FD070041
:1048500066FC07008040E900E9CF500003003E00FD
:1048600000812000014878000D0037000004EB00B3
:1048700098678800D108200060872000728A0200B3
:104880000000000088017800A20020001100200034
:1048900090002000C2FD0700018120008048E9004F
:1048A0000044EB000081200091C0B30090CF1000C5
:1048B00010003A0037FD07004CFC07000044780068
:1048C0000004E0000B003A000004EB009867880049
:1048D000E0B528009A6D0200000000008801780011
:1048E000F2FF27008800780020022000ACFD0700BE
:1048F000004478004101200030902000728A0200BC
:104900000000000011012000A0192100728A02009D
:10491000000000006C700200000000000004E000D5
:10492000FCFF32000081200091C0B30090CF100046
:1049300003003A00084078002471020000000000E3
:104940004A7002000000000008C2B300FA700200C2
:1049500000000000884F5000FCFF3A004F04780030
:1049600000000600575249005445200042495400B7
:104970003A2020002A6E650078742000636C6F0076
:10498000636B2000285E2900207769006C6C200092
:1049900075736500207468006973200076616C008F
:1049A00075654E006F2064006576690063652C00B4
:1049B0002074720079202800414C4100524D29009A
:1049C000205345004152430048206D00616372004E
:1049D0006F206600697273007441440044524500C0
:1049E000535320004D414300524F200020302E00F1
:1049F0004D616300726F20006D656E00754D610042
:104A000063726F002020200020203100574952009F
:104A10004520610064647200657373000D0A200014
:104A200020202A003157490052452000524F4D00A6
:104A300020434F004D4D41004E4420004D41430066
:104A4000524F73003A0D0A00203531002E524500B6
:104A500041442000524F4D0020283000783333006D
:104A600029202A00666F7200207369006E676C004F
:104A700065206400657669006365200062757300D7
:104A80000D0A200038352E004D41540043482000C7
:104A9000524F4D00202830007835350029202A005B
:104AA000666F6C006C6F770065642000627920008F
:104AB00036346200697420006164640072657300BA
:104AC000730D0A0020323000342E53004B49500041
:104AD00020524F004D202800307843004329200009
:104AE0002A666F006C6C6F00776564002062790045
:104AF00020636F006D6D61006E640D000A2032004E
:104B000033362E00414C4100524D200053454100A8
:104B1000524348002028300078454300290D0A0000
:104B200020323400302E53004541520043482000CB
:104B3000524F4D00202830007846300029414C006B
:104B400041524D0020534500415243004820280067
:104B50003078450043295300454152004348200026
:104B60002830780046302900446576006963650086
:104B70002049440073206100726520006176610065
:104B8000696C6100626C650020627900204D410013
:104B900043524F002C207300656520002830290007
:104BA0002E52450041442000524F4D002028300035
:104BB00078333300293A20004D4154004348200007
:104BC000524F4D00202830007835350029534B00D6
:104BD00049502000524F4D002028300078434300B8
:104BE00029556E006B6E6F00776E20006D6163005B
:104BF000726F2C002074720079203F00206F7200C9
:104C000020283000292066006F72200068656C0043
:104C10007042550053205200455345005420570020
:104C200061726E00696E67003A202A0053686F0057
:104C3000727420006F7220006E6F200070756C001F
:104C40006C2D750070202A004E6F20006465760080
:104C500069636500206465007465630074656400C1
:104C60002044530031385300323020004869670037
:104C7000682050007265730020446900672054006A
:104C8000686572006D4453003138420032302000B4
:104C900050726F00672052006573200044696700FE
:104CA0002054680065726D00445331003832320080
:104CB000204563006F6E200044696700205468003F
:104CC00065726D0044533200343034002045630077
:104CD0006F6E7200616D200074696D006520430085
:104CE00068697000445332003433310020314B0086
:104CF0002045450050524F004D556E006B6E6F00C1
:104D0000776E2000646576006963650050574D003A
:104D100020646900736162006C656400314B480077
:104D20007A2D34002C303000304B48007A2050006F
:104D3000574D46007265710075656E0063792000FD
:104D4000696E20004B487A00205072006573630042
:104D5000616C65003A505200323A44007574790033
:104D600020637900636C650020696E0020252000B7
:104D700050574D002061630074697600654552000C
:104D8000524F52003A205000574D2000616374008A
:104D9000697665002C20670020746F00206469002C
:104DA000736162006C6541005558200046726500D1
:104DB000717565006E6379003A20410055582000F6
:104DC000494E500055542F0048492D005A41550076
:104DD000582048004947480041555800204C4F0092
:104DE00057564F004C544D004554450052204D003D
:104DF0004F444500564F4C00544147004520500059
:104E0000524F4200453A200056457200726F7200C0
:104E100028292000406C69006E653A00204070002F
:104E2000676D730070616300653A200062797400F9
:104E300065732E00546F6F00206C6F006E67210049
:104E400053796E007461780020657200726F720091
:104E50004E6F200045455000524F4D004572610095
:104E600073696E0067646F006E6553006176690058
:104E70006E672000746F2000736C6F00742049000F
:104E80006E7661006C69640020736C006F744C0076
:104E90006F616400696E6700206672006F6D2000AC
:104EA000736C6F007420450052524F00523A20003C
:104EB000636F6D006D616E00642068006173200097
:104EC0006E6F20006566660065637400206865008B
:104ED00072654100434B4E0041434B004932430051
:104EE000205354004152540020424900544932009A
:104EF00043205300544F500020424900544932008F
:104F000043206D006F6465003A0D0A0020312E00C9
:104F100020536F0066747700617265000D0A2000EF
:104F2000322E200048617200647761007265530080
:104F3000657420007370650065643A000D0A2000F6
:104F4000312E20007E354B00487A0D000A203200B9
:104F50002E207E0035304B00487A0D000A203300A9
:104F60002E207E00313030004B487A000D0A2000A0
:104F7000342E20007E343000304B48007A574100F8
:104F8000524E49004E473A002048410052445700D3
:104F900041524500204932004320690073206200DD
:104FA000726F6B00656E20006F6E20007468690080
:104FB000732050004943210020285200455620000C
:104FC00041332900536574002073700065656400E7
:104FD0003A0D0A0020312E0020313000304B4800BD
:104FE0007A0D0A0020322E0020343000304B480069
:104FF0007A0D0A0020332E0020314D00487A4900F6
:1050000032432000286D6F00642073007064290013
:105010003D28200020302E004D616300726F20007B
:105020006D656E00750D0A0020312E003762690033
:1050300074206100646472006573730020736500FE
:1050400061726300680D0A0020322E00493243006D
:1050500020736E00696666006572530065617200B8
:10506000636869006E672000493243002061640074
:1050700064726500737320007370610063652E00B5
:1050800020466F00756E64002064650076696300D9
:105090006573200061743A00536E690066666500AE
:1050A000722842004153490043295200656164005F
:1050B00079612F00412F400020636F006E747200F1
:1050C0006F6C73002041550058207000696E6100BC
:1050D0002F412F00402063006F6E7400726F6C00D0
:1050E0007320430053207000696E43006F6D6D00A4
:1050F000616E6400206E6F0074207500736564003B
:1051000020696E0020746800697320006D6F640070
:10511000655075006C6C2D00757020007265730011
:10512000697374006F727300204F4600465075001B
:105130006C6C2D00757020007265730069737400CB
:105140006F727300204F4E0053656C00662D740023
:105150006573740020696E00204869005A206D0054
:105160006F646500206F6E006C79520045534500F6
:1051700054424F004F544C004F41440045524100AF
:1051800055582000494E500055542F0048492D00D5
:105190005A2C200052454100443A2000504F5700FD
:1051A0004552200053555000504C490045532000B3
:1051B0004F4E50004F57450052205300555050005D
:1051C0004C49450053204F0046464400415441009D
:1051D00020535400415445003A204400454C4100BE
:1051E0005920750073575200495445003A20520027
:1051F000454144003A2043004C4F43004B2C2000D3
:1052000031434C004F434B002C20300044415400AC
:1052100041204F005554500055542C00203144007B
:1052200041544100204F550054505500542C20004B
:1052300030202A0070696E0020697300206E6F00B4
:1052400077204800695A43004C4F43004B205400DC
:1052500049434B00533A200052454100442042004C
:1052600049543A00205379006E746100782065003B
:1052700072726F00722061007420630068617200B6
:1052800020782E0020657800697428007769740002
:10529000686F75007420630068616E00676529009F
:1052A0006E6F20006D6F64006520630068616E00A2
:1052B000676523003A204E006F2073006F6674000C
:1052C00077617200652072006573650074206F005D
:1052D0006E207600342C2000757365002074680001
:1052E0006520720065736500742062007574740037
:1052F0006F6E2E004E6F6E006578690073746500E6
:105300006E74200070726F00746F63006F6C210008
:10531000782E200065786900740D0A00496E7600C9
:10532000616C690064206300686F690063652C002C
:105330002074720079206100676169006E44450045
:10534000564944003A68740074703A002F2F640084
:10535000616E670065726F0075737000726F740024
:105360006F747900706573002E636F006D2A2D00D5
:105370002D2D2D002D2D2D002D2D2D002A4F7000AF
:10538000656E200064726100696E20006F757400A4
:105390007075740073202800483D4800692D5A003C
:1053A0002C204C003D474E0044294E006F726D008A
:1053B000616C20006F757400707574007320280094
:1053C000483D33002E3376002C204C003D474E00E4
:1053D00044294D0053422000736574003A204D006B
:1053E0004F535400207369006720620069742000E5
:1053F0006669720073744C00534220007365740038
:105400003A204C0045415300542073006967200046
:1054100062697400206669007273740020426F0034
:105420006F746C006F61640065722000762031003B
:105430002E20480045580D000A2032002E2044003E
:1054400045430D000A2033002E204200494E0D0036
:105450000A2034002E205200415744006973700026
:105460006C61790020666F00726D610074207300BA
:10547000657456006F6C740061676500206D6F0085
:105480006E6974006F7273003A203500563A20003E
:10549000207C2000332E3300563A2000207C200050
:1054A000565055004C4C5500503A2000536574003E
:1054B00020736500726961006C2070006F72740067
:1054C00020737000656564003A20280062707300E4
:1054D000290D0A0020312E0020333000300D0A0043
:1054E00020322E002031320030300D000A203300EF
:1054F0002E203200343030000D0A2000342E2000DF
:1055000034383000300D0A0020352E0020393600A6
:1055100030300D000A2036002E20310039323000A4
:10552000300D0A0020372E00203338003430300090
:105530000D0A2000382E20003537360030300D009F
:105540000A2039002E2031003135320030300D0074
:105550000A3130002E20420052472000726177004D
:10556000207661006C75650041646A007573740093
:1055700020796F0075722000746572006D696E008D
:10558000616C410072652000796F750020737500B1
:1055900072653F002043460047313A0020434600F1
:1055A00047323A00285C2D002F5F5C002D2928002F
:1055B0005C5F2F002D295300656C6500637420002B
:1055C0006F757400707574002074790070653A000E
:1055D0000D0A2000312E20004F7065006E206400FF
:1055E000726169006E202800483D4800692D5A000C
:1055F0002C204C003D474E0044290D000A2032006B
:105600002E204E006F726D00616C200028483D0016
:10561000332E3300562C20004C3D47004E442900C9
:1056200052325700202873007064200068697A00A5
:10563000293D2800202030002E4D610063726F004C
:10564000206D65006E750D000A2031002E49530053
:105650004F37380031362D003320410054520D00B1
:105660000A2032002E4953004F37380031362D00C2
:10567000332070006172730065206F006E6C7900DA
:1056800049534F002037380031362D003320410078
:10569000545220002852450053455400206F6E009C
:1056A00020435300290D0A00524553004554200061
:1056B00048494700482C2000434C4F00434B2000F2
:1056C000544943004B2C20005245530045542000C0
:1056D0004C4F570049534F002037380031362D00CA
:1056E0003320720065706C007920280075736500A6
:1056F0007320630075727200656E7400204C530055
:105700004220730065747400696E6700293A2000B6
:1057100050726F00746F63006F6C3A002073650005
:10572000726961006C332000776972006532200075
:10573000776972006552460055756E006B6E6F009A
:10574000776E5200656164002074790070653A00DC
:1057500020746F0020656E006476610072696100DC
:10576000626C6500206C65006E67740068446100BF
:1057700074612000756E690074733A00206E6F00CA
:1057800020696E0064696300617469006F6E440093
:105790006174610020756E00697420006C656E0094
:1057A000677468002028620069747300293A200039
:1057B00043532000454E4100424C450044435300B2
:1057C00020444900534142004C45440052335700A5
:1057D000202873007064200063736C0020686900E7
:1057E0007A293D00282029000D0A440069736300CE
:1057F0006F6E6E006563740020616E007920640036
:1058000065766900636573000D0A43006F6E6E0074
:10581000656374002028560070752000746F2000A6
:105820002B355600292061006E6420002841440079
:10583000432074006F202B00332E33005629430081
:1058400074726C00415558004D4F440045204C0087
:1058500045445000554C4C005550200048505500D0
:105860004C4C550050204C005652450047414400D6
:10587000432061006E64200073757000706C7900C5
:1058800035565600505533002E33560041444300E0
:1058900042757300206869006768420075732000D4
:1058A00048692D005A203000427573002048690075
:1058B0002D5A2000314D4F0044452000616E640098
:1058C00020565200454720004C4544007320730089
:1058D000686F75006C642000626520006F6E2100A7
:1058E000466F75006E64200020657200726F720052
:1058F000732E4D004F534900434C4B004D4953000C
:105900004F435300204F4B0020464100494C530069
:10591000657420007370650065643A000D0A20000C
:10592000312E200033304B00487A0D000A2032001F
:105930002E20310032354B00487A0D000A2033000A
:105940002E20320035304B00487A0D000A203400FA
:105950002E2031004D487A00436C6F00636B2000AD
:10596000706F6C006172690074793A000D0A200052
:10597000312E200049646C0065206C006F77200098
:105980002A646500666175006C740D000A2032009F
:105990002E204900646C65002068690067684F002C
:1059A0007574700075742000636C6F00636B200069
:1059B00065646700653A0D000A2031002E20490019
:1059C000646C650020746F00206163007469760068
:1059D000650D0A0020322E002041630074697600B4
:1059E000652074006F206900646C6500202A6400E3
:1059F00065666100756C7400496E700075742000F6
:105A000073616D00706C65002070680061736500E3
:105A10003A0D0A0020312E00204D690064646C00AC
:105A200065202A006465660061756C00740D0A00CB
:105A300020322E0020456E0064535000492028007B
:105A40007370640020636B00702073006B6520002E
:105A5000736D7000206373006C206800697A290000
:105A60003D28200020302E004D616300726F200021
:105A70006D656E00750D0A0020312E00536E6900B1
:105A800066662000435320006C6F77000D0A2000EB
:105A9000322E53006E696600662061006C6C200037
:105AA0007472610066666900632D7000202D6600C7
:105AB000202A42007974650073206400726F7000C0
:105AC000706564002A464100494C4500442C200082
:105AD0004E4F200044415400414461007461200055
:105AE00062697400732061006E642000706172004E
:105AF000697479003A0D0A0020312E0020382C00FC
:105B0000204E4F004E4520002A64650066617500F6
:105B10006C7420000D0A2000322E2000382C20004A
:105B2000455645004E200D000A2033002E20380037
:105B30002C204F00444420000D0A2000342E200069
:105B4000392C20004E4F4E00455374006F702000DA
:105B500062697400733A0D000A2031002E20310072
:105B6000202A640065666100756C74000D0A2000CF
:105B7000322E200032526500636569007665200090
:105B8000706F6C006172690074793A000D0A200030
:105B9000312E200049646C0065203100202A640009
:105BA00065666100756C74000D0A2000322E2000BD
:105BB00049646C0065203000554152005420280093
:105BC00073706400206272006720640062702000BD
:105BD0007362200072787000206869007A293D00A5
:105BE00028202000302E4D00616372006F206D0070
:105BF000656E75000D0A2000312E540072616E0032
:105C00007370610072656E007420620072696400D6
:105C100067650D000A2032002E4C69007665200071
:105C20006D6F6E0069746F00720D0A0020332E00D4
:105C3000427269006467650020776900746820001B
:105C4000666C6F00772063006F6E7400726F6C007B
:105C50000A0D2000342E410075746F00204261004F
:105C6000756420004465740065637400696F6E009C
:105C70005541520054206200726964006765520009
:105C800065736500742074006F2065007869740086
:105C9000526177002055410052542000696E700017
:105CA0007574550041525400204C4900564520005F
:105CB00044495300504C4100592C20007D20540091
:105CC0004F205300544F50004C495600452044008B
:105CD000495350004C415900205354004F5050003C
:105CE0004544570041524E00494E47003A2070004B
:105CF000696E7300206E6F0074206F0070656E0017
:105D00002064720061696E0020284800695A2900E9
:105D100020524500564944003A0D0A00496E76006B
:105D2000616C690064206300686F690063652C0022
:105D30002074720079206100676169006E6D7300E4
:105D4000525320004C4F57002C2043004F4D4D0024
:105D5000414E4400204D4F0044455200532048001E
:105D6000494748002C20440041544100204D4F0039
:105D7000444541006464720065737300206F6600DF
:105D8000205043004638350037343F0054686900DE
:105D900073206D006F646500207265007175690085
:105DA0007265730020616E00206164006170740090
:105DB00065724C004344200074797000653A0D0010
:105DC0000A2031002E204800443434003738300097
:105DD0002028750073696E00672050004346380024
:105DE0003537340020494F002065780070616E001F
:105DF00064657200294C43004420280074797000C7
:105E00002061640064722900203D200028202000C9
:105E1000302E4D00616372006F206D00656E75005D
:105E20000D0A2000312E4C004344200052657300BF
:105E300065740D000A2032002E496E00697420003E
:105E40004C4344000D0A2000332E43006C65610072
:105E500072204C0043440D000A2034002E4375008C
:105E600072736F00722070006F73690074696F0045
:105E70006E206500783A280034292000300D0A0091
:105E800020362E0057726900746520007465730017
:105E900074206E00756D6200657273002065780075
:105EA0003A28360029203800300D0A0020372E000D
:105EB0005772690074652000746573007420630074
:105EC0006861720061637400657273002065780018
:105ED0003A283700292038003044690073706C007C
:105EE000617920006C696E0065733A000D0A20002C
:105EF000312E200031200D000A2032002E204D00CE
:105F0000756C740069706C0065494E00495443001B
:105F10004C4541005243550052534F00522053000C
:105F200045544E006F204100434B2C002063680015
:105F300065636B00206164006170740065724300EA
:105F40004C4B09004D4F53004909430053094D0084
:105F500049534F0050696E0073746100746573009B
:105F60003A474E00440933002E33560009352E00BF
:105F7000305609004144430009565000550941007C
:105F800055580900500950000950090049094900B5
:105F9000092D09004F574400092D09002D2D090036
:105FA00054784400092D09005278440053434C00B2
:105FB0000953440041092D00092D500047430900B1
:105FC00050474400092D09002D312E00284252006F
:105FD000290932002E28520044290900332E2800B6
:105FE0004F52290009342E0028595700290935003D
:105FF0002E2847004E290900362E2800424C290041
:1060000009372E0028505500290938002E2847004E
:1060100052290900392E28005754290009302E0032
:1060200028426C006B2947004E440900474E44004B
:1060300009414400430935002E30560009332E0033
:10604000335609005650550009415500580965005E
:106050007865630075746500203A20002061750042
:10606000746F7200616E670065202B004D487A00E6
:10607000292B6B00487A2900526177002076610055
:106080006C75650020666F00722042005247200048
:10609000284D490044493D0031323700295741001D
:1060A000524E49004E473A0020506F00737369000A
:1060B000626C65002062750066666500726F76002E
:1060C000657266006C6F7700416E7900206B650029
:1060D000792074006F206500786974005370610046
:1060E00063652000746F2000636F6E0074696E003A
:1060F00075654E00756D6200657220006F66200048
:106100006269740073207200656164002F77720009
:10611000697465003A204300533A0D000A203100AB
:106120002E204300530D0A0020322E00202F430062
:1061300053202A006465660061756C0074506F001E
:1061400073697400696F6E0020696E0020646500D9
:106150006772650065735300657276006F20610099
:10616000637469007665570061697400696E670041
:106170002061630074697600697479002E2E2E0008
:106180002A2A2000456172006C7920004578690058
:1061900074212A002A42610075643E0031366D0088
:1061A0003A20420050204300616E6E006F74200060
:1061B0006D6561007375720065203E002031360008
:1061C00030303000303030002C2044006F6E6500DD
:1061D0002E0A0D0043616C0063756C0061746500EC
:1061E000643A2000090A0D0045737400696D61006E
:1061F000746564003A20200009206200707320005A
:1062000047656E00657261006C09090009090900A3
:1062100050726F00746F63006F6C2000696E7400C1
:1062200065726100637469006F6E20002D2D2D0072
:106230002D2D2D002D2D2D002D2D2D002D2D2D0042
:106240002D2D2D002D2D2D002D2D2D002D2D2D0032
:106250002D2D2D002D2D2D002D2D2D002D2D2D0022
:106260002D2D2D002D2D2D002D2D2D002D2D2D0012
:106270002D2D2D002D2D2D002D2D2D002D2D2D0002
:106280002D2D2D002D2D2D002D2D2D002D2D2D00F2
:10629000203F09005468690073206800656C700035
:1062A0000909090028302900094C6900737420008D
:1062B0006375720072656E0074206D006163720018
:1062C0006F7320003D582F007C580900436F6E000B
:1062D0007665720074732000582F72006576650031
:1062E00072736500205809000928780029094D00BB
:1062F000616372006F207800207E090053656C0096
:10630000667465007374090009095B000953740021
:1063100061727400202309005265730065742000C7
:1063200074686500204250002020200009090900FF
:106330005D095300746F7000202409004A756D00D8
:10634000702074006F2062006F6F74006C6F6100CA
:106350006465720009097B0009537400617274005E
:10636000207769007468200072656100642026004F
:106370002F25090044656C006179200031207500EB
:10638000732F6D0073090900097D090053746F00B4
:10639000702061002F412F004009410055585000E6
:1063A000494E2000286C6F00772F4800492F52007B
:1063B0004541440029090900226162006322090065
:1063C00053656E0064207300747269006E6720006C
:1063D0006209530065742000626175006472610097
:1063E000746509000909310032332000632F43002E
:1063F000094155005820610073736900676E6D0094
:10640000656E74002028610075782F0043532900C1
:106410000909300078313200332064002F4409002C
:106420004D65610073757200652041004443200092
:10643000286F6E0063652F00434F4E00542E2900D5
:106440000930620031313000095365006E6420006C
:1064500076616C007565200066094D00656173000A
:10646000757265002066720065717500656E630067
:1064700079090900720952006561640020672F00E4
:1064800053094700656E6500726174006520500015
:10649000574D2F0053657200766F0900092F0900D0
:1064A000434C4B002068690020680900436F6D0071
:1064B0006D616E006468690073746F007279090021
:1064C00009095C0009434C004B206C006F206900F7
:1064D00009566500727369006F6E69006E666F0021
:1064E0002F7374006174750073696E00666F090024
:1064F000095E0900434C4B0020746900636B200067
:106500006C2F4C0009426900746F72006465720060
:1065100020286D0073622F004C53420029090900A6
:106520002D09440041542000686920006D09430092
:1065300068616E00676520006D6F64006509090081
:10654000095F090044415400206C6F00206F09006E
:1065500053657400206F75007470750074207400AA
:1065600079706500090909002E0944004154200092
:1065700072656100642070002F50090050756C0036
:106580006C7570002072650073697300746F72001F
:10659000732028006F6666002F4F4E0029092100E6
:1065A000094269007420720065616400207309006B
:1065B000536372006970740020656E0067696E0035
:1065C00065090900093A09005265700065617400A7
:1065D00020652E00672E2000723A310030207600B0
:1065E000095368006F772000766F6C0074732F007A
:1065F000737461007465730009093B000942690006
:1066000074732000746F200072656100642F77003E
:1066100072697400652065002E672E0020307800B6
:1066200035353B00322077002F5709005053550075
:1066300020286F0066662F004F4E290009093C0094
:10664000783E2F003C783D00203E2F003C303E003D
:106650000955730065726D00616372006F207800E8
:106660002F617300736967006E2078002F6C6900DA
:1066700073742000616C6C000371800084E2200060
:10668000E3407A0030C8B30080CF50000D003A00DC
:106690000301E80002718800E2407A0000CEB300F6
:1066A00080CF500007003E000380E8000400400057
:1066B00001CEB3000201E800B0CF1000FDFF3600AC
:1066C00002718800000006000003780080E22000CC
:1066D0009040780000CEB30080CF500017003E00FD
:1066E000140037008180FB0000F22F008082400000
:1066F0006400420082E22000E0407900C808DD002A
:1067000065004200604079000080FB00808040000E
:10671000810F53001700320005824100E30142005F
:1067200080E22000E340780000CEB30080CF50002C
:10673000ECFF3E008081EB000E0037008180FB0003
:1067400000F22F008082400090E220001080FB00C9
:106750004800DD00A1E220009180FB000100400024
:106760008001EB00800F5300020032008001EB003B
:10677000E9FF37000300780000000600881F78005A
:106780000371800088E2200063417C0080C2B30076
:10679000804F51000C003A000300E80000718800AF
:1067A000BE0007000002780002718000E2407C0019
:1067B00090C2B30080CF500080003A000200E80091
:1067C000007188007D003700F0CBB300004041002D
:1067D000F94F500009003E000280FB00000040001D
:1067E000E1F72F000100400001DC2000608278000A
:1067F0000300E800007188007000370000C8B30093
:10680000804F5100650036000300E80000718800E9
:1068100070C9B300804F51003A0032000A003E00B8
:1068200063405000804F51001600320000C0E80065
:10683000804F51002A00320063405000804F5100C9
:1068400054003A0018003700A0C9B300804F51002F
:106850003500320004003E0000C0E900804F5100C6
:106860004C003A0038003700B0C9B300804F5100E7
:106870003000320000C0E800804F510045003A006F
:1068800013003700A0408000020320000280B900FE
:106890006A004000C2922000600079000000010000
:1068A0000002780045003700A0408000020320006D
:1068B0000280B90068004000C292200060047900A4
:1068C0007600070008000100000278003B00370056
:1068D0006047020000000000000278003700370027
:1068E000A0408000020320000280B9007400400034
:1068F000C2922000600079000000010000027800D0
:106900002E003700A0408000020320000280B90062
:1069100078004000C2922000600079000000010071
:106920000002780025003700C2C2BF00610260008B
:1069300022003700CBC2BF004300DE0061006000D0
:106940000082EA001D00370021E3A800C0C0B300A8
:1069500094880200000000000002780021E3A900F2
:10696000160037006A20B9000281FB0000014100D7
:1069700000FD2F00000241008301E800354178004E
:1069800000404100E94F5000F6FF360003718800D7
:106990000A0037000002EB000800370000CDB3000A
:1069A00000404100E94F5000FAFF3E0090E2200015
:1069B000808241000002EB00EAFF3700040078000B
:1069C0004F04780000000600889FBE008A9FBE002A
:1069D0006AFF070000047800F9C2B3006AC2B3007E
:1069E000CBC7B3000271800080E22000E240780053
:1069F000A0C2B30080CF50000600320089CF500003
:106A0000040032008ACF5000020032008BCF5000C9
:106A10001E003A000200E80000718800A0C2B30026
:106A200080CF50000900320003003E008ACF5000A2
:106A3000ECFF3A000F00370089CF5000070032000A
:106A40008BCF5000E7FF3A000D0037004BFF0700E7
:106A500000C0B90000047800E2FF370047FF0700DC
:106A600000017800110009000204D8000004780039
:106A7000DCFF370041FF070000046400D9FF370046
:106A80003EFF070000047400D6FF370008007800BE
:106A90004F05BE004F04BE0000000600889FBE00E8
:106AA0008A9FBE00C8FF07000004780089E220002A
:106AB000EBC3B300DAC3B30002718000E2C07C0014
:106AC000D0C2B30080CF50000A00320000C0E900FD
:106AD00080CF5000070032007140400080CF50004E
:106AE000040032008BCF5000020032008ACF5000E9
:106AF00054003A000200E80000718800C0C3B300EF
:106B000080CF50002800320007003E007140500046
:106B100080CF50000C00320000C0E80080CF500051
:106B2000E5FF3A00050037008ACF50003E003200F2
:106B30008BCF5000E0FF3A0006003700A2FF0700AD
:106B400000045400DCFF37009FFF070000044400EE
:106B5000D9FF37000280E80060C07C008A4F5000F7
:106B60000A003A0098FF07008000EB00800F5400F5
:106B7000010039001100200001047800007180003C
:106B80000000E80000718800CBFF37008EFF07008F
:106B90008000EB00800F540001003600110020003F
:106BA00001047800C4FF37000280E80060C07C0068
:106BB0008B4F500009003A0083FF070000006C0073
:106BC0008000EA00808070004F0CDE0000718000C1
:106BD0000000E80000718800B7FF37008A4F5000BE
:106BE0000A003A0078FF07008000EB00800F540095
:106BF00001003E00110020000104780000718000B7
:106C00000000E80000718800ABFF37006EFF07004E
:106C10008000EB00800F54000100310011002000C3
:106C200001047800A4FF370067FF07000800680030
:106C30008000EA0080807000CF08DE0061841000D0
:106C40009DFF3700080078004F05BE004F04BE00CE
:106C500000000600E4874700889FBE008A9FBE00B0
:106C60008C9FBE008E1F78000000EB000071880032
:106C7000107188002071880030718800A081200088
:106C80001080A00002DC20000000EB0043DF2000A9
:106C900000197800828F5100FDFF3A0080BF9F00ED
:106CA0008BE22000AE81200002718000E2C07D00F6
:106CB000F0CDB30080CF500002003E002A0020003B
:106CC000D20237008180FB0000F22F0000864000D6
:106CD0000200E800E0C07D00C808DD000280E80096
:106CE00060C07D000080FB008080700081BF9F003D
:106CF000097180006380440060C07D000080FB005B
:106D0000010020000008B1000180B1001202200043
:106D1000820F5000E08F580023003E000060010009
:106D200023003700300037001F0037001E003700F7
:106D30004E003700560037006A00370079003700F0
:106D40007D003700C3003700F90037001600370018
:106D5000350137005E013700A3013700B20137006B
:106D6000A6013700C8013700BB013700D201370048
:106D70000D0037005A023700420237000A00370080
:106D800009003700F3013700E501370077023700CB
:106D900083023700D5013700010237001C0237009B
:106DA00087023700930237003A0020009202370032
:106DB00066804400007188006480440060C47D00E7
:106DC0000884FB00F0FB2F000004440033FF0700A1
:106DD0000804440001DC200000B4780026FE07000F
:106DE0008001EB00BB023700648044000071880022
:106DF0002AFF07000000E000A802320002718000B4
:106E000062C07D008200E800017188008001EB0013
:106E100021C8B300814F5000AE023A000280E90061
:106E20000071880013002000AA0237008100E800EA
:106E30009241780030C8B30080CF51000600320084
:106E40000201E80000CEB30080CF5100F7FF36000A
:106E50000171880094FF3700017188000180E9000A
:106E600000718800130020009A02370064804400FB
:106E70000071880009FF070013FE0700E10F4000C2
:106E800092023200007188008001EB00910237000D
:106E9000648044000071880023718000E98F5100F4
:106EA000020034007A0020005802370003814100BC
:106EB0000C0040000000E90041DF200000B1780034
:106EC0000300E80020718800F4FE0700FEFD0700C3
:106ED000E10F40007D023200007188008001EB006C
:106EE0007C02370020B92800826D020000000000FB
:106EF000207180000000E00002003A008A002000BB
:106F0000420237000000E9002071880000004000C4
:106F100041DF200060807800007188008001EB0074
:106F20006C0237000C804400630040000071880050
:106F30008001EB0067023700648044000071880024
:106F40002DC2B300AA8120002C0037008D4F5100C4
:106F500016003A000300E8000071880083E2200078
:106F6000E0C0790082CF50000D003200A8812000DF
:106F7000830478001880A1000000E80000718800F8
:106F8000014078000E710200000000001880A0008F
:106F900000718000E0C07C008DCF5000F5FF3A000A
:106FA0000000E8000071880014003700F0CBB30047
:106FB00000404100F94F50000500360000C8B30002
:106FC00000404100F1C5B300814F500006003E0073
:106FD000B2FE07001A80A100146F0200000000003A
:106FE0001A80A00005003700B0C3B300804F5100E5
:106FF00002003A000300E80000718800037180007D
:1070000080E2200063417800F0CDB300804F510052
:1070100003003E0030C8B300804F5100CBFF3A0060
:107020000300E900E0C07D00B0C3B30080CF500092
:10703000050032001E80A10080C228009A6D020067
:10704000000000001E80A0008BFD07008001EB0007
:10705000200237001E80A100648044000071880077
:1070600081E2200060C1780020C2B300804F51004F
:1070700012003A006580440000718800E0C078008A
:1070800082CF50000B00320088E2200029C2B300FA
:107090000000E80000718800014078000E710200D5
:1070A0000000000000718000E0407C0089CF5000AB
:1070B000F7FF3A000000E8000071880002718000CC
:1070C000E2C07D003A002000C0C2B30080CF500073
:1070D00003003A000200E800007188000005EB00A0
:1070E0000071800060C47D000884FB00F0FB2F006D
:1070F000000444008001EB00F2FF270083007800C9
:1071000003007800D01F02000000000008044400C3
:1071100001DC200000B47800007180000000E8006D
:107120000071880054FD07001E80A000B5013700E3
:10713000E480440001718800107180004A00200042
:10714000E30F500003003C000000E80010718800CD
:107150000005EB0061C07D000084FB001071800021
:107160006600B9000080E80002FC2F000201440024
:1071700083E0200002B0790065804400007188003F
:10718000E0C07D00D0C3B30080CF500002003200C9
:107190003A00200008003700668044000071880033
:1071A0003EFE070088004400E2F72F008280400086
:1071B00002DC20008030790000718000E0C07D009A
:1071C0000000E80000718800B0C8B30080CF500014
:1071D000020032003A0020000600370018718000DB
:1071E0002EFE07006644B9006404440081E02000DC
:1071F00000B4780003718000E3C07D00F0CDB300DF
:1072000080CF500002003E003A002000040037000A
:10721000107180006600B90082E020000331780020
:1072200015FD0700770137006480440060C07D00D1
:107230000081FB0000FC2F0000064100E5834400B4
:1072400007718800117180005A0020000100E000E1
:107250001D003500810278000002EB005A0020007A
:10726000A3E02000F0FB2F0000004100800440005C
:10727000930F56000C003A0008DC200069017C00E6
:1072800013009000800F510005003D000200E8004F
:1072900080347C00F3BB97000005EB000200370050
:1072A0008500E9000005EB000402E800E6814100EA
:1072B000810F520002003C0081027800ECFF370091
:1072C0001171880007718800EBFC07004D01370041
:1072D000E4814400037188000005EB0030718000F8
:1072E0000000E0001A003A00640137008000EB0063
:1072F00034F22F0065F22F0082E22000E6C8B300CE
:107300000080FB0000804000840040000500400039
:1073100060407900864F50000500320061407900DE
:107320000004E00009003200F5FF37008000EB00A8
:1073300061C07D000004E000040032006480400071
:10734000307188000005EB00010037009A00200032
:10735000317180000171880063C47D000884FB00E6
:10736000F0FB2F000004440004FD07000804440063
:1073700001DC200000B478000271800032718800C6
:107380006580440000718800E2C07D00C0C2B30087
:1073900080CF500002003A000200E80030718800FF
:1073A0003271800083E22000E2C0790000CEB30099
:1073B00080CF50000A00360063004100E0C0790031
:1073C000E0C8B30080CF5000030032000000EB00A3
:1073D000307188000200370064004100307188007D
:1073E000A5FC0700070137000C8044006300400043
:1073F000007188008001EB00360137006480440092
:1074000000718800A0408000020320000280B900C3
:10741000C3922000630078000000010096FC070082
:107420008001EB002B01370064804400007188006C
:10743000A0408000020320000280B9000080E80024
:10744000C392200060807900000001008AFC0700E0
:107450008001EB001F013700648044000071880048
:10746000A0408000020320000280B90064004000B8
:10747000C392200060807900000001007EFC0700BC
:107480008001EB0013013700648044000071880024
:10749000A0408000020320000280B9006600400086
:1074A000C3922000608079000000010072FC070098
:1074B0008001EB0007013700648044000071880000
:1074C000A0408000020320000280B9006800400054
:1074D000C39220006084790070FD0700080001005D
:1074E00065FC07008001EB00FA003700648044006F
:1074F0000071880069FD07000000E0000300320011
:107500002847020000000000020037004447020044
:107510000000000058FC07008001EB00ED00370080
:1075200064804400007188005CFD07000000E000FA
:1075300003003200C002A900C202A8000200370006
:10754000C002A900C202A9004BFC07008001EB00A9
:10755000E000370064804400007188004FFD0700A0
:107560000000E0000600320001B420001140780065
:107570000014A1000004A000804878000500370036
:1075800001B42000114078000014A1000004A00004
:107590008048780038FC07008001EB00CD00370000
:1075A00064804400007188003CFD0700505F880043
:1075B0000000E00002003D000000EB00505F88008A
:1075C00001FA2000505F8000810F5000010034005C
:1075D000515F8800605F8000E10F500002003C00B6
:1075E00020002000605F880031062000605F80007E
:1075F000810F500001003400615F8800943F020059
:10760000000000001CFC07008001EB00B100370007
:10761000648044000071880020FD070000017800AC
:10762000605F8800505F80000000E00002003D00C5
:107630000000EB00505F880001FA2000505F8000DE
:10764000810F500001003400515F8800E10F5100AC
:1076500002003C0020002000605F8800310620000E
:10766000605F8000810F500001003400615F88007E
:10767000943F020000000000FFFB07008001EB00C8
:1076800094003700648044000071880003FD070007
:107690000000E00008003200A0408000020320004B
:1076A0000280B90070004000C39220006080790021
:1076B0000000010007003700A04080000203200006
:1076C0000280B90072004000C392200060807900FF
:1076D00000000100E8FB07008001EB007D0037009F
:1076E0006480440000718800ECFC0700E10F50004A
:1076F0000C003200E20F5000120032000000E000E7
:1077000017003A00A0408000020320000280B90068
:107710006E004000C39220006080790000000100EC
:107720000F003700A0408000020320000280B90053
:107730006C004000C39220006080790000000100CE
:1077400007003700A0408000020320000280B9003B
:1077500076004000C39220006080790000000100A4
:10776000C5FB07008001EB005A003700648044002D
:1077700000718800C9FC07000000E000030032002F
:10778000C962A800CB62A90002003700CB62A90041
:10779000C962A900B8FB07008001EB004D0037006B
:1077A0006480440000718800BCFC07009E890200D0
:1077B00000000000B0FB07008001EB00450037002F
:1077C0006480440000718800B4FC0700A24080007F
:1077D000010320000191B9007C014100C392200007
:1077E000E280790001000100A3FB07008001EB00AB
:1077F000380037001A0020000C804400630040006D
:10780000007188000A00E00027FD32001E80A10000
:10781000E10F55003200320061002000C037200027
:10782000188A0200000000000A007800146F0200AD
:10783000000000008100200020382000188A02008B
:10784000000000000FB89700146F02000000000055
:10785000B1002000A0382000188A020000000000BB
:1078600000718000146F02000000000080C2280038
:107870009A6D02000000000019003700B1E22000FC
:10788000E0C8B300914F1000A8FE32001B40780002
:107890000004E00095FE3A00ACFE37000171800064
:1078A00083E2200061C1790030C8B300804F5100ED
:1078B0006AFD320000CEB300804F5100FAFC3E005A
:1078C0000100E8000301400058FD37006A00200075
:1078D000CEFF37000300E00005FD3A00F2FC370060
:1078E0004F0778004F06BE004F05BE004F04BE0094
:1078F0004F00B10000000600881F780000047800E7
:1079000000C2B3000E710200000000000800780001
:10791000826D02000000000000C2B3000E71020080
:10792000000000004F04780000000600889FBE00A1
:107930000000EB000071880080E220001044780015
:107940000804E00030003200800478000804E00001
:1079500004003500084078000E71020000000000AD
:107960002300370000CEB300804F540012003600D1
:1079700080C228009A6D02000000000000718000A3
:107980000081E8000000E80060C07C004800DD00E5
:10799000E2C07C008180FB00010040000271880091
:1079A000146F02000000000000C2B3000E7102005C
:1079B000000000000E00370000C2B3000E7102008C
:1079C000000000000880FB000000400001F02F00D4
:1079D0000100400081AE200060807800826D0200CE
:1079E0000000000000C2B3000E71020000000000A1
:1079F000007180000000E8000071880060C47C0015
:107A00000804E000D1FF3A0080C228009A6D02000D
:107A100000000000007180000000E900146F020007
:107A2000000000007100200050392000728A02001E
:107A3000000000004F04BE00000006008001780036
:107A40008167800001027800104178000204E000A4
:107A500010003A000D003700E0BE200061407800C1
:107A6000804F510003003200846788000000EB0063
:107A70000D0037000100E8008080FB00816788006E
:107A8000534178000204E000F3FF3A0010002000A8
:107A900005003700E0BE200061407800804F5100B3
:107AA000F1FF3A00F3FF370000000600889FBE0098
:107AB0008A1F78008004EB0088AE20002A02200094
:107AC00018007800DDFF07000000E000040032002D
:107AD00000C8B30000C044000080FB000500370070
:107AE0008904E8000884E8008A8F5400F4FF3A0013
:107AF0000000EB004F0578004F04BE0000000600B8
:107B00002400FA00889FBE008A9FBE008C1F780068
:107B1000846780008400780073678000848F510040
:107B20000E003200E5BE2000F7C9B300F8CDB30067
:107B3000F60F200061C17A0007404100F94F500064
:107B400002003E000840610080F07A000100E80079
:107B500086006000818F5100F6FF3A00E0BE2000F1
:107B60006440780001CDB30001404000E94F50006F
:107B70009B003E0020FD2F000F0040000041EB0065
:107B8000EB80570002587800808F5000FDFF3A00CC
:107B9000F61C020000000000C880DE00B1D79F0084
:107BA000C0D79F00C8FA070000027800E10F40002C
:107BB0002100320080E22000644078000080FB0059
:107BC00031F22F0081004000004020008101500070
:107BD000848F510002003C00840078000B003700C5
:107BE0008100420080E220008080400000014200CD
:107BF0000000EB0084815100315978000000E8005A
:107C0000808F5100FCFF3A0080004200F03F2000CE
:107C1000808F500008003C0080E22000008040007F
:107C20008041EB0002402000035878008100E8000A
:107C3000828F5000FCFF3A00CA1E020000000000C4
:107C4000380020008004EB00210037000900E0002C
:107C50000E003A00CA1E02000000000093FF070059
:107C60008080FB000004E0000800320022FD2F00AD
:107C70000F01410001717C00010078007088B200A2
:107C80000000E900CF04DE000D00370082678000AD
:107C9000E0BE2000E240780020C2B30080CF500058
:107CA00001003A000900A20020FD2F000F00400053
:107CB00001707C000200E800F00FB20080678800CD
:107CC0000804E80040022000800F540076003200D3
:107CD0008167800070678000808F5000DBFF3A0072
:107CE000E30F540079003200E40F540077003200B3
:107CF000C0CDB30080444400A9D79F00BFD09700F7
:107D0000C808DD004FD097000080FB008083400052
:107D10000001EB008202780084E2200006CEB3006E
:107D200008F22F0062407A00864F500010003600A3
:107D30000080FB00880140000200E800E0407A007B
:107D4000C808DD000280E80060407A000080FB0087
:107D500080804000878F5000020031000280410087
:107D6000E30240000280410063014000EDFF370064
:107D70000200E000EBFF32008980FB0030F22F00B0
:107D800000824000850F51000800350081E220008C
:107D900081014100020042000100400023507800B0
:107DA0000201E900850F5100FCFF3D000400E000E6
:107DB0004600340080E22000008042008000EB009A
:107DC00022FD2F000F01410062C1780002587800A7
:107DD0008100E800810F52003C003200F8FF3700BC
:107DE00090C2280015FF07000000E00005003200E7
:107DF00098FB070080C228009A6D02000000000076
:107E000032003700D0C228000CFF07000000E0005D
:107E100002003200C5FE07002C00370020C32800F6
:107E200006FF07000000E00003003200A0812000F0
:107E30001090A1002500370070C32800FFFE070046
:107E40000000E000120032000005EB008CE2200090
:107E50000B4020008C0445000004EB003980FB003F
:107E6000A46F02000000000000C2B3000E71020007
:107E7000000000000804E800F00F5400F7FF3A008B
:107E8000700545008B0F550010003200F1FF3700E0
:107E9000D0C32800E9FE07000000E0000700320020
:107EA0000F0007000900370091002000C0392000B2
:107EB000728A02000000000004003700C1002000A8
:107EC000503A2000728A0200000000004F0678003D
:107ED0004F05BE004F04BE000080FA0000000600FF
:107EE00080E220000041EB0081222100025878004E
:107EF000810F5000FDFF3A0011CEB30080E2200058
:107F00000148780080C0EB0090E220000148780032
:107F1000A0E220000148780011CAB300B0E22000BE
:107F200001487800000006000000EB00800888008F
:107F3000F0088800E00C8800525F80000200E0003A
:107F400006003A00CAC6BF0001CEB300014060007F
:107F5000CAE6B700425E88002E003700E30F5100EA
:107F600004003C0010A1A8001081A800E00320003C
:107F700010003700FE0F510004003C0010A1A800C3
:107F80001081A900A00F20000A003700400F200038
:107F9000800F510004003C0010A1A9001081A8002E
:107FA000007D20000300370010A1A9001081A90066
:107FB00000E82300110009000280D8000000E90059
:107FC00060088800625F80000280B90042062000DD
:107FD000110009000280D800A26C20001241780034
:107FE00003CEB300034161006241B3000001FD0014
:107FF000CAE6B7000001FD00D00C8800C00C880064
:1080000060002000E00C880011E1A80020002000A2
:10801000405E880000000600889FBE008A9FBE0068
:108020008C1F78000004EB0088088800F80888009E
:10803000E80C8800405E8000E20F500010003A001B
:10804000CAC6BF0001CEB30001406000CAE6B70057
:10805000C1002000E02B2000728A02000000000016
:10806000485E8800806780000000E8000080FB0018
:10807000E1BE200060C078000004E0008B00320008
:10808000806780000000E8000080FB0080678800B7
:10809000CA1E020000000000F61C020000000000E2
:1080A00000047800CA1E020000000000F61C020056
:1080B00000000000CF80DE0000040200000000008D
:1080C0000005BE000001EB008800E900E0F9200097
:1080D000808F500001003E001200200082047800D2
:1080E0006011B8000A00BE00560402000000000043
:1080F0000000E0000800340002002000832C24006F
:108100000A00BE005A040200000000000000E00067
:1081100001003D008904E800E28F540011003200A4
:108120000004EB009867880011012000A02C2000BB
:10813000728A02000000000011012000B02D200012
:10814000188A0200000000008801780002FA20006E
:108150001100200020032000D01F020000000000BA
:1081600000047800E30F540004003E0010A1A800B2
:108170001081A800E003200010003700FE0F54001B
:1081800004003E0010A1A8001081A900A00F20004B
:108190000A003700400F2000800F540004003E000A
:1081A00010A1A9001081A800007D20000300370065
:1081B00010A1A9001081A90000E823001100090006
:1081C0000880D8000006E900E28F54000E0032005B
:1081D00001012000902F2000188A020000000000FA
:1081E0008001EB003206200083007800200320008D
:1081F000D01F020000000000CF80DE00000402005B
:10820000000000000005BE0002002000832C2400B6
:108210000A00BE005E040200000000000004BE0070
:108220006160B90000040200000000000C00E000E2
:1082300004003D000200200003782400E404020052
:10824000000000000001BE000800BE009E05020004
:10825000000000000606020000000000A26C2000E2
:108260001241780003CEB300034161006241B300C4
:108270000001FD00CAE6B7000001FD00D00C880037
:10828000C00C880060002000E00C88006C088800AA
:1082900011E1A800A100200090302000728A0200A5
:1082A0000000000020002000405E88004F0678009B
:1082B0004F05BE004F04BE0000000600889FBE00B0
:1082C0008A9FBE00405E8000E20F500005003A0029
:1082D000F101200030312000728A0200000000000D
:1082E00019023700F100200020332000188A020014
:1082F000000000000004EB00F808880088088800EF
:10830000C942A80086C6BF0001CEB300014060008C
:10831000A040B30086E6B700A003200080088800D4
:108320002C0207000002BE000803780088037800D2
:10833000F0FF2300010020006011B8000020E100E0
:1083400001A8E10002B0E10003B8E1000D00360031
:108350000605BE000404BE00C85DDD004850DE0016
:108360008B0570004855DD004848DE000A057000A6
:10837000C84CDD004840DE00890470004844DD0040
:1083800009003700B1002000A0132100188A020064
:1083900000000000A0002000800888000D020700F7
:1083A0000004BE006055B800F0F920000100200074
:1083B0006011B8000040E10001C8E10002D0E10016
:1083C00003D8E100070036000800BE004A6E020034
:1083D00000000000A0C828009A6D02000000000004
:1083E000D4013700E00F5400E08F5C00E00F5D0027
:1083F000E08F5D00CC013200B1002000A01321000D
:10840000188A02000000000008007800120207002D
:108410000002BE006033B80000A821006100200007
:108420006011B8000020E10001A8E10002B0E10005
:1084300003B8E1006A003600E00F5200E08F5A00F6
:10844000E00F5B00E08F5B00050035000400BE001C
:108450000601BE003C0602000000000014003700C8
:1084600010002000010020006011B800040060002E
:108470008580600006016100878161008703D1006B
:108480000683D3008582D3000482D30000007200EB
:108490008180720002017300838173003C06020038
:1084A000000000000001BE00E40402000000000023
:1084B0000001BE00703B2400A13B25005E040200C9
:1084C00000000000B4060200000000000205BE002B
:1084D0000004BE00046A2800150020006033B800C4
:1084E000EA070200000000004A6E020000000000DF
:1084F000E0C2B3000E71020000000000046A280010
:10850000150020006033B8000800BE000A01BE005C
:10851000F8070200000000000205BE000004BE00D3
:10852000F0702200010020006011B8000040E1005E
:1085300001C8E10002D0E10003D8E10003003E00E1
:1085400000C3B3000E71020000000000703E200066
:10855000010020006011B8000040E10001C8E10006
:1085600002D0E10003D8E10003003E0000C3B300E5
:108570000E71020000000000300620000100200003
:108580006011B8000040E10001C8E10002D0E10044
:1085900003D8E10003003E0000C3B3000E710200E7
:1085A0000000000090002000010020006011B800D1
:1085B0000040E10001C8E10002D0E10003D8E10081
:1085C00003003E0000C3B3000E7102000000000073
:1085D0000800BE00E46D0200000000004E013700FC
:1085E000B0E12E00110020006011B8000020E10071
:1085F00001A8E10002B0E10003B8E1005F0036002D
:10860000E00F5200E08F5A00E00F5B00E08F5B004C
:10861000050035000400BE000601BE003C06020055
:1086200000000000140037001000200001002000AE
:108630006011B800040060008580600006016100E0
:10864000878161008703D1000683D3008582D30030
:108650000482D30000007200818072000201730066
:10866000838173003C060200000000000001BE0090
:10867000E4040200000000000001BE00902F200072
:10868000512125005E04020000000000B406020033
:10869000000000000205BE000004BE0004712200BC
:1086A000050020006033B800EA0702000000000067
:1086B0004A6E020000000000E0C2B3000E7102002A
:1086C0000000000004712200050020006033B800A3
:1086D0000800BE000A01BE00F8070200000000000A
:1086E0000205BE000004BE00703E20000100200014
:1086F0006011B8000040E10001C8E10002D0E100D3
:1087000003D8E10003003E0000C3B3000E71020075
:108710000000000030062000010020006011B800B9
:108720000040E10001C8E10002D0E10003D8E1000F
:1087300003003E0000C3B3000E7102000000000001
:1087400090002000010020006011B8000040E1000E
:1087500001C8E10002D0E10003D8E10003003E00BF
:1087600000C3B3000E710200000000000800780092
:10877000146F020000000000E700370000C4290069
:10878000010020006011B8000020E10001A8E10014
:1087900002B0E10003B8E10054003600E00F5200DF
:1087A000E08F5A00E00F5B00E08F5B0005003500B2
:1087B0000400BE000601BE003C06020000000000EE
:1087C0001400370010002000010020006011B800E4
:1087D00004006000858060000601610087816100FF
:1087E0008703D1000683D3008582D3000482D3009F
:1087F00000007200818072000201730083817300A7
:108800003C060200000000000001BE00E40402007B
:10881000000000000001BE0080B22600E106250035
:108820005E04020000000000B40602000000000028
:108830000205BE000004BE00843E200005002000AA
:108840006033B800EA070200000000004A6E020030
:1088500000000000E0C2B3000E7102000000000042
:10886000843E2000050020006033B8000800BE00F0
:108870000A01BE00F8070200000000000205BE0069
:108880000004BE0030062000010020006011B80086
:108890000040E10001C8E10002D0E10003D8E1009E
:1088A00003003E0000C3B3000E7102000000000090
:1088B00090002000010020006011B8000040E1009D
:1088C00001C8E10002D0E10003D8E10003003E004E
:1088D00000C3B3000E710200000000000800780021
:1088E000146F0200000000008B0037009016230078
:1088F000010020006011B8000020E10001A8E100A3
:1089000002B0E10003B8E10049003600E00F520078
:10891000E08F5A00E00F5B00E08F5B000500350040
:108920000400BE000601BE003C060200000000007C
:108930001400370010002000010020006011B80072
:10894000040060008580600006016100878161008D
:108950008703D1000683D3008582D3000482D3002D
:108960000000720081807200020173008381730035
:108970003C060200000000000001BE00E40402000A
:10898000000000000001BE0000C22B00E1EB24004B
:108990005E04020000000000B406020000000000B7
:1089A0000205BE000004BE004406200005002000B1
:1089B0006033B800EA070200000000004A6E0200BF
:1089C00000000000E0C2B3000E71020000000000D1
:1089D00044062000050020006033B8000800BE00F7
:1089E0000A01BE00F8070200000000000205BE00F8
:1089F0000004BE0090002000010020006011B800BB
:108A00000040E10001C8E10002D0E10003D8E1002C
:108A100003003E0000C3B3000E710200000000001E
:108A2000084078005E6F0200000000003A00370046
:108A3000E00F5200E08F5A00E00F5B00E08F5B0018
:108A4000050035000400BE000601BE003C06020021
:108A5000000000001400370010002000010020007A
:108A60006011B800040060008580600006016100AC
:108A7000878161008703D1000683D3008582D300FC
:108A80000482D30000007200818072000201730032
:108A9000838173003C060200000000000001BE005C
:108AA000E4040200000000000001BE00006829008C
:108AB00081D124005E04020000000000B406020020
:108AC000000000000205BE000004BE00A40020005B
:108AD000050020006033B800EA0702000000000033
:108AE0004A6E020000000000E0C2B3000E710200F6
:108AF00000000000A4002000050020006033B80042
:108B00000800BE000A01BE00F807020000000000D5
:108B10005E6F020000000000A0C828009A6D0200ED
:108B20000000000003003700E0C828009A6D020032
:108B300000000000F0C1B3008666B7000000EB0043
:108B4000F0088800800888004F05BE004F04BE0072
:108B5000000006000000EB00F00888008008880094
:108B6000C942A80086C6BF0001CEB3000140600024
:108B7000A040B30086E6B700A0032000800888006C
:108B800014000700F20F2000820F5000E08F580001
:108B9000050036004809DD00C801DE0083017100D0
:108BA0004801DD0004003700A00020008008880094
:108BB000080007000001BE00F0C1B3008666B700E0
:108BC0000000EB00F0088800800888000200BE006A
:108BD000000006000080EB00700888006008880034
:108BE0000000EB004008880030088800B0088800CA
:108BF000A008880080002000F0088800400F2000B6
:108C0000E008880000402200D00888008780A90082
:108C10001FE1A80011E1A80087C0BF000048A30021
:108C2000FDFF320011E1A9001FE1A900300880001A
:108C3000705E88004208800003002000C011DD0043
:108C40000200200000004100E0804900505E8800E2
:108C5000615E880000000600889FBE008A9FBE00FB
:108C60008C9FBE008006780084A0A9008420A90003
:108C70008FC6BF0001CEB30001406000A040B3002A
:108C80008FE6B7008EC6BF0001406000A040B30071
:108C90008EE6B7000000EB0040088800300888002E
:108CA000800020008008880011E1A800300020002A
:108CB000300A880030082000100A880042C1BF0036
:108CC0000038A30007003200000A80006101B800EC
:108CD00042C1BF000038A300FBFF3A00225F8800BA
:108CE000335F880046C1BF000038A3000700320090
:108CF000200A80006101B80046C1BF000038A3000F
:108D0000FBFF3A00025F8800135F880042C1BF008A
:108D10000038A300FDFF3200000A80006104B800A3
:108D2000085F8800195F8800200A80006101B80090
:108D3000C25E8800D35E88006000B800805E880054
:108D4000915E88000002EB00445F88000D00E000A7
:108D500026003200040678000005BE0042C1BF00B4
:108D60000038A300FDFF3200000A80006103B80054
:108D7000200A80006102B8000200520083805A007D
:108D8000C000DD00000020000801530089815B0065
:108D900000004100818049000A0540008B854800A1
:108DA0000C06E8008C8F5600030032000401BE0060
:108DB0000604BE00E9FF3700A05E8800B15E8800AF
:108DC000E45E8800F55E88004D5F88008A5E88005A
:108DD0009B5E8800C45E8800D55E8800065F8800C0
:108DE000175F8800265F8800375F88000000EB006F
:108DF000100A8800100A880011E1A9006169B80012
:108E0000805E8000915E80000C090200000000007E
:108E10004F06BE004F05BE004F04BE000000060016
:108E200000B42000104078006340600002003A0067
:108E3000C942A80001003700C8C2A800E100200014
:108E400010342000188A0200000000000000060014
:108E500000B42000104078006340600003003A0036
:108E6000C942A900CB42A80002003700C8C2A9002D
:108E7000CAC2A80081002000F0342000728A0200DB
:108E8000000000000000060000B420001040780040
:108E90006340600003003A00C942A900CB42A90028
:108EA00002003700C8C2A900CAC2A9007100200090
:108EB00070352000728A02000000000000000600E9
:108EC00000B42000104078006340600007003A00C2
:108ED000C942A8000000000000000000CBC2BF0093
:108EE0004200DE006140600006003700C8C2A800F2
:108EF0000000000000000000CAC2BF004600DE0003
:108F0000614060000080FB0000000600889FBE00FA
:108F10008A1F78000004EB0088088800F8088800A1
:108F2000E80C8800405E8000E20F500011003A001B
:108F3000806780000000E8000080FB00E1BE2000A8
:108F400060C078000004E0000A003A00CAC6BF0012
:108F500001CEB30001406000CAE6B700C1002000A6
:108F6000E02B2000728A020000000000485E8800AA
:108F700060003700806780000000E8000080FB0090
:108F800080678800CA1E020000000000F61C020074
:108F900000000000CF80DE0000040200000000009E
:108FA0000004BE009A6780000A00E00006003A0054
:108FB0000200200043332400560402000000000099
:108FC0000000E000110034000004EB009867880006
:108FD00031012000301E2100728A020000000000D2
:108FE00088017800420B200088007800A00520004E
:108FF000D01F020000000000CF80DE00000402004D
:10900000000000000004BE001AC0B30010A1A800B8
:109010001081A80002002C00A35524000800BE0007
:109020005E0402000000000002002400C349240086
:109030009E0502000000000002002000832724009B
:10904000E404020000000000060602000000000028
:10905000A26C20001241780003CEB30003416100EE
:109060006241B3000001FD00CAE6B7000001FD0047
:10907000D00C8800C00C880060002000E00C880044
:10908000204E20006008880011E1A800C1002000E7
:10909000601F2100728A02000000000020002000F2
:1090A000405E8800E14F550012003A001300200096
:1090B000420B20008000EB000080EB00D01F02007C
:1090C00000000000CF80DE0000040200000000006D
:1090D0000004BE006011B8005A0402000000000045
:1090E0000000E000C9FF3D0030CB28009A6D02006F
:1090F000000000004F0578004F04BE00000006008D
:1091000000B420001064A000E0B4200010407800FB
:109110006840600005003200CAC2A900F0C2B30076
:109120000E7102000000000001003700CAC2A80052
:10913000A100200090AB2000728A02000000000015
:109140000000060000B420001064A100E0B420007C
:10915000104078006840600005003200CAC2A900D3
:10916000F0C2B3000E7102000000000001003700E1
:10917000CAC2A800A100200090AB2000728A0200A1
:109180000000000000000600E0B42000104078005D
:109190006840600005003200CAC2A800F0C2B300F7
:1091A0000E7102000000000001003700CAC2A900D1
:1091B000B100200030AC2000728A020000000000E4
:1091C0000000060000C0EB00CA0107000080FB00A1
:1091D00000000600C70107000041780000B420002D
:1091E00001C4B30010C060008000EB000100320039
:1091F0008280FB000100780000000600881F7800D4
:109200000102200000CA2000188A020000000000AD
:10921000E0B220001040E8005E6F02000000000095
:1092200000C2B3000E71020000000000E8B420008C
:109230009840780061C060005E6F0200000000008E
:1092400000C2B3000E710200000000001880FB0095
:109250000000D100614060005E6F0200000000006D
:1092600000C2B3000E710200000000001880FB0075
:109270004200DE00614060005E6F020000000000FE
:1092800000C2B3000E710200000000001880FB0055
:109290004300DE00614060005E6F020000000000DD
:1092A00000C2B3000E7102000000000000B42000F4
:1092B0001080FB004400DE00614060005E6F020031
:1092C0000000000000C2B3000E71020000000000A8
:1092D0003100200020AE2000188A020000000000AB
:1092E0004F04780000000600889FBE008A9FBE00E1
:1092F0008C1F7800CA1E020000000000F61C02004D
:109300000000000000047800CA1E020000000000F7
:10931000F61C02000000000080047800CA1E020053
:1093200000000000F61C02000000000000057800AC
:10933000CA1E020000000000F61C0200000000002F
:1093400080057800CA1E020000000000F61C020022
:109350000000000000067800CA1E020000000000A5
:10936000F61C020000000000000178000800E9007F
:10937000E30F5000020036000004EB00020037004B
:10938000E0B220000848E9000900E900E10F5000C0
:10939000020036000004EB0005003700E1B42000B5
:1093A0000940E900614060001104A100914870008B
:1093B0000A00E900E10F5000020036000004EB0053
:1093C00006003700E1B420000A40E9006140600077
:1093D000004040001114A100914870000B00E9000A
:1093E000E10F5000020036000004EB0006003700D9
:1093F000E1B420000B40E900614060004200DD0064
:109400001124A100914870000C00E900E10F500008
:10941000020036000004EB0006003700E1B4200033
:109420000C40E900614060004300DD001134A10000
:10943000914870000200E900E10F500008003E0072
:1094400000B42000E1406100C408DD001041780054
:109450000244A100014871000800E0005B003A00EE
:109460008004EB00996788007103200000BC200095
:10947000728A02000000000089017800420020008A
:109480001100200010002000D01F0200000000008A
:10949000E1B220008048E9005103200070BF2000A5
:1094A000728A02000000000089017800220020007A
:1094B0001100200010002000D01F0200000000005A
:1094C000E8B420000040E900614060001804A100F9
:1094D000184C700031042000C0C22000728A0200C3
:1094E0000000000089017800220020001100200007
:1094F00020002000D01F0200000000000040E90012
:1095000061406000004040001814A100184C700039
:1095100011032000F0C62000728A02000000000043
:109520008901780022002000110020001000200096
:10953000D01F0200000000000040E9006140600010
:109540004200DD001824A100184C7000D101200059
:10955000601C2100728A020000000000890178006E
:10956000220020001100200020002000D01F020057
:10957000000000000040E900614060004300DD00A1
:109580001834A100184C7000F1042000E093200072
:10959000728A020000000000890178002200200089
:1095A0001100200010002000D01F02000000000069
:1095B00002B42000614060004400DD009240780069
:1095C0000144A10000C97000010037000BFF070033
:1095D00000B420001064A1004F0678004F05BE00C3
:1095E0004F04BE0000000600E0B220009080FB00A7
:1095F000E08120006140780073000700E0B42000A3
:109600001080FB004300DE00614060004600DD008A
:10961000A12C2000914078000164A10080C070005E
:1096200001007800CAE2B70000000600A3000700AE
:109630000000060001002000EF0F5000E08F5800EE
:1096400057003E00006001000F0037001300370094
:109650001E00370056003700510037005000370019
:109660004F0037004E0037004D0037004C003700E8
:10967000220037002400370026003700280037007A
:109680002A0037002C0037004103200000CC2000C6
:10969000728A0200000000004500370071002000BF
:1096A00070562000728A020000000000F1002000C5
:1096B000B0182100728A02000000000011C0B3003F
:1096C0000040EB00940007003900370071002000D3
:1096D00070562000728A020000000000F100200095
:1096E000B0182100728A02000000000011C0B3000F
:1096F00001407800880007002D003700E0B420000A
:109700001004A1000E003700E0B420001004A000F7
:109710000B003700E0B420001014A100080037004F
:10972000E0B420001014A00005003700E0B42000D1
:109730001024A10002003700E0B420001024A00093
:10974000E2B4200012407800E1406000C608DD006D
:1097500042C2BF000064A1000140700042E2B700B5
:109760009280FB000101D1006141610043C2BF0052
:109770000004A1000240700043E2B700C208DE000E
:10978000E1C0600081C0400043C2BF000014A100DE
:109790000140700043E2B70098FE07000400370064
:1097A00041022000E01D2000728A0200000000003B
:1097B000000006000101200040062100728A02001C
:1097C00000000000000006000041780041E2A9000E
:1097D00000B42000104078007040600004003200A7
:1097E000CEE2A800CF02A800CEC2A8000300370036
:1097F000CEE2A900CF02A900CEC2A900A8C6BF0030
:1098000001CEB300014060007040B300A8E6B7008D
:10981000C9C6BF00014060007040B300C9E6B70090
:10982000C8C6BF00014060000034A000C8E6B70011
:10983000CAC2A800C8C2A900C902A900C8E2A800FB
:10984000C922A9000280FB001012880042A2A800D1
:10985000E2B4200012407800E1406000C608DD005C
:1098600042C2BF000064A1000140700042E2B700A4
:109870009280FB000101D1006141610043C2BF0041
:109880000004A1000240700043E2B700C208DE00FD
:10989000E1C0600081C0400043C2BF000014A100CD
:1098A0000140700043E2B7000000EB002012880086
:1098B0000012880041E2A8000000060041E2A90071
:1098C000F0C1B300A866B700C9C6BF0001CEB3009F
:1098D00001406000C9E6B700C8C6BF000140600093
:1098E000C8E6B700CEE2A900CF02A900CEC2A90007
:1098F000000006000080FB004012880085C0BF0009
:109900000028A300FDFF3200401280008540A9001E
:109910000080FB0000000600889FBE008A9FBE00FA
:109920008C9FBE008046780081457800AC81200085
:109930007A70020000000000E0FF070071000700DD
:109940000D04E00007003A0042E2A80062E2A8002D
:109950000600370020CD28009A6D020000000000AC
:10996000F3FF3700E1CF560064003E0041E2A8005B
:1099700061E2A800610037000A04E00007003A0035
:10998000CAC2BF000068A30004003200D0C5B30003
:10999000D2700200000000001AC0B30040C2BF0035
:1099A0000058A30028003A0060C2BF0001C2B30003
:1099B0000144600024003A00401280008044780096
:1099C000E14F550004003A00B0C5B300D270020068
:1099D00000000000084578000B04E000040032009D
:1099E0000980FB00C06F0200000000000600370085
:1099F000C0C5B300D270020000000000094078002A
:109A0000D270020000000000401380000044780083
:109A10000B04E0000A00320080C2B300D2700200E2
:109A2000000000000880FB00C06F02000000000082
:109A300090C2B300D27002000000000002003700A4
:109A4000D27002000000000040C2BF000068A30006
:109A500007003A0060C2BF000068A30004003A009B
:109A6000004020001C0060000D003200050037009F
:109A7000004020001C00600002003A00AC700200B0
:109A8000000000000000EB000012880000138800B6
:109A90000B04E000AFFF3A00C222A9000D0037001E
:109AA00088700200000000007470020000000000D6
:109AB000E14F5000B0FF3A00FA70020000000000D1
:109AC0000B04E0000300320030CE28009A6D020043
:109AD000000000005A000700E0B220009080FB0068
:109AE000E08120006140780037FF07004F06BE008C
:109AF0004F05BE004F04BE00000006001AC0B300B0
:109B0000A6FF3700C8C2A800C902A800C8E2A80082
:109B1000C922A800AAC6BF0001CEB3000140600060
:109B20006040B300AAE6B700AEC6BF0001406000C7
:109B30006040B300AEE6B700A8C6BF0001406000B9
:109B40009040B300A8E6B700A9C6BF00014060007E
:109B50000034A000A9E6B700ACC6BF000140600019
:109B60007040B300ACE6B700ADC6BF000140600076
:109B70000034A000ADE6B700E0B220009080FB000A
:109B8000E0812000614278000482FB00141288000A
:109B9000E1B4200011407800E1416000C619DD0009
:109BA00042C2BF00F6CBB300064060000340700025
:109BB00042E2B7001181FB000201D1006141610066
:109BC00043C2BF00E5CFB300054060000240700013
:109BD00043E2B7008000EB002112880001128800E8
:109BE0001413880062C2BF0006406000034070008A
:109BF00062E2B70063C2BF0005406000024070002F
:109C000063E2B70021138800011388004112880025
:109C1000411388004322A9006322A9004362A800DF
:109C200042A2A9006362A80062A2A90040C2A900E2
:109C300060C2A9004402A8006402A8000000060057
:109C400041E2A9004362A90061E2A9006362A900A0
:109C5000F0C1B300AA66B700AE66B700A866B70049
:109C6000A966B700AC66B700AD66B7000000060095
:109C700040CE2800826D02000000000000000600B7
:109C80000400FA00889FBE008A9FBE008C9FBE0021
:109C900011C0B300E0B2200001487800E0B4200019
:109CA0001004A1001014A0001024A10000B4200092
:109CB0001044A0002082200010409000C2FE070047
:109CC000EBFF0700CCB42000FA7002000000000097
:109CD00080417800004E78000080FB00C400DE0068
:109CE000B0B4200001487800E4CF500023013200D6
:109CF00005003E000104E00008003200E1CF500002
:109D000050013A0008013700E6CF5000220132002E
:109D1000E8CF50004B013A002B013700E5CF51004E
:109D20000A003E00E4CF51002F003100E1CF510086
:109D3000130032000C003900E2CF51001200320053
:109D4000E3CF5100F4003A0014003700EDCF51008A
:109D500017003200EECF51001C003200E6CF510058
:109D6000ED003A006D003700D4FE07004F06BE003C
:109D70004F05BE004F04BE000080FA000000060040
:109D8000BBFF0700D0FF3700CCC2A90010C0B30052
:109D90000E71020000000000CBFF3700CCC2A8000B
:109DA00010C0B3000E71020000000000C6FF3700B3
:109DB00010C0B3000E710200000000008040EB00F4
:109DC00010C0B300D4FE0700BFFF370010C0B300BF
:109DD0000E710200000000008040EB00014078009E
:109DE000CDFE0700B8FF3700FA7002000000000047
:109DF0004804DD00FA700200000000000080FB0053
:109E000000057400FA700200000000004804DD0044
:109E1000FA700200000000000080FB008005740062
:109E200000002100800F550002003E00808F550089
:109E3000080136000040EB000E7102000000000037
:109E4000A1FF37008004EB00ED8020001D8444005A
:109E5000FA70020000000000004C78008904E8005D
:109E6000890F5500F9FF3A0040C0B3009C4F100025
:109E700001003A00CAC2A9000A00E000070032004F
:109E80000004EB00704080006840780099FE0700F5
:109E90000804E800880F5500FAFF3A00100020007F
:109EA000C2890200000000000B00E000090032003F
:109EB0008004EB00EA8020001A84440000C0EB001C
:109EC0008CFE0700004C78008904E800898F55005B
:109ED000F9FF3A0041C0B3009CCF100001003A00E6
:109EE000CAC2A80010C0B3000E710200000000003A
:109EF0000B00E00074FF32000004EB0070408000B3
:109F0000684078000E710200000000000804E800BC
:109F1000888F55006CFF3200F8FF370010C0B30087
:109F20000E71020000000000FA7002000000000044
:109F3000004E7800E14F5000080032000300390065
:109F4000E24F500070003A000E00370010C0B3001E
:109F50000E710200000000005BFF370010C0B3006C
:109F60000E710200000000000040EB000E710200C4
:109F70000000000010C0B3000E71020000000000DD
:109F800051FF37000004EB006022B80084BF9F003F
:109F900095BF9F00C9B42000FA70020000000000C5
:109FA00000417800804C78000FBA97009FBA970064
:109FB0004828DD00C820DE00810070004820DD0058
:109FC0000281FB000300200002007000838070000B
:109FD00080BF9F0091BF9F000804E800E40F540079
:109FE000EDFF3A006055B800C9B42000FA700200D5
:109FF0000000000000417800804C78004858DD00E7
:10A00000C850DE00810070004850DD000281FB0076
:10A010000300200002057000838570000804E90039
:10A02000F2FF3A00F2FF2F00030020000FB8970064
:10A030009FB89700820F5000838F580008003E00A1
:10A04000820F5500838F5D0005003E000000450033
:10A0500081804D00820F5000838F5800040036002D
:10A060000040EB000E7102000000000016FF3700F8
:10A0700010C0B3000E710200000000000FBC97007A
:10A08000E00F5500E08F5D000FFF320000C2B3000B
:10A0900018FE0700C844DE000940780015FE0700DE
:10A0A0000840780013FE07000040EB0011FE070097
:10A0B0000E71020000000000E10F5500E08F5D000E
:10A0C00001FF320080C2B3000AFE07000940780099
:10A0D00008FE07000840780006FE07000040EB007D
:10A0E00004FE07000E71020000000000620555002A
:10A0F000E0855D000804E800E00F5500E08F5D009A
:10A10000F1FE3200E1FF37000040EB000E7102006B
:10A1100000000000ECFE37000040EB000E71020072
:10A1200000000000E8FE37006FC06100004EE8004C
:10A1300010C0B3000E71020000000000A0B42000A7
:10A140000048EB001C04E000DFFE32000004780051
:10A15000C9B42000FA70020000000000E5FD07000D
:10A160000E710200000000001840E800004C78006A
:10A17000994F5000D4FE3100F6FF370003407800BD
:10A18000308E02000000000010C0B3000E7102000B
:10A1900000000000CCFE370067C06100004E780070
:10A1A000E1B22000804878000080FB00218220007E
:10A1B00060C0780084FD070010C0B3000E7102007B
:10A1C00000000000C0FE3700E1B420001104A1002F
:10A1D0001114A1001124A10000B420001044A1001A
:10A1E0000381FB000228A300010032001104A0003B
:10A1F0000218A30002003200E0B420001014A000F6
:10A200000308A30002003200E0B420001024A000E4
:10A210000238A30002003A0000B420001044A0005D
:10A22000E0B220009080FB00208220006140780096
:10A2300065FD070010C0B3000E71020000000000B1
:10A24000A1FE37000040EB000E710200000000008C
:10A250009DFE37000A00E00003FF3200F9FE3700E0
:10A26000881F7800408D0200000000000004E0001C
:10A270001A00320032C2BF000038A30004003200CE
:10A280003100200040CF2000188A020000000000AA
:10A2900032C2BF000028A3000400320031002000B9
:10A2A00070CF2000188A020000000000368D0200E6
:10A2B000000000000004780032C2BF000018A300B4
:10A2C0000B003200F1002000A0CF2000188A02000D
:10A2D000000000003222A90005003700F100200034
:10A2E00090D02000188A0200000000000004EB005B
:10A2F000080078004F047800000006002A8D020054
:10A30000000000000000EB0000000600881F78003D
:10A3100001022000F0DB2000188A0200000000008B
:10A32000E8B22000184078005E6F020000000000D4
:10A3300000C2B3000E710200000000001840780057
:10A34000E94F500007003A00C0118000146F02006E
:10A350000000000000C2B3000E7102000000000007
:10A36000090037000080FB0000004000E1AB200046
:10A3700060807800146F02000000000000C2B3008B
:10A380000E7102000000000008DA200098407800FA
:10A3900063C060005E6F02000000000000C2B300F6
:10A3A0000E710200000000001880FB004200DE0079
:10A3B000614060005E6F02000000000000C2B30058
:10A3C0000E710200000000001880FB004300DE0058
:10A3D000614060005E6F02000000000000C2B30038
:10A3E0000E7102000000000000B420001080FB008D
:10A3F0004400DE00614060005E6F0200000000006B
:10A4000000C2B3000E710200000000003100200005
:10A4100020AE2000188A0200000000004F047800DF
:10A4200000000600889FBE008A9FBE008C1F780037
:10A43000CA1E020000000000F61C0200000000001E
:10A44000000478000006EB00EA0F500005003A0017
:10A45000CA1E020000000000F61C020000000000FE
:10A4600000067800CA1E020000000000F61C020070
:10A470000000000080047800CA1E020000000000F6
:10A48000F61C02000000000000057800CA1E020051
:10A4900000000000F61C02000000000080057800AB
:10A4A000CA1E020000000000F61C020000000000AE
:10A4B000800178000800E900E90F50000200360032
:10A4C0000004EB0002003700E0B220000848E90079
:10A4D0000900E900E30F5000020036000004EB0021
:10A4E0000600370000DA20008940E900E3C0600080
:10A4F000C2CFB3001048610010C870000A00E90024
:10A50000E10F5000020036000004EB0006003700A7
:10A5100001DA20000A40E900614060004200DD00ED
:10A520001124A100914870000B00E900E10F5000D8
:10A53000020036000004EB000600370001DA2000BC
:10A540000B40E900614060004300DD001134A100D0
:10A55000914870000300E900E10F500008003E0040
:10A5600000B42000E1C06100C408DD0010417800A3
:10A570000244A100014871000800E0005B003A00BD
:10A580000004EB0098678800D10820006087200055
:10A59000728A02000000000088017800A2002000FA
:10A5A0001100200010002000D01F02000000000059
:10A5B0000040E900E1B2200080487800E94F5000F7
:10A5C0000B003A00C1012000F0142100728A020041
:10A5D0000000000088017800F2FF27001100200031
:10A5E00020022000D01F020000000000C0118800DF
:10A5F0004105200080D12000188A020000000000E0
:10A600008001EB004200200011002000100020001B
:10A61000D01F02000000000008DA20000040E9001E
:10A6200063406000C1CFB30018CC6000184C7000CC
:10A6300011022000C0D62000188A0200000000008D
:10A640008001EB00220020001100200010002000FB
:10A65000D01F0200000000000040E90061406000DF
:10A660004200DD001824A100184C700021032000D6
:10A67000D0D82000188A0200000000008001EB0002
:10A68000220020001100200010002000D01F020036
:10A69000000000000040E900614060004300DD0070
:10A6A0001834A100184C7000F1042000E093200041
:10A6B000728A0200000000008001EB0022002000EE
:10A6C0001100200010002000D01F02000000000038
:10A6D00002B42000614060004400DD009240780038
:10A6E0000144A10000C970000D003700E0B2200055
:10A6F00091C0B30090CF100008003A006161B9002A
:10A7000000902000D10320000C090200000000008E
:10A7100061005000E0805800C0118800FBFE070077
:10A720004F0678004F05BE004F04BE000000060033
:10A73000E0B2200090417800E9CF510010003A00CB
:10A74000C011800003DA20001381FB004212DE00FA
:10A750004311DE006141610001B420009180FB00E3
:10A76000C408DE00E1C060006142620093417800ED
:10A77000E3C16100A08C020000000000120037005D
:10A7800005DA20001581FB004212DE004311DE00D5
:10A790006141610000B420009080FB00C408DE002D
:10A7A000E1C060000380FB0000004000E3AB20003C
:10A7B000608079006142620095427800E3C16200E6
:10A7C000A08C02000000000000DA20001040780099
:10A7D00063406000E34F500003003A0091C0B300B3
:10A7E000F0B22000014878000A8D0200000000004D
:10A7F000C111800040118000808F500004003100A2
:10A8000001022000B0162100728A02000000000040
:10A8100000000600148D0200000000000000060089
:10A82000889FBE0000047800E20F500057003200FD
:10A8300005003E000000E00008003200E10F50007B
:10A8400079003A000E003700E30F50000800320094
:10A85000E40F500074003A0064003700A1062000A5
:10A86000F0DD2000188A02000000000072003700AE
:10A87000C062A900C082A800C8C2A800C902A9007D
:10A88000B100200090E42000728A02000000000065
:10A89000D100200040E52000728A02000000000084
:10A8A000088B0200000000000000E000620032009F
:10A8B0003222A900D9FF2F0032C2BF000008A30036
:10A8C0000500320023C2BF000018A30002003A00B6
:10A8D000B011800020118800747002000000000098
:10A8E000E14F500007003A0033C2BF000018A30038
:10A8F00004003A00FA700200000000000080FB0033
:10A90000A011880032C2BF000018A30003003A0063
:10A9100022C2BF000018A300070032008004FD001F
:10A920003222B6008004FD008004FD002222B60021
:10A930008004FD00C222A900E30F5400DEFF3A00AC
:10A94000212C200091407800C408DE00E1806000E6
:10A95000CBC2BF000004A10001407000CBE2B700F1
:10A96000CAC2BF004600DE00610060004300DD0097
:10A97000212C2000914078000134A10080C070009B
:10A9800001007800C2E2B700CBFF3700E1002000F1
:10A9900010E62000728A020000000000F100200092
:10A9A000B0182100728A0200000000003222A900C3
:10A9B00032C2BF000008A3000500320023C2BF005E
:10A9C0000018A30002003A00B01180002011880096
:10A9D0007470020000000000E14F5000F4FF3A00E4
:10A9E000FA7002000000000013003700148D02000E
:10A9F000000000000000EB00920007000A8D02003A
:10AA000000000000C111800040118000808F5000C4
:10AA10000900310001022000B0162100728A0200F4
:10AA2000000000000400370041022000E01D20006B
:10AA3000728A0200000000004F04BE000000060001
:10AA40003222A90000DA20001044A00000B4200047
:10AA50001024A000C1012000F0E62000728A02004C
:10AA6000000000000000060000DA20001044A100F1
:10AA700000B420001024A10041012000B0E8200013
:10AA8000728A02000000000000000600881F7800A3
:10AA90000004EB002C00370000DA200010407800A2
:10AAA000704060002500320020C428009A6D02002A
:10AAB000000000006100200080662000188A02006B
:10AAC0000000000032C2BF000038A30004003200C2
:10AAD0003100200040CF2000188A02000000000052
:10AAE00032C2BF000028A300040032003100200061
:10AAF00070CF2000188A020000000000368D02008E
:10AB000000000000128902000000000032C2BF00F5
:10AB10000018A30005003200F1002000A0CF2000A3
:10AB2000188A0200000000003222A90020C4280078
:10AB30009A6D02000000000002003700368D02000E
:10AB40000000000018002000408D020000000000FE
:10AB50000004E000D0FF3A00080078004F047800BD
:10AB600000000600B1002000B00A2100728A020035
:10AB700000000000000006000000EB00F008880064
:10AB80008008880081002000810888004008880033
:10AB900030088800B0088800A0088800F108880004
:10ABA0000000060011E1A9001FE1A900F0C1B300F7
:10ABB0008666B7000000EB00F00888008008880077
:10ABC0003008880040088800000006000002BE002F
:10ABD0001100200080C428001001BE00840F510025
:10ABE000858F590010003600C208DD0040C42800DF
:10ABF0008080400061BB9700F1BB970006005100C8
:10AC0000878059008100D1000080D30006004000F9
:10AC100087804800800F5200818F5A0007003E0055
:10AC20000601BE00050037008100E8006400400016
:10AC3000EF8F5000E8FF3A006011B8000200BE003C
:10AC400000000600889FBE008A9FBE008C9FBE0049
:10AC500080067800CAE2A900C8E2A8000000E0006F
:10AC600004003A003101200020202100728A0200F5
:10AC700000000000CA42E20007003D006300370008
:10AC800000000000CA42E20003003D0022C2BF00F3
:10AC90000008A300FAFF320022C2BF000008A30090
:10ACA0000800320030118000BEFF0700E1002000E4
:10ACB00050212100728A0200000000006044B800A8
:10ACC000560037008004EB006055B80008C8B30098
:10ACD0000006EB00A8FF0700CAC2BF0008406000E2
:10ACE000FDFF32001FE1A80011E1A80001C8B30078
:10ACF000CAC2BF0001406000FDFF3A0011E1A90097
:10AD00001FE1A900F0C1B3008666B700FC08880007
:10AD10008C0888004008800001002000C000DD0091
:10AD2000000020003208800002004000E08048005F
:10AD30000900E00007003200E00F5500E08F5D00E1
:10AD4000030032008A0F50008B8F58000100310041
:10AD50000005BE008904E800F98F5400DDFF3A00C9
:10AD600090FF07000A01BE0000402200410F2000B2
:10AD70000C090200000000000004BE000D00E0000D
:10AD800026003A00009F240021002000800F54007C
:10AD9000818F5C0005003600F10220003022210086
:10ADA000728A0200000000001C003700F100200041
:10ADB00020252100188A0200000000000800BE00C3
:10ADC000E46D020000000000410020000027210087
:10ADD000728A020000000000F1002000102621000D
:10ADE000188A0200000000000800BE0077FF07007C
:10ADF000E46D020000000000410020000027210057
:10AE0000728A0200000000000400370022C2BF0066
:10AE10000008A3009AFF32009FFF37000800BE0021
:10AE20004F06BE004F05BE004F04BE0000000600E6
:10AE300040C82800826D02000000000000000600EB
:10AE4000889FBE008A9FBE008C1F780001DA200018
:10AE5000C0CFB300914860001124A1001134A100BB
:10AE600000B420001044A00090568000D06C8800F0
:10AE70001144A1001181FB004212DE004311DE00EB
:10AE8000614161006142620091407800E3C160006D
:10AE900011C0B300A08C0200000000000A8D020067
:10AEA00000000000E2FF070008DA2000EAD92000D5
:10AEB0000BB42000408D0200000000000004E00000
:10AEC0000A0032009840780070C06000050032002F
:10AED000368D0200000000000E710200000000002C
:10AEE00002003700368D02000000000032C2BF00B1
:10AEF0000018A300010032003222A9007470020081
:10AF000000000000E14F5000EAFF3A00FA70020032
:10AF10000000000080417800004D78000080FB00B8
:10AF2000C400DE00D0D9200001487800E4CF5000F2
:10AF30008A00320005003E000104E0000A003200F1
:10AF4000E1CF5000E1003A006C003700E6CF50003E
:10AF500089003200DD00390068C05000E14F500028
:10AF6000DA003E00A5003700E2CF510015003200A4
:10AF700005003E000304E0000A003200E1CF51006A
:10AF80005A003A000D003700E7CF51001B00320095
:10AF9000EFCF51003D003200E3CF510053003A00A3
:10AFA00011003700148D0200000000004F067800E9
:10AFB0004F05BE004F04BE00000006009CFF0700C6
:10AFC000BCFF370010C0B3000E710200000000008B
:10AFD00032C2BF000018A300010032003222A900D3
:10AFE0001844A000B3FF37001844A10010C0B300FC
:10AFF0000E71020000000000AEFF370010C0B30069
:10B000000E71020000000000148D0200000000001C
:10B01000FA700200000000004800DD00D06C8800DB
:10B0200010C0B3000E71020000000000FA700200B0
:10B03000000000000080FB00D16C80000100700067
:10B04000D06C88001881FB004212DE004311DE0044
:10B05000614161009B80FB00C408DE00E1C060002C
:10B060006142620098427800E3C16200A08C020055
:10B07000000000000A8D02000000000010C0B300B4
:10B080000E710200000000008AFF370010C0B300FC
:10B090000E710200000000003222A90032C2BF007F
:10B0A0000008A3000500320023C2BF000018A3005F
:10B0B00002003A00B0118000201188007470020074
:10B0C00000000000E14F5000F4FF3A0033C2BF001F
:10B0D0000018A300F1FF3A00FA700200000000001F
:10B0E0000080FB00A0118800ECFF37000040EB005F
:10B0F0000E710200000000006EFF37006FC061009B
:10B10000004DE80010C0B3000E7102000000000006
:10B11000C0D920000048EB001A04E00065FF3200AF
:10B1200080047800ECD92000FA70020000000000D2
:10B130000080FB002A8D02000000000010C0B30058
:10B140000E710200000000001940E800804C7800F9
:10B150009C4F500057FF3100F3FF37000340780049
:10B16000308E02000000000010C0B3000E7102001B
:10B17000000000004FFF37006FC06100E1D92000E0
:10B1800080487800EA4F500002003600A0C0B300AB
:10B19000804878001A80FB000000400021AD2000AC
:10B1A00060807800D06C8800148D020000000000E0
:10B1B0001881FB004212DE004311DE006141610094
:10B1C0009B80FB00C408DE00E1C06000D06C800002
:10B1D0006142620098427800E3C16200A08C0200E4
:10B1E000000000000A8D02000000000010C0B30043
:10B1F0000E710200000000002EFF370001DA20006F
:10B20000C4CFB300914862001124A1001134A10001
:10B210001B44A1000381FB000238A300050032009B
:10B220009142780063C062000014A00084C86200EC
:10B23000914870000228A300060032009840780070
:10B2400063C060000004A000C1CFB30018CC600050
:10B25000184C70000218A300010032001824A0004E
:10B260000308A300010032001834A0000248A30024
:10B2700001003A001B44A000148D020000000000F1
:10B280001881FB004212DE004311DE0061416100C3
:10B290009B80FB00C408DE00E1C06000D06C800031
:10B2A0006142620098427800E3C16200A08C020013
:10B2B000000000000A8D02000000000010C0B30072
:10B2C0000E71020000000000FAFE37000040EB00A3
:10B2D0000E71020000000000F6FE3700C0D1280009
:10B2E000826D02000000000000000600889FBE0082
:10B2F0008A9FBE008C1F780001B4200011407800A6
:10B300000034A1000044A0008048780018C0B300B9
:10B31000E0B220000848780081C0B300F0B22000FD
:10B320000148780020C0B300A1DB200080487800ED
:10B3300080C0EB009A77020000000000C922A9003B
:10B34000C902A900C8E2A80008407800C679020036
:10B3500000000000E1FF0700EADB2000CCDB20005A
:10B36000FA7002000000000080417800004D780073
:10B370000080FB004400DE00D1DB20008048780024
:10B38000E34F5000C700320004003E00E14F500080
:10B3900086003200BA003E000B003700E64F500036
:10B3A0007202320003003E00E44F5000A3023A0054
:10B3B00067023700E84F50007B023200EA4F50002E
:10B3C0009E023A00D80037000380FB0001002000F5
:10B3D000ED0F5000E08F580070003E00006001004B
:10B3E0009A0237000C0037000D00370012003700BA
:10B3F000170037001D003700230037003A003700E0
:10B400003E00370042003700480037004E0037004A
:10B41000540037005A003700B0FF0700D0FF370054
:10B420000C7802000000000010C0B3000E71020092
:10B4300000000000CAFF3700407802000000000052
:10B4400010C0B3000E71020000000000C4FF3700FE
:10B450000040EB00C67902000000000010C0B300FD
:10B460000E71020000000000BDFF370010C0B300E5
:10B47000C67902000000000010C0B3000E71020087
:10B4800000000000B6FF3700A0DB200021C0B300A1
:10B4900090CF100004003A00047902000000000080
:10B4A000004E780004003700F00F20005C780200A6
:10B4B00000000000004E780000B42000104078002A
:10B4C00068406000040032001C80FB00F08902002C
:10B4D00000000000004E78001C4078000E71020051
:10B4E000000000009EFF37004679020000000000C7
:10B4F0000E7102000000000099FF3700D2790200AF
:10B50000000000000E7102000000000094FF3700F0
:10B5100010C0B300887902000000000010C0B30022
:10B520000E710200000000008DFF37000040EB00AC
:10B53000BA7902000000000010C0B3000E710200D2
:10B540000000000086FF370010C0B300BA79020087
:10B550000000000010C0B3000E71020000000000E7
:10B560007FFF37000040EB00AE79020000000000D2
:10B5700010C0B3000E7102000000000078FF370019
:10B5800010C0B300AE7902000000000010C0B3008C
:10B590000E7102000000000071FF37000040EB0058
:10B5A0000E710200000000006DFF37006FC06100E7
:10B5B000004DE80010C0B3000E7102000000000052
:10B5C000004EEB001A04E00065FF3200B9DB2000FA
:10B5D0000BB42000FA7002000000000080407800E8
:10B5E000804C78001B417800684061000400320004
:10B5F0000180FB00F089020000000000804C780010
:10B60000A0DB200021C0B30090CF100007003A005B
:10B610001980FB00BC7802000000000010C0B300DD
:10B620000E7102000000000010003700B8DB20009F
:10B630001880FB005C780200000000008040780069
:10B64000004C78001B417800684061000400320023
:10B650000180FB00F089020000000000004C78002F
:10B66000194078000E710200000000001C40E80044
:10B67000004E78009A4F500039FF3100D5FF370057
:10B680006FC061000040E800004D7800887902003A
:10B690000000000010C0B3000E71020000000000A6
:10B6A0002FFF37006FC06100004DE80010C0B300ED
:10B6B0000E71020000000000FA700200000000009D
:10B6C000D1DB200080487800004EEB001A04E00037
:10B6D0001100320001047800C9DB20001804E000EA
:10B6E00004003D0010C0B3006A79020000000000B1
:10B6F000030037000040EB006A7902000000000000
:10B7000018407800004C40001940E800804C780058
:10B710009A4F5000F1FF390010C0B3000E710200C3
:10B72000000000000EFF370040CAB30080CF510078
:10B730001400320004003E006440500080CF5100ED
:10B740007F013A000700370050CAB30080CF510094
:10B750009800320000C0E80080CF510078013A0024
:10B76000ED003700FA7002000000000061AE20001A
:10B770008048780010C0B3000E7102000000000085
:10B78000F7FE370060AE200010407800E14F500017
:10B7900003003200E24F500082003A002A003700D6
:10B7A000FA700200000000000080FB006300B90096
:10B7B000C06D88000001EB00926D88000000E00081
:10B7C0000C00320082007800E980200019844000DB
:10B7D000FA70020000000000004C7800906D8000BC
:10B7E0008000E800916D8800C06D8000808F50005F
:10B7F000F6FF39008000EB00916D8800C06D80007D
:10B800000000E0000C0032007040800001004000A9
:10B81000204190009040900010407800D701070030
:10B82000906D8000E3004000916D8800C06D800045
:10B83000808F5000F4FF390010C0B3000E71020079
:10B8400000000000C6FE3700FA7002000000000091
:10B850000080FB004200DD00C06D88008000EB002E
:10B86000916D88000B003200E980200019844000AF
:10B87000FA70020000000000004C7800906D80001B
:10B880008000E800916D8800C06D8000808F5000BE
:10B89000F6FF39000000EB00906D8800C06D80005D
:10B8A0000000E0003B0032000040EB006A7902003B
:10B8B000000000000040EB006A7902000000000078
:10B8C0000040EB006A790200000000000040EB003D
:10B8D0006A79020000000000916D800070408000D5
:10B8E000614078000080FB00BC780200000000008E
:10B8F00070408000916D8000010040001040900079
:10B900000080FB00BC780200000000007040800056
:10B91000916D800001004000204090000080FB00FD
:10B92000BC78020000000000926D8000E0802000E2
:10B930001000410063004000904078006FC8600034
:10B94000004EEB007040800000004100304090004D
:10B950000004E0000A003200C8DB2000B801070044
:10B960001840E800004C7800926D80007140800023
:10B9700082804000B1409000814F5000F7FF3900B5
:10B98000E4004100916D8800C06D8000808F500000
:10B99000C5FF390010C0B3000E71020000000000A6
:10B9A0006FFE37000040EB000E7102000000000047
:10B9B0006BFE370060AE200010407800E14F500071
:10B9C00003003200E24F500065FE3A0030003700BD
:10B9D000FA700200000000000080FB00C06D8800CB
:10B9E000FA70020000000000D1DB200080487800DF
:10B9F0000000EB00906D8800C06D80000000E0004A
:10BA000057FE3200B8DB2000C9DB2000D0DB20006D
:10BA1000104C7800804CEB001880FB000008A3005D
:10BA20000400320010C0B3006A7902000000000078
:10BA3000030037000040EB006A79020000000000BC
:10BA40001880FB000000D100004C78001940E8008D
:10BA5000804C7800E34F5000EFFF3600047902007D
:10BA60000000000004790200000000000E710200D6
:10BA700000000000906D80000000E800906D8800DC
:10BA8000C16D8000810F500035FE3100DFFF3700AF
:10BA9000FA700200000000008080FB00C16D880089
:10BAA0008000EB00916D88000004E0002CFE320065
:10BAB00022C0B30060B92000A10B20009F01070045
:10BAC000CB01070022C0B30060BB2D00A10B2000FA
:10BAD0009A01070022C0B300603D2D00A10B200099
:10BAE00096010700C201070022C0B30060BB20001E
:10BAF000A10B200091010700BD010700906D80009F
:10BB00000000E800906D8800C16D8000810F50003A
:10BB100013FE3100E6FF3700FA700200000000005B
:10BB20000080FB00B06D8800FA7002000000000089
:10BB30000081FB00A26D880060AE200010407800FC
:10BB4000E24F500005003A00B06D80006500B9007A
:10BB500000004100C06D880014003700E14F500024
:10BB600006003A00B06D8000000040000000410077
:10BB700000004000C06D88000C003700E34F50000B
:10BB800006003A00B06D8000000040000000410057
:10BB900000004000C06D8800040037000040EB004A
:10BBA0000E71020000000000EDFD37008000EB0088
:10BBB000916D8800C06D80000000E0000B00320035
:10BBC000E980200019844000FA70020000000000A3
:10BBD000004C7800906D80008000E800916D880036
:10BBE000C06D8000808F5000F6FF3900A06D80008E
:10BBF0000000E0000300320010C0B3000E7102002C
:10BC0000000000000000EB00906D880068AE20008E
:10BC10004000370070408000E2407800E1CF5000E3
:10BC200021003A0098407800E3CF500009003A0024
:10BC30000200400030419000A04090001040900071
:10BC40009A000700906D800064004000906D8800AD
:10BC500030003700E1CF500009003A0002004000F8
:10BC600030419000A040900010409000C3000700B9
:10BC7000906D800064004000906D880025003700C2
:10BC8000E2CF500023003A0002004000C040900084
:10BC90000000E80000010700906D80006500400092
:10BCA000906D88001B003700E2CF500019003A0069
:10BCB00098407800E3CF500007003A0002004000AF
:10BCC0001040900065000700906D80000080E80043
:10BCD000906D88000F003700E1CF500007003A0058
:10BCE00002004000104090008C000700906D800022
:10BCF0000080E800906D880006003700E2CF500019
:10BD000004003A003A010700906D80000000E8004E
:10BD1000906D8800926D8000C06D8000800F510092
:10BD2000BCFF3900A06D80000000E0008CFD3A00EF
:10BD300010C0B3000E7102000000000088FD370043
:10BD40000040EB000E7102000000000084FD37008F
:10BD500003407800308E02000000000010C0B300E5
:10BD60000E710200000000007DFD3700E3C061009D
:10BD7000014D7800E0B2200001487800A0DB2000EF
:10BD8000104078009A7702000000000010C0B30055
:10BD9000C67902000000000010C0B3000E7102005E
:10BDA000000000006EFD370002B420001240780051
:10BDB0000040A100004978008380FB000138A30007
:10BDC00002003A000044A00000497800A2DB2000F5
:10BDD00020C0B300004978000128A300020032000F
:10BDE00030C0B3000049780002B42000124078004F
:10BDF0000030A100004978000118A30002003200C1
:10BE00000034A00000497800E0B2200090407800A3
:10BE1000A0DB2000104078009A77020000000000AC
:10BE200010C0B300C67902000000000010C0B300CB
:10BE30000E7102000000000049FD37000040EB00D9
:10BE40000E7102000000000045FD37004F0678002B
:10BE50004F05BE004F04BE0000000600889FBE00D4
:10BE60000044780069C0B300614064006A79020050
:10BE7000000000000880FB000004D1008944E900B4
:10BE8000F9FF3A0004790200000000000E71020080
:10BE90000000000004790200000000000E710200A2
:10BEA000000000004F04BE0000000600889FBE0096
:10BEB0008A9FBE008C1F780000447800814578007E
:10BEC0000246780000C8B3000045640069C0B300B2
:10BED000614064006A790200000000000880FB00F5
:10BEE0000004D1008944E900F9FF3A000A04E000A7
:10BEF00006003A000B80FB00BC7802000000000046
:10BF00000C80FB00BC780200000000004F067800A7
:10BF10004F05BE004F04BE0000000600889FBE0013
:10BF20000044780049C0B3000808A30004003200B0
:10BF300010C0B3006A79020000000000030037005F
:10BF40000040EB006A790200000000000880FB005E
:10BF50000004D1008944E900F3FF3A0004790200AB
:10BF60000000000004790200000000000E710200D1
:10BF7000000000004F04BE0000000600889FBE00C5
:10BF80008A9FBE008C1F78000044780081457800AD
:10BF9000024678000080FB004605DE008044EB008E
:10BFA0000F003700E3CF54000D003A000A04E00010
:10BFB0000A00320010C0B300BA790200000000008D
:10BFC0000A80FB009E890200000000000040EB0098
:10BFD000BA790200000000000C00370039C0B3003D
:10BFE0000808A3000400320010C0B3006A79020000
:10BFF00000000000030037000040EB006A790200F7
:10C00000000000000880FB000004D1008944E80023
:10C01000E3CF5400E3FF36000B80FB00BC78020046
:10C02000000000000C80FB00BC7802000000000053
:10C030004F0678004F05BE004F04BE00000006000A
:10C040000040EB006A790200000000000040EB00B5
:10C050006A790200000000000040EB006A790200EB
:10C06000000000000040EB006A79020000000000C0
:10C070000000EB00BC780200000000000000EB00B4
:10C08000BC780200000000000000EB00BC78020059
:10C090000000000000000600889FBE000004780039
:10C0A000814478000040EB006A7902000000000043
:10C0B0000040EB006A790200000000000040EB0045
:10C0C0006A790200000000000040EB006A7902007B
:10C0D000000000001880FB00BC7802000000000097
:10C0E000184090000080FB00BC78020000000000B7
:10C0F000284090000080FB00BC7802000000000097
:10C100006FC064000041E900E14F410009003200C6
:10C11000024478000080EB000090B900004041002C
:10C120008044E900C6FF07000844E90088CF5400B6
:10C13000FCFF3A004F04BE0000000600889FBE00CE
:10C140008A1F78000004BE00024578000040EB0022
:10C150006A790200000000000040EB006A790200EA
:10C16000000000000040EB006A79020000000000BF
:10C170000040EB006A79020000000000080078002F
:10C18000F089020000000000BC78020000000000FE
:10C190004849DD004840DE0000007100C848DE006C
:10C1A000F089020000000000BC78020000000000DE
:10C1B000404CDE0008007800F0890200000000001A
:10C1C000BC780200000000006F45650005003200E9
:10C1D0000044EB009AFF07000844E800884F550030
:10C1E000FCFF3A004F0578004F04BE000000060037
:10C1F000881F780010C0B3006A79020000000000B8
:10C200000040EB006A790200000000000040EB00F3
:10C210006A790200000000000040EB006A79020029
:10C22000000000000000EB00BC78020000000000ED
:10C230000479020000000000000478000479020084
:10C24000000000000E7102000000000008407800AD
:10C250000E7102000000000079FF070078FF070060
:10C260004F04780000000600B05A80000000E00093
:10C270001100320000C2B3000E7102000000000085
:10C280003100200030412000188A02000000000028
:10C2900000C2B3000E71020000000000A05A80002E
:10C2A0000000E00002003A006A790200000000008D
:10C2B0000000EB00B05A88008040EB00A05A8000DC
:10C2C0000000E00003003A000479020000000000D2
:10C2D0008040780010002000B05A88000180FB00E8
:10C2E00000000600881F780000047800B05A800023
:10C2F0000000E0001100320000C2B3000E71020025
:10C30000000000003100200030412000188A0200A7
:10C310000000000000C2B3000E7102000000000027
:10C32000A05A80000000E00002003A006A79020092
:10C33000000000000000EB00B05A8800A05A800006
:10C340000000E00006003A0008007800BC78020017
:10C350000000000046790200000000000084FB009D
:10C3600000C2B3000E710200000000000800E000EF
:10C3700006003A003100200030412000188A0200F7
:10C3800000000000003020000500370041002000C0
:10C3900060412000188A0200000000000010200008
:10C3A0004F04780000000600B05A80000000E00052
:10C3B0000F0032004100200060412000188A020076
:10C3C00000000000A0CE28009A6D020000000000CE
:10C3D000A05A80000000E00003003A0010C0B30043
:10C3E0006A790200000000000000EB00B05A8800EB
:10C3F000A05A80000000E0000F003A000C78020014
:10C40000000000000000E0000B003200910020005E
:10C41000C0202000188A0200000000005101200006
:10C4200050212000188A020000000000A0CE280041
:10C430009A6D020000000000D1002000A041200001
:10C44000728A02000000000000000600B05A80005E
:10C450000000E0000F003200410020006041200099
:10C46000188A020000000000A0CE28009A6D020089
:10C4700000000000A05A80000000E00003003A0025
:10C4800010C0B3006A790200000000000000EB0059
:10C49000B05A8800A05A80000000E00002003A0074
:10C4A0004078020000000000C1002000704220001F
:10C4B000728A020000000000000006000101200056
:10C4C000404F2000188A0200000000000040EB00EE
:10C4D0005E6F02000000000000C2B3000E71020097
:10C4E00000000000E0B22000104078005E6F020003
:10C4F0000000000000C2B3000E7102000000000046
:10C50000B0CE28009A6D0200000000000000060076
:10C51000881F78000000EB00A05A8800CA1E0200A5
:10C5200000000000F61C02000000000080007800FF
:10C530000000E900E30F500004003E00E0B22000DC
:10C540000148E9000100E00010003A000004EB009F
:10C5500098678800A85A8800B10320008045200011
:10C56000728A02000000000088017800420020006A
:10C570001100200010002000D01F02000000000069
:10C58000E1B220008048E9000B00370081812000E3
:10C5900030002300910F100004003E0051032000E2
:10C5A00030492000188A020000000000C3FF070085
:10C5B0000000EB00B05A880000B420001044A00036
:10C5C0004F04780000000600A05A80000000E00040
:10C5D00009003A00C922A800C902A800CB02A9009C
:10C5E000CB22A900E0B220009040780020C0B30028
:10C5F0009A77020000000000000006000000EB0037
:10C60000B05A8800A05A8000E10F500001003A00A3
:10C6100007E2A90000000600889FBE00E10F50005D
:10C620000900320003003900E20F50006B003A00AD
:10C630005B0037005103200040502000188A0200A0
:10C6400000000000690037008040EB00003020004F
:10C65000DA79020000000000E1022000905320007F
:10C66000728A020000000000CBC2BF000008A300D5
:10C6700005003200CBC2BF00190020000004EB000F
:10C680000018A3000C003A0091002000C0202000F8
:10C69000188A0200000000005101200050212000F3
:10C6A000188A020000000000A0CE28009A6D020047
:10C6B000000000004D003700A05A80000000E0009C
:10C6C00008003A000C780200000000000800780022
:10C6D000BC78020000000000467902000000000063
:10C6E0008084FB000900E00020003A000800780088
:10C6F000128902000000000080C2B3000E71020027
:10C70000000000000880D100128902000000000033
:10C710000808A30004003A00D0CE2800826D020071
:10C72000000000000B003700A05A80000000E0006D
:10C7300005003A00047902000000000010C0B300B8
:10C740006A7902000000000000CF2800826D02001C
:10C7500000000000B0CE2800826D02000000000042
:10C7600000C2B3000E71020000000000A05A800059
:10C770000000E00002003A004078020000000000E3
:10C780000804E80000102000800F5400CAFF3A009F
:10C79000A0CE28009A6D02000000000013003700B0
:10C7A000A05A8000E10F500001003A0007E2A90002
:10C7B0007100200070562000728A02000000000004
:10C7C000F1002000B0182100728A02000000000071
:10C7D00010C0B3000C000700040037004102200025
:10C7E000E01D2000728A0200000000004F04BE001D
:10C7F00000000600B1002000600B2100728A0200D8
:10C800000000000000000600E4874700889FBE008B
:10C810008A9FBE008C9FBE008E1F780090F79F00FD
:10C820007A70020000000000C922A800C902A80016
:10C83000CB02A900CB22A90062A0A80062C0A80078
:10C840008660A900CBC2BF000000D100B12C20003F
:10C85000914078006146600061C460000047EB00D1
:10C860008E4678008EF79F00060037000B46780052
:10C870000A4478000047EB00020037000B467800BE
:10C880000A44780086C0BF000038A3000E003A00BA
:10C8900088700200000000007470020000000000B8
:10C8A0000004E000F7FF3200FA7002000000000010
:10C8B00062A0A90062C0A9009FF097000104E000F7
:10C8C00057003200530037008660A900CBC2BF007A
:10C8D0000000D100E104600089457800CBC2BF00B0
:10C8E00061406000004578000E04E0002F00320037
:10C8F0000804E0002F003A000004E000DFFF3200EF
:10C90000E7CF56000B003E000FF0970000404000BC
:10C9100080F79F000904E000020032000004A0003C
:10C9200080F79F008D46E8000B4678000A447800A7
:10C93000D4FF37001FF097000004E000050032002C
:10C940008FF097000180FB00C06F02000000000024
:10C9500006003700C0C5B300D2700200000000001E
:10C960000FF09700D2700200000000000904E00000
:10C9700007003200D0C2B300D270020000000000F5
:10C980000B4678000A4478008046EB00BDFF370074
:10C99000B0C2B300D2700200000000000B46780065
:10C9A0000A4478008046EB00B6FF37000804E00038
:10C9B000AEFF32000004E000B0FF32000C04E000E3
:10C9C0000A0032000904E000ACFF3A00B0C5B30031
:10C9D000D2700200000000000B4678000A44780084
:10C9E0001EC0B30089467800A6FF37000904E000A6
:10C9F000A2FF3200D0C5B300D270020000000000D8
:10CA00000B4678000A4478000047EB008E46780019
:10CA10009CFF3700A0CE28009A6D020000000000A5
:10CA20004F0778004F06BE004F05BE004F04BE0002
:10CA30004F00B1000000060030CF2800826D0200D8
:10CA40000000000000000600889FBE008A9FBE0014
:10CA50008C9FBE008E1F7800C922A800C902A800C2
:10CA6000CB02A900CB22A900C8C2A90001B42000B2
:10CA7000114078000034A1000044A00080487800F4
:10CA800080C0EB0020C0B3009A77020000000000D5
:10CA9000E9FF07002AB520000EB42000FA7002005A
:10CAA0000000000080417800004D78000080FB000D
:10CAB0004400DE0011B5200080487800E14F5000AE
:10CAC000D200320005003900E44F5000F10032007E
:10CAD000E64F5000F6003A00E50037000380FB0007
:10CAE00001002000EF0F5000E08F5800C3003E000F
:10CAF00000600100F50037000E0037000F0037001E
:10CB00001400370019003700BC0037001C00370044
:10CB100022003700280037007D003700B7003700BB
:10CB2000B6003700B5003700B4003700B300370057
:10CB3000AC003700C0FF0700D8FF37000C780200B8
:10CB40000000000010C0B3000E71020000000000E1
:10CB5000D2FF3700407802000000000010C0B30090
:10CB60000E71020000000000CCFF370004790200C3
:10CB7000000000000E71020000000000C7FF370037
:10CB80000040EB006A7902000000000010C0B30012
:10CB90000E71020000000000C0FF370010C0B3009B
:10CBA0006A7902000000000010C0B3000E7102009C
:10CBB00000000000B9FF3700FA700200000000001A
:10CBC0004804DD00FA700200000000000080FB0055
:10CBD00080057400FA700200000000004804DD00C7
:10CBE000FA700200000000000080FB0000067400E4
:10CBF00000002100808F550002003E00800F56008B
:10CC0000AF0036000040EB000E7102000000000093
:10CC1000A2FF37008004EB00ED8020001D8444005B
:10CC2000FA70020000000000004C78008904E8005F
:10CC3000898F5500F9FF3A000C78020000000000CF
:10CC40000B00E0000D0032000004EB00704080009B
:10CC5000684078000080FB00BC7802000000000003
:10CC60004679020000000000E14F5000E5FF32006D
:10CC70000804E800888F5500F4FF3A008C05E900AD
:10CC80000C00E000120032008004EB00ED80200078
:10CC90001D8444000479020000000000004C78006C
:10CCA0008B8F5400040031000040EB006A790200D1
:10CCB000000000000300370010C0B3006A790200D2
:10CCC000000000008904E800890F5600F0FF3A00D8
:10CCD000407802000000000010C0B3000E71020096
:10CCE000000000000C00E0006CFF32000004EB00CC
:10CCF00070408000684078000E7102000000000063
:10CD00000804E800880F560064FF3200F8FF37007F
:10CD100010C0B3000E7102000000000022C2BF006C
:10CD20000008A300FDFF3200301180008040780031
:10CD3000004D7800E24F50001700320005003E0021
:10CD40000004E0000C003200E14F500008003A00FF
:10CD50000D003700F04F50001600320000C2B30043
:10CD600080CF500017003200E3CF50000E00320099
:10CD700010002000180037004447020000000000A7
:10CD800010002000140037002847020000000000B7
:10CD900010002000100037001047020000000000C3
:10CDA000100020000C003700604702000000000067
:10CDB00009003700C0CFB3001E4F600010002000F4
:10CDC000050037001E4078000014A1000004A000F8
:10CDD000004F7800100020000E71020000000000DB
:10CDE0002EFF37000040EB0087FE070010C0B300A5
:10CDF0000E7102000000000028FF37000040EB0029
:10CE00000E7102000000000024FF37006FC06100B7
:10CE1000004DE80010C0B3000E71020000000000D9
:10CE200000B520000048EB001A04E0001BFF3200B0
:10CE30000004780029B52000FA700200000000000C
:10CE40000080FB00BC780200000000004679020070
:10CE5000000000000E710200000000001840E80011
:10CE6000004C7800994F50000CFF3100F2FF370062
:10CE7000E3C06100014D780020C0B3009A77020042
:10CE80000000000010C0B3000E710200000000009E
:10CE900002FF370003407800308E020000000000DF
:10CEA00010C0B3000E71020000000000FBFE37004E
:10CEB0000040EB000E71020000000000F7FE37009A
:10CEC0000B00E0005CFF320052FF37004F07780094
:10CED0004F06BE004F05BE004F04BE000000060016
:10CEE00000C0EB007C8C0200000000000080FB0012
:10CEF000000006007C8C02000000000000102000F2
:10CF00000000060010C0B300328C020000000000D8
:10CF10000080FB000000060080B520001040780073
:10CF2000328C0200000000000000060080B52000E6
:10CF30001080FB000000060080B520000048EB00D8
:10CF400041022000B0002000728A020000000000B0
:10CF50000000060011C0B30080B520000148780031
:10CF600041022000B0002000728A02000000000090
:10CF70000000060000B420001044A000A0B620006D
:10CF80000048EB00C922A800CB22A900000006003F
:10CF9000889FBE008A1F7800800078000004E900A6
:10CFA00010032000800F540030003E00A0B6200087
:10CFB0001080FB00800F5400050039009102200012
:10CFC000F0022000728A0200000000000E0137000B
:10CFD000E100200080052000188A02000000000007
:10CFE0000840E8005E6F02000000000080CF2800CB
:10CFF000826D0200000000008040EB0040B620007F
:10D000000148780001407800C344DD00BAB6200032
:10D0100048B620000080FB000900400060407D0011
:10D020000080FB00128902000000000000C2B30073
:10D030000E710200000000001880FB000900400093
:10D0400060407D007C8C0200000000001840E80079
:10D05000004C7800E74F5000EEFF3600B0CF2800BC
:10D060009A6D020000000000E70037005005200024
:10D07000808F5000CE00320006003E000100E0002C
:10D080000E00320030032000808F5000DA003A009A
:10D09000A4003700C00E2000808F500048003200EE
:10D0A00064004000808F500045003200C00C20001A
:10D0B000808F5000D0003A00C6003700D100200019
:10D0C00060062000728A020000000000710120004A
:10D0D00030072000728A020000000000A0B6200085
:10D0E0001004E00005003A0091022000F002200048
:10D0F000728A0200000000002C00370050B62000A9
:10D100000048EB008004780048B62000BAB6200042
:10D1100000C2B3000E710200000000001940E800D8
:10D120005E6F020000000000C0CF2800826D020088
:10D13000000000000040EB00004C78000080FB0085
:10D140009980FB00C308DD000100400060407D00C5
:10D150000080FB00128902000000000000C2B30042
:10D160000E710200000000001840E800004C78003A
:10D17000E74F5000F1FF360061002000A0082000BA
:10D18000188A0200000000001980FB004300DD0047
:10D1900060407D00C80007009940E800814C78009D
:10D1A000A0B6200090CF5000D9FF3900310D2000EB
:10D1B00000092000728A020000000000920037007F
:10D1C000A082200001487800C00E2000808F50000F
:10D1D00005003A003101200030162000728A02005A
:10D1E0000000000004003700D1002000601720007C
:10D1F000728A020000000000710120003007200048
:10D20000728A0200000000000044EB0040B62000DB
:10D2100008487800D700070051B620008048780001
:10D22000A1B62000884878000004E00038003200F1
:10D230004AB620008004EB00B8BB200000C2B30057
:10D240000E710200000000001A40E8005E6F02004C
:10D2500000000000C0CF2800826D02000000000026
:10D26000195B88000900780060407C000080FB00AA
:10D27000128902000000000000C2B3000E7102001B
:10D2800000000000105B80000000E800105B8800D8
:10D29000E70F5000F4FF360061002000A0082000D6
:10D2A000188A020000000000184078008200070081
:10D2B0009A427800E9CF52000F003E00195B8800C7
:10D2C00089007800A2B62000B4B62000B3BB2000CD
:10D2D0001280FB004300DD000100400061C37900C3
:10D2E00006707A008100E800E88F5000F8FF3A00ED
:10D2F000115B88001249E800054DE800A70007000F
:10D3000051B62000804878000004E000CBFF3A00CE
:10D31000B102200030182000728A020000000000D4
:10D32000390037004000070011012000E01A2000FA
:10D33000188A02000000000030C3B3007C8C020099
:10D34000000000000000EB00105B88000004780083
:10D3500099B5200000C0EB007C8C020000000000AA
:10D3600000F47C00105B800060C07C000080FB004B
:10D37000128902000000000000C2B3000E7102001A
:10D3800000000000105B80000004E800185B8800CB
:10D39000E70F5400EFFF3600B0CF28009A6D02006F
:10D3A0000000000019407800430007001600370015
:10D3B0001D00070001012000F01B2000728A0200FE
:10D3C0000000000050C5B3007C8C0200000000008B
:10D3D0000D00370014000700F1002000F01C2000B1
:10D3E000728A020000000000C0CCB3007C8C0200F6
:10D3F000000000000400370041022000E01D200072
:10D40000728A0200000000004F0578004F04BE0041
:10D410000000060091002000200A2100728A02000C
:10D420000000000000000600881F7800F68B020054
:10D430000000000000447800A1002000202020000F
:10D44000188A0200000000000804E00005003A000D
:10D450003100200080BB2000728A02000000000022
:10D460001300370091002000C0202000188A02001D
:10D47000000000000808A300040032005101200051
:10D4800050212000188A0200000000000818A300A4
:10D490000400320041012000A0222000188A02006E
:10D4A00000000000B0CF28009A6D020000000000CC
:10D4B0004F047800000006008040780020C2B300CE
:10D4C00080CF50001700320005003E00E4CF50002E
:10D4D00019003200F0CF500021003A000700370059
:10D4E00080C2B30080CF5000090032006540400088
:10D4F00080CF50001A003A0014003700B10120001C
:10D50000E0232000728A02000000000018003700AB
:10D51000A101200090252000728A02000000000076
:10D52000130037005101200030272000728A0200CA
:10D53000000000000E00370081012000802820003C
:10D54000728A02000000000009003700010120007B
:10D55000002A2000728A0200000000000400370048
:10D56000E1002000002B2000188A020000000000CB
:10D57000000006008040EB0030BC2000014878002D
:10D5800050BC20000148780040BC200001487800D1
:10D59000050007000080FB000000060002000700F5
:10D5A0000080FB0000000600889FBE008A9FBE002E
:10D5B0008C9FBE000044EB0060BC2000084878004F
:10D5C00059BC20001904E00067003A00F68B020005
:10D5D000000000000004E0000700320030BC200022
:10D5E00008487800884C780040BC20000848780043
:10D5F0000000EB0064003700A0822000104078009B
:10D600007C8C0200000000001BC0B3008046EB00D1
:10D610000D4578008B447800BCBB200010C0B300DF
:10D62000328C0200000000000044780010C0B300FB
:10D63000328C020000000000E14F540003003A0069
:10D64000E14F50001D003A0036003700804F540073
:10D6500002003200884178002000370030BC2000F2
:10D660001040780080CF5500060031000A80FB0092
:10D6700060407E0080C164000600320013C0B30029
:10D680000400370000C06D000080FB000000E900CE
:10D69000CF01DE000304E00006003A00E8CF5500A9
:10D6A0000C003E0040BC20000B4878008B46780000
:10D6B0000A003700E1CF510008003A008A80FB00E1
:10D6C00061407E0000C0740080707E0013C0B30013
:10D6D000070037008B4678008041EB000A80FB0092
:10D6E00089C0EA0060417E0082C0600001707E0057
:10D6F00003407800328C0200000000008B45E800F7
:10D7000089C4440005003A000A80FB0060407E00A6
:10D71000570007000A45E80019C0B300E74F55005D
:10D72000BEFF360000C4B30080CF55000E003600A7
:10D7300060BC20001004E0000B003A0030BC200068
:10D740000D4878000D04E00003003A0011C0B3005A
:10D7500050BC20000148780011C0B300B0BB2000CD
:10D760001004E00007003A008040EB0030BC2000CD
:10D770000148780050BC20000148780040BC2000DF
:10D78000014878000180FB004F06BE004F05BE0037
:10D790004F04BE00000006000800FA00889FBE008B
:10D7A0008A1F78000000EB00B1BB2000E0C17800C8
:10D7B0006E815700037178000000E800E80F500008
:10D7C000FAFF3A0032BC20001245780051BC20001C
:10D7D0009144780040BC20001044780000C4B3009D
:10D7E000004978008048EB006FFF07000004E0006C
:10D7F0000C0032000001EB00B3BB20006E8057002C
:10D80000E040790062C0790080CF500005003A0006
:10D810000201E800E80F5100F8FF3A0012C0B3001F
:10D82000010037000041EB000000EB00B1BB20001D
:10D83000EE815700E37078000000E800E80F500028
:10D84000FBFF3A0030BC20000A48780050BC2000A2
:10D850000948780040BC2000084878000280FB009E
:10D860004F0578004F04BE000080FA00000006005B
:10D8700062BC2000124068000080FB00B1822000E2
:10D8800060C07800004978000080FB0000000600BE
:10D89000E0CF2800826D02000000000000000600BA
:10D8A000889FBE008A9FBE008C1F7800C922A800F6
:10D8B000CB22A900C8C2A90001B420001140780001
:10D8C0000034A1000044A00080487800F0FF070069
:10D8D0009AB620006CB62000FA700200000000002A
:10D8E00080417800004D78000080FB004400DE009D
:10D8F00081B6200080487800E14F5000530032008C
:10D9000003003900E44F50006E003A006600370013
:10D91000E2CF51000F00320005003E000304E0009A
:10D920006C003200E1CF510044003A00070037009C
:10D93000E4CF51000E0032004000390068C05100B1
:10D94000E14F50003D003E000F003700D0FF0700C0
:10D95000E1FF3700F68B020000000000004E780067
:10D9600010C0B3000E71020000000000DAFF3700A3
:10D9700000C0EB007C8C0200000000000E71020071
:10D9800000000000D4FF370010C0B3000E71020089
:10D990000000000090C0B3009A4F100004003A004D
:10D9A000C1CEB300A08220000148780003003700F8
:10D9B00001CFB300A082200001487800EDFE0700EF
:10D9C000004E78000004E0001100320078B620001C
:10D9D0008045EB00B9BB20000B4C78000B40780071
:10D9E0000080FB0060C07C000E710200000000009F
:10D9F0001840E800004C7800E74F5000F8FF360070
:10DA0000E6FE0700004E78000004E000F2FF3A0056
:10DA100070B620000048EB000004780000C0EB0066
:10DA20000E710200000000001840E800004C780071
:10DA3000E74F5000A8FF3E00F8FF37000040EB0022
:10DA40000E71020000000000A3FF37006FC06100EC
:10DA5000004DE80010C0B3000E710200000000008D
:10DA600070B620000048EB001A04E0009AFF320074
:10DA70000004780099B62000FA700200000000004F
:10DA80007C8C02000000000010C0B3000E71020088
:10DA9000000000001840E800004C7800994F50004A
:10DAA0008DFF3100F4FF370003407800308E020014
:10DAB0000000000010C0B3000E7102000000000062
:10DAC00085FF37000040EB000E71020000000000EF
:10DAD00081FF37004F0678004F05BE004F04BE009F
:10DAE000000006000000E0000300320010C3B30095
:10DAF000CA0107000200370000C3B300C7010700D6
:10DB000000000600881F7800B0407800000478000C
:10DB10000104E0000500320001407800BF01070069
:10DB2000B84078000104E000FBFF3A004F047800A1
:10DB300000000600881F7800B040780000047800DC
:10DB40000104E0000500320001407800B301070045
:10DB5000B84078000104E000FBFF3A00D0C0B300F9
:10DB6000AE010700A0C0B300AC0107004F0478006D
:10DB700000000600889FBE008A1F780000457800DC
:10DB800040CB2800DFFF070009C8B30088C0B300FE
:10DB9000094065000300320010C3B3009F01070075
:10DBA0000200370000C3B3009C0107000980FB009E
:10DBB0008004D1000844E900F5FF3A004F057800E1
:10DBC0004F04BE0000000600E4874700889FBE00A7
:10DBD0008A9FBE008C9FBE008E1F78000006BE008C
:10DBE0000040EB0080F79F000A102E005B5F2000D2
:10DBF0008EC0B3000A01BE000C00BE000C0902007A
:10DC0000000000000004BE008FF097000104E00057
:10DC100003003A00E00F5400E08F5C000C0032007B
:10DC200001C3B300014044007C0107000851B80063
:10DC30000BC0B9000300400009D2B90084014000C4
:10DC40000206560083865E0010C0B30080F79F0076
:10DC5000A2002000030020000A00BE000C09020000
:10DC6000000000000005BE000E47E900E1FF3A0099
:10DC700001C3B30001404600680107004F07780068
:10DC80004F06BE004F05BE004F04BE004F00B1005E
:10DC900000000600889FBE008A9FBE008C1F78008F
:10DCA0000004BE00F0232400F1002000800F540087
:10DCB000818F5C001700360002242400F30020004E
:10DCC0000800BE000C09020000000000560007001A
:10DCD000C0C2B3005101070002242400F300200059
:10DCE0000800BE002C090200000000000004BE0075
:10DCF0001C002000703E2000800F5400E08F5C006C
:10DD00000A003E0070CB28007EFF070010002000B4
:10DD10002B0037000000EB00713E2000810F540003
:10DD2000E08F5C00260036000006EB00823E2000FB
:10DD3000030020000800BE000C09020000000000E3
:10DD40000005BE0030062000800F5500E08F5D000A
:10DD5000030036000A007800330007000F00370088
:10DD60000C00E0000B003200E90F5500E08F5D0071
:10DD70000300360000C3B30028010700020037008B
:10DD8000C0CB28005FFF07000A00780026000700CC
:10DD9000020037000A00780023000700C0C2B30069
:10DDA0001E010700823E2000030020000800BE0084
:10DDB0002C090200000000000004BE00100020003A
:10DDC00031062000810F5400E08F5C000300360014
:10DDD00008007800140007000F0037000000E00082
:10DDE0000B003200E90F5400E08F5C0003003600A6
:10DDF00000C3B3000901070002003700C0CB2800B0
:10DE000040FF070008007800070007000200370005
:10DE100008007800040007004F0678004F05BE0098
:10DE20004F04BE0000000600889FBE008A9FBE000F
:10DE30008C1F7800800478008040EB000A7122007B
:10DE40004BC0B300AC002000811F78001100090016
:10DE50008A84D80000047800CF0078000104E00034
:10DE600002003A000800E0000600320001C3B300DF
:10DE700001404400E90007000AC0B9008084540052
:10DE800011C0B300811F7800110009000C85D80073
:10DE900000057800CF0078008B45E900EAFF3A00E2
:10DEA00001C3B30001C04400DC0007004F06780046
:10DEB0004F05BE004F04BE0000000600889FBE0054
:10DEC0008A9FBE00804478008041EB004AC6B300C0
:10DED0002BC0B3000980FB000A81FB001100090080
:10DEE0000280D8008000FD00014478000304E000B7
:10DEF00002003A000104E0000600320001C3B30052
:10DF000001404400C50007000AC0B90080C45400A5
:10DF100013C0B3000A80FB00A2002000110009001A
:10DF20000280D800004578008B45E900E9FF3A00FF
:10DF300001C3B30001C04400B80007004F05BE0094
:10DF40004F04BE0000000600889FBE0080047800D9
:10DF5000F0CC2800EBFE07004448DE006F006000B4
:10DF6000F8CB280060407C00AC0007006F806400A4
:10DF700060407C00A90007004F04BE0000000600BE
:10DF8000889FBE008004780000C3B30085000700AE
:10DF900080C7B300830007004448DE006F006000C4
:10DFA000F8CB280060407C007E0007006F80640092
:10DFB00060407C007B0007004F04BE0000000600AC
:10DFC000889FBE0080047800F0CC2800CDFE0700BA
:10DFD0004C48DE00F8CB280060407C008F00070032
:10DFE0004848DE006F00600060407C008B00070046
:10DFF0004448DE006F00600060407C00870007003E
:10E000006F80640060407C00840007004F04BE0005
:10E0100000000600881F78007D00B900D2022000B1
:10E02000110009000280D8008000FD004206200097
:10E03000110009008280D800010478009FFF0700CA
:10E04000E0C2B30075000700E94F540002003E0033
:10E0500000C3B300710007000840780097FF070075
:10E060004F047800000006002203200012417800CF
:10E0700032E0B7001180BA009100BA000001FD0043
:10E0800032E0B7000001FD004800DD000100700033
:10E09000000006000081200010407800E94F500089
:10E0A000050032000080FB0000004000C1AA2000F3
:10E0B000E0807800411188000000EB00001188002A
:10E0C0002062A8001011880021E2A8002342A800C5
:10E0D0008560A9000000060023C2BF000000D10037
:10E0E000610060000000060022C2BF006100600005
:10E0F000000006000000EB00C06C8800100020004B
:10E10000B06C8800A081200010A0A10000000600D3
:10E1100023C2BF000018A3000E003A00C06C8000AC
:10E120008000E80000002100808F500001003A00CC
:10E130008000EB00B06C8000808F50000500320042
:10E14000C16C880070408000614078000080FB0056
:10E150002011880000000600B26C8000744080002E
:10E1600003002100C06C80008000E800838F500015
:10E1700001003A008000EB00828F5000080032005E
:10E1800023C2BF000018A300F6FF3A00C16C88004C
:10E1900061407A000080FB0020118800F1FF370009
:10E1A0000000060000417800B16C8000C06C800067
:10E1B000808F500004003A00C222A900A0812000F4
:10E1C00010A0A0000A003700704080008270780024
:10E1D000B06C80000000E800B06C880001002100F5
:10E1E000810F500002003A000000EB00B06C880084
:10E1F0000000060022C2BF000008A300FDFF32009D
:10E20000301180000080FB000000060023C2BF0028
:10E210000008A300FDFF3200000006000041780066
:10E22000A1812000001020001100600005003A00CC
:10E2300023C2BF000018A300FDFF3A000200FB004C
:10E2400020118800000006000080FB0040118800BB
:10E250000000060022C2BF000000D1006100600083
:10E26000000006002222A9000000060095C0BF00A1
:10E270000048A3000D003A0041408000504080005B
:10E28000810F50000900320023C2BF000018A30014
:10E29000FDFF3A008580A9009580A80030408000ED
:10E2A000614078000080FB0020118800000006001B
:10E2B000809FBE00821F78003211800021408000C4
:10E2C0000040800082707800204080000000E8005C
:10E2D0002040880011408000810F500001003A006A
:10E2E0009560A9008560A9004F0178004F00BE002D
:10E2F00000400600809FBE00404080008000E80093
:10E300004140880050408000808F500002003A0059
:10E310009580A900040037003040800061407800FB
:10E320000080FB00201188008580A9004F00BE00FE
:10E330000040060060D12800826D0200000000004D
:10E3400000000600889FBE00C222A800D800070077
:10E35000F8FF0700D200070080407800E0DA2000D4
:10E36000014878000104E000C800350002003A00CE
:10E37000F0FF0700F7FF3700E1CF500006003A003A
:10E38000CB000700404E020000000000C80007005C
:10E39000E8FF0700EFFF3700E2CF500006003A0029
:10E3A000C30007002465020000000000C000070051
:10E3B000E0FF0700E7FF3700E3CF500006003A0018
:10E3C000BB0007002057020000000000B800070053
:10E3D000D8FF0700DFFF3700E4CF500006003A0007
:10E3E000B3000700506C020000000000B0000700FE
:10E3F000D0FF0700D7FF3700E5CF500006003A00F6
:10E40000AB0007007659020000000000A8000700DA
:10E41000C8FF0700CFFF3700E6CF500006003A00E4
:10E42000A30007001C84020000000000A0000700F9
:10E43000C0FF0700C7FF3700E7CF500004003A00D5
:10E440009B0007009A000700BAFF0700C1FF3700D2
:10E45000EFCF500008003A0010C0B3000E71020068
:10E4600000000000C222A9000671020000000000A6
:10E470000000FE00B7FF3700F0CF500003003A0065
:10E480000040EB0019010700B2FF3700F1CF500048
:10E4900003003A0010C0B30014010700ADFF3700BD
:10E4A000F2CF500025003A000000EB008008880001
:10E4B000F0088800E00C8800CAC6BF0001CEB30097
:10E4C000014060006041B300CAE6B7007400070075
:10E4D0000080FB000018A3000100320010A1A8007A
:10E4E0000008A300010032001081A8006C000700A2
:10E4F0004804DD006A0007000080FB000000740093
:10E50000D00C8800C00C880060002000E00C88005F
:10E51000630007004804DD00610007000080FB0085
:10E52000000074006008880011E1A80010C0B3006A
:10E530000E7102000000000086FF3700F3CF50008C
:10E540000B003A000000EB0080088800E00C880017
:10E55000CAC6BF0001CEB30001406000CAE6B700E2
:10E5600010C0B3000E7102000000000079FF3700F8
:10E57000F4CF50000D003A0021E3A800C0C0B30062
:10E5800094880200000000000004780021E3A90044
:10E590004800DE000E710200000000000840780014
:10E5A0000E710200000000006AFF3700F5CF500036
:10E5B00015003A0021E3A800C0C0B300948802000F
:10E5C0000000000000047800067102000000000056
:10E5D0004840DE000E710200000000000840780094
:10E5E0000E710200000000007470020000000000C4
:10E5F000E14F5000F0FF3A00FA7002000000000006
:10E6000021E3A90053FF3700F6CF500014003A0071
:10E61000AA450200000000000004BE004808DE0019
:10E620000E710200000000004048DE0001002000E2
:10E630000E710200000000004849DD004840DE0085
:10E6400000007100C848DE000E71020000000000EA
:10E65000084078000E710200000000003DFF370006
:10E660000168A30005003200014078001500070092
:10E670000E7102000000000036FF37000040EB0082
:10E680000E7102000000000032FF370001407800E8
:10E690004A0007000E710200000000002DFF370045
:10E6A000FA700200000000000080FB00000006007D
:10E6B00000C0EB00030007000040EB003F00070034
:10E6C00000000600881F7800004478000081FB00ED
:10E6D000C410DE00E1C06000C208DD00C9C2BF0096
:10E6E0000024A10001407000C9E2B700C310DE00A1
:10E6F000E1C0600081C04000C9C2BF000014A10099
:10E7000001407000C9E2B700C210DE00E1C0600045
:10E71000C9C2BF000004A10001407000C9E2B700F7
:10E720000201D1004711DD00C8C2BF000074A10082
:10E7300002407000C8E2B700E1406400C608DD0096
:10E74000C8C2BF000064A10001407000C8E2B70069
:10E7500050002000C28902000000000000CEB3007B
:10E7600080406400CBC2BF000028A300010032003B
:10E770000144A000CBC2BF000018A300010032007A
:10E780000134A000CBC2BF000008A300010032008A
:10E790000124A000CA42E20001003D000114A000D3
:10E7A000CAC2BF000068A300010032000104A0003B
:10E7B0000180FB004F04780000000600881F7800ED
:10E7C000004478000081FB000268A30003003200CF
:10E7D000C002A900C202A80002003700C002A900BE
:10E7E000C202A9000258A30003003200C962A800B7
:10E7F000CB62A90002003700CB62A900C962A90060
:10E80000C410DE00E1C06000C208DD00CBC2BF0062
:10E810000024A10001407000CBE2B700C310DE006D
:10E82000E1C0600081C04000CBC2BF000014A10065
:10E8300001407000CBE2B700C210DE00E1C0600012
:10E84000CBC2BF000004A10001407000CBE2B700C2
:10E850008200D100C708DD00CAC2BF000074A10059
:10E8600001407000CAE2B700E1406400C608DD0064
:10E87000CAC2BF000064A10001407000CAE2B70034
:10E8800050002000C28902000000000000CEB3004A
:10E8900080406400CBC2BF000028A300010032000A
:10E8A0000144A000CBC2BF000018A3000100320049
:10E8B0000134A000CBC2BF000008A3000100320059
:10E8C0000124A000CA42E20001003D000114A000A2
:10E8D000CAC2BF000068A300010032000104A0000A
:10E8E0000180FB004F04780000000600881F7800BC
:10E8F000804078000040EB00C8810200000000006A
:10E90000004478000004E00001003200C222A800A8
:10E91000084078000E7102000000000074700200D0
:10E92000000000000004E0000D003200FA70020058
:10E9300000000000E14F40000400320000404400AD
:10E940000E710200000000000500370010C0B30087
:10E950000E710200000000004F0478000000060065
:10E960000804E000EDFF3A00806D80000000E00048
:10E970000D003A000080EB00806D8800C2C2BF002D
:10E980000000D100610060000004A20000404000CF
:10E99000212C2000914078000114A10080C070005B
:10E9A00001007800C2E2B700806D80000000E9003D
:10E9B000806D8800D9FF37000C08000012000000AD
:10E9C00002000000000042001200000000000000F1
:10E9D0000000000000000000000000002E0B0000FE
:10E9E0001A000000000000004212000000100000A9
:10E9F00000000000480B00000200000000000000C2
:10EA00001E0800000C0000000200000000181C009E
:10EA10001D0018001C1D03000B131B004A0B0000F7
:10EA20000600000000000000500B0000080000007D
:10EA3000000000002A08000002010000020000009F
:10EA4000F0005E00BCE261003FDD8300C29C7E00FE
:10EA500020A3FD001F419D00C3217F00FCA24000B8
:10EA60001E5F0100E3BD3E006082DC00237D9F004D
:10EA7000C1421C00FEA0E100BF5D030080DE3C003F
:10EA800062BEE000025CDF0081633D007C22C000CA
:10EA90009E1D4300A1FF460018FAA40027799B00A1
:10EAA000C584DA003866E500BB590700DB856700DE
:10EAB00039BAE4000658190047A5FB007826C400BF
:10EAC0009A653B00D98704005AB8E600A7F91B00F5
:10EAD00045C698007A24F800A6441A0099C7250074
:10EAE0007B3A640086D85B0005E7B9008CD2300021
:10EAF0006EEDB300510F4E0010F2AC002F71930079
:10EB0000CD114F00ADF370002ECC9200D38D6F006D
:10EB100031B2EC000E50AF00F1134D00CE907200F8
:10EB20002C6D3300D18F0C0052B0EE00326C8E0091
:10EB3000D0530D00EFB1F000AE4C120091CF2D007C
:10EB400073CA94007628AB00F51749000856B40044
:10EB5000EA693700D58B570009EBB50036688A00A3
:10EB6000D495CB002977F400AA481600E9B75500E0
:10EB70000B88D600346A2B007597C9004A14F6003A
:10EB8000A8742A00C89615004BA9F700B6E80A0039
:10EB900054D789006B350000580B0000700000004E
:10EBA00000000000C80B000026000000000000006C
:10EBB0002C0900008001000002000000CA8DCA007C
:10EBC0008DCA8D00CA8DD8008DE88D00CA8DCA000F
:10EBD0008DCA8D00CA8DE8008DCA8D00E88DE800D1
:10EBE0008DF88D00068E06008E128E001E8E280077
:10EBF0008E4869005A00000000000000146A1400EA
:10EC00006ACA8D00CA8D7A0067706700CA8DCA0013
:10EC10008DAA67009C679600678C67008267E80092
:10EC20008DC86700BA67BA0067128E000A6A2800AA
:10EC30008E312D005749520045000000205520001C
:10EC40005534550034557E0051305100CA8DCA00EC
:10EC50008DCA8D00CA8DE8008DCA8D00E88D4600F2
:10EC60005510540012529800530A5400B2558600B1
:10EC7000515541005254000000000000D461D400FE
:10EC8000612662002662720061346100CA8DCA008A
:10EC90008DCA8D00CA8DE8008DCA8D00E88DE80010
:10ECA0008D0C63008862E40062FE6200FA635E001D
:10ECB000624932004300000000000000A2488000CA
:10ECC00048C44800CA8DEA0048E24800CA8DCA001C
:10ECD0008DCA8D00CA8DE8008DCA8D00E88DE800D0
:10ECE0008D1A4B007449F4004A164B00DA4BFE00B3
:10ECF000485350004900000000000000547A5400BE
:10ED00007A6A7A006A7A4C007A467A00987A900099
:10ED10007AB07A00A87A88007AA07A00807AE8002F
:10ED20008D7C7B00EA7A68007B128E00A27BB800A3
:10ED30007A32570049524500000000008686540090
:10ED400086B88600B88640008638860002870A00AA
:10ED5000871287001A87F20086FA8600EA86E800A2
:10ED60008DF88D006287220088128E003E88220076
:10ED7000873357004952450000000000727F72003F
:10ED80007F807F00807F60007FE88D00CA8DCA0091
:10ED90008DCA8D00CA8DE8008DCA8D00E88DE8000F
:10EDA0008DD27F008E7F94007F5E4C00088128000A
:10EDB0008E4C43004400000000000000EE0B0000F9
:10EDC000A801000000000000AC0A000012000000D2
:10EDD00002000000143404000D8206004003A0006D
:10EDE00001CF00006700440000220000960D0000E3
:10EDF0000400000000000000000800000C000000FB
:10EE000000000000BE0A0000280000000200000010
:10EE1000143404000D8206004003A00001CF00005E
:10EE200067004400002200007F00140034040D003D
:10EE30008206400003A00100CF007F0000670000B1
:10EE400044002200000000009A0D000008000000AD
:10EE500000000000A20D0000020000000000000001
:10EE6000A40D00000A00000000000000AE0D00002C
:10EE70000400000000000000E60A0000020000009C
:10EE80000200000003000000B20D00000E000000B0
:10EE900000000000E80A0000460000000200000038
:10EEA000768B7A008B7D8B00828B87008B8C8B001E
:10EEB000928B99008B9D8B00A38BA9008BAD8B004F
:10EEC000B08BB5008BBA8B00BF8BC6008BCC8B0090
:10EED000D28BD7008BDC8B00E48BE8008BEC8B00B3
:10EEE000F48BF8008BFF8B00038C0A008C108C00D5
:10EEF000148C19008C1E8C00248C00000000000073
:10EF0000C00D00006804000000000000281200008E
:10EF100002000000000000002A12000002000000B1
:10EF2000000000002C12000016000000000000008D
:10EF3000000000000141780041DA2000804878009C
:10EF4000E34F500005003A0000202000306D88009B
:10EF500000082000406D88000300370000202000DA
:10EF6000306D8800406D8800E14F51000E00320086
:10EF700003003900E24F51001F003A00140037002F
:10EF800041C1B300A0DA20000148780041C6B300B7
:10EF9000B0DA20000148780021C3B300C0DA2000B5
:10EFA000014878001B00370021C0B300A0DA200020
:10EFB00001487800A1C0B300B0DA20000148780011
:10EFC00051C0B300C0DA20000148780011003700BA
:10EFD00011C0B300A0DA20000148780051C0B3008E
:10EFE000B0DA20000148780021C0B300C0DA200068
:10EFF00001487800070037008040EB00A0DA2000CD
:10F0000001487800B0DA200001487800C0DA20001A
:10F010000148780000000600889FBE00B0DA20009A
:10F020009040780000302000E2000700CBC2BF0013
:10F030000008A30004003200CBC2BF008004EB0034
:10F040000018A30001003A0019002000B8DA2000DF
:10F050009840780000202000E600070098407800E3
:10F0600000102000E30007009840780000202000F6
:10F07000D0000700090078004F04BE000000060021
:10F08000881F7800B8DA200098407800003020000F
:10F09000D80007009840780000102000C500070045
:10F0A0009840780000202000C20007000000EB001C
:10F0B0004F04780000000600889FBE008A9FBE00B3
:10F0C0008C9FBE008E1F780080017800F0B2200077
:10F0D000104178000280FB000000E90011002000D0
:10F0E000800EDD008005EB000204E0001C00320011
:10F0F000830478000005EB008A057800AEDA200072
:10F10000BCDA20000D8064001E4178000120200040
:10F11000BF0007009C40780000102000A5000700F9
:10F1200000082000CF000700004478009C407800D1
:10F1300000102000AF000700898444008B85450043
:10F140000804E000010032008B05E8000A05E80031
:10F15000F0B220001080FB008A0F5000E9FF3E0053
:10F160000B0078004F0778004F06BE004F05BE0029
:10F170004F04BE0000000600889FBE008A9FBE00AC
:10F180008C1F780080017800F0B2200010417800D8
:10F190000280FB000000E90011002000800DDD006E
:10F1A0000204E00014003200030478008004EB0045
:10F1B000ACDA2000BADA20000B0064001C417800B1
:10F1C00001202000920007009A40780000102000E3
:10F1D000780007009A4078000010200085000700A2
:10F1E000080444008904E800F0B220001080FB000D
:10F1F000808F5400F0FF39004F0678004F05BE00A5
:10F200004F04BE0000000600889FBE008A9FBE001B
:10F2100000202000930007000005EB00F0B2200062
:10F220001004E000150032008004EB0009057800AE
:10F23000BBDA20009B407800001020005D00070032
:10F240000020200087000700004478009B407800E1
:10F2500000102000670007000A0545000804E000D0
:10F26000010032000A05E8008904E800F0B220003D
:10F270001080FB00890F5000EEFF3E000A0078006E
:10F280004F05BE004F04BE0000000600889FBE0070
:10F2900088DA20001800780072000700B9DA200030
:10F2A0009940780000102000420007001800780004
:10F2B0006C0007000044780099407800001020009E
:10F2C0004C0007000884FB00080078004F04BE00D3
:10F2D00000000600881F78000080FB00A1DA2000F3
:10F2E00011417800316D800049000700B8DA200034
:10F2F00098407800001020002E0007009840780009
:10F30000001020003B0007004F04780000000600BA
:10F31000889FBE008A1F7800804478000004E000C7
:10F320000B0032000044EB00BADA20009A4078006B
:10F33000001020001F0007009A40780000102000F5
:10F340002C0007000844E80088CF5400F7FF3A007B
:10F350004F0578004F04BE00000006000080FB004F
:10F36000A1DA200011417800316D800028000700EB
:10F37000000006000080FB00A1DA200011417800A7
:10F380000110200022000700000006000080FB00A2
:10F39000A1DA200011417800010420001C000700C0
:10F3A00000000600406D80002E0007000080FB007A
:10F3B000000006000001780000B420001040780032
:10F3C0007040600005003A0002007800CC22B700CF
:10F3D0000280EA00C822B60002003700020078006E
:10F3E000C822B7000180FB00C289020000000000B3
:10F3F000000006000080EA00CC22B600C822B60059
:10F400000180FB00C289020000000000000006002D
:10F410000000E00004003A000180EA00CC22B600BF
:10F42000C822B6000B00370000B42000104078005E
:10F430007040600005003A0001007800CC22B7005F
:10F440000180EA00C822B6000200370001007800FF
:10F45000C822B7000280FB00C28902000000000041
:10F4600000000600C822B7000000000000000000F5
:10F47000000000008000EB00CA02B600010032006C
:10F48000110020000100780000000600047902004D
:10F490000000000000000600BC7802000000000030
:10F4A00000102000000006000C78020000000000A0
:10F4B0008100200000932000188A02000000000054
:10F4C000D1002000A0412000728A0200000000004C
:10F4D00000000600407802000000000061002000EB
:10F4E00080932000188A020000000000C100200064
:10F4F00070422000728A0200000000000000060036
:10F5000046790200000000000080FB0000000600B9
:10F51000D2790200000000000080FB00000006001D
:10F520000040EB00BA790200000000000000060075
:10F5300010C0B300BA79020000000000000006000D
:10F5400010C0B3008879020000000000000006002F
:10F550000040EB00AE790200000000000000060051
:10F5600010C0B300AE7902000000000000000600E9
:10F5700001012000D0982000188A0200000000003D
:10F58000E0B22000104078005E6F02000000000032
:10F5900000C2B3000E7102000000000000B42000A1
:10F5A0001080FB004400DE00614060005E6F0200DE
:10F5B0000000000000C2B3000E7102000000000055
:10F5C0003100200020AE2000188A02000000000058
:10F5D00000000600881F7800CA1E0200000000001C
:10F5E000F61C02000000000000047800CA1E0200A1
:10F5F00000000000F61C02000000000080007800FF
:10F600000800E900E30F5000020036000004EB00A0
:10F6100002003700E0B220000848E9000100E900DC
:10F62000E10F500008003E0000B42000E1C060007F
:10F63000C408DD00104178000244A10001487100B7
:10F640000800E0001F003A000004EB009867880003
:10F65000B103200080452000728A020000000000F3
:10F6600088017800420020001100200010002000D6
:10F67000D01F020000000000E1B220008048E90035
:10F68000F1042000E0932000728A020000000000D4
:10F6900088017800220020001100200010002000C6
:10F6A000D01F02000000000002B420006140600092
:10F6B0004400DD00924078000144A10000C97000C0
:10F6C00001003700AAFF07004F0478000000060081
:10F6D000CB02A900CB22A900C922A800C902A90017
:10F6E000E0B220009040780020C0B3009A7702007A
:10F6F0000000000000000600E10F50000900320089
:10F7000003003900E20F500009003A0006003700FC
:10F7100081032000D0992000188A02000000000018
:10F72000070037000C0007001F0007000400370027
:10F7300041022000E01D2000728A0200000000004B
:10F7400000000600B1002000600B2100728A020058
:10F750000000000000000600F1032000509D200082
:10F76000728A0200000000000040EB00C67902002F
:10F7700000000000F00F2000C2890200000000001D
:10F7800010C0B300C67902000000000010C0B30032
:10F7900088790200000000000040EB00C6790200FA
:10F7A00000000000000006000400FA00889FBE0070
:10F7B000D102200040A12000188A020000000000B1
:10F7C00068845700E48457000479020000000000B8
:10F7D000005C78000080FB00A46F020000000000C5
:10F7E00000C2B3000E71020000000000888F5400B8
:10F7F000F5FF3A00A0D228009A6D02000000000038
:10F80000A100200010A42000188A020000000000BF
:10F810008FF897000180FB004400DE00E94F5000A4
:10F820000E00320003003E00E84F50001A003A007C
:10F8300005003700EA4F50000D003200EF4F500036
:10F8400015003A000F00370061002000B0A420002E
:10F85000188A020000000000130037006100200039
:10F8600010A52000188A0200000000000E003700DA
:10F870006100200070A52000188A0200000000002E
:10F880000900370031002000D0A52000188A0200AE
:10F8900000000000040037007100200000A62000D6
:10F8A000188A020000000000A0D228009A6D020011
:10F8B00000000000B100200070A62000188A02009D
:10F8C000000000001FFC97000878A30005003A0024
:10F8D0006100200020A72000188A0200000000001C
:10F8E00004003700F100200080A72000188A0200E1
:10F8F00000000000A0D228009A6D02000000000065
:10F90000C100200070A82000188A0200000000003A
:10F91000080078008007B2004380DE0000417800D4
:10F920000004E00005003A00D100200030A92000CA
:10F93000188A0200000000001000370000042000B8
:10F940008040EB00EF4F510005003A0031002000ED
:10F95000D0A52000188A0200000000000700370030
:10F96000000040008140E800814F5100FCFF3A0058
:10F9700082FF9F00146F020000000000A0D2280048
:10F980009A6D0200000000009101200000AA2000F2
:10F99000188A0200000000001FF89700674160000D
:10F9A00010002000060032008040EB001000200014
:10F9B000000040008140E800814F5100FCFF3A0008
:10F9C0005E6F020000000000A0D228009A6D0200C5
:10F9D000000000004F04BE000080FA000000060096
:10F9E000007C2000C822B7000F00070020C0B30031
:10F9F0002100070074700200000000000004E00015
:10FA000005003200FA700200000000001A00070032
:10FA10000004E00003003A00F80007000004E000E2
:10FA2000F4FF320000000600C222A9000001EB0032
:10FA300042038800520388000203880012038800F2
:10FA4000F2088800ADC0BF00F1C8B30001406000FB
:10FA5000ADE0B700E208880000642000D00888000C
:10FA60000000210000928800E02321000248780075
:10FA7000629188000000060080417800B09180000B
:10FA8000E10F50007000320003003900E20F500017
:10FA9000D8003A0076003700E2CF51001000320063
:10FAA00005003E000304E0000A003200E1CF5100EF
:10FAB0005A003A000F003700F1CF5100CD0032005C
:10FAC000F3CF5100CB003200E4CF510053003A0095
:10FAD0001A003700D4FF070010002000C6003700CE
:10FAE00040D02800826D0200000000000000EB0002
:10FAF000C1003700C222A8000001EB00F208880014
:10FB0000B2088800A208880080002000F008880061
:10FB10008660A9009660A900ADC0BF00F1C8B3001F
:10FB2000014060000044A000ADE0B70010002000DC
:10FB30006091880002007800AF00370010C0B30069
:10FB40000E7102000000000090D02800826D0200BB
:10FB5000000000000040EB000E71020000000000F9
:10FB600010C2B3000E710200000000000040EB0064
:10FB70000E710200000000000040EB000E71020058
:10FB80000000000000C1B3000E7102000000000080
:10FB90000040EB000E7102000000000030C2B30014
:10FBA0000E710200000000000040EB000E71020028
:10FBB00000000000F0C0B3000E7102000000000061
:10FBC00020C4B3000E7102000000000000C4B300A6
:10FBD0000E7102000000000000C4B3000E710200AC
:10FBE0000000000050C0B3000E71020000000000D1
:10FBF00010C4B3000E7102000000000020C0B3006A
:10FC00000E710200000000000040EB000E710200C7
:10FC1000000000000000EB0077003700E022210028
:10FC20000348780041C0B300302321000148780028
:10FC3000402321000048EB0010002000B091880014
:10FC40000000EB006C003700422321001240E80066
:10FC5000004978000080FB00E122210003F07800D9
:10FC60003023210012417800904F5100610039008B
:10FC7000E02221009040780010C8B30080CF5000EF
:10FC80001900320000CCB30080CF500004003200D5
:10FC900000C8B30080CF500053003A002000370066
:10FCA000F0222100104078008080FB000148A30072
:10FCB000010032006200A8000138A30001003200F8
:10FCC00062A0A8000128A3000100320062C0A800C1
:10FCD0000118A3000100320062E0A8000008A300A0
:10FCE000010032006300A800002321001080FB0007
:10FCF0004800DD00F12221009180FB00010070002E
:10FD00004200DD00640040000092880001002100F4
:10FD1000810F500034003600019288003200370015
:10FD200010232100104078004800DD000100200071
:10FD300002232100124178000281FB000300200011
:10FD40000200700083807000C808DD000080FD00A4
:10FD5000804078000040EB00F22221001241780040
:10FD60000281FB000300200002007000838070000D
:10FD70004209DD00CE00DE00810071004200DD009E
:10FD800064004000E0804800920120000300200051
:10FD90000C09020000000000C0918800D191880089
:10FDA000F00F5000E08F5800050036007000500042
:10FDB000E0805800C0918800D1918800040037008D
:10FDC0001000200001002000C0918800D19188001F
:10FDD000C2918000D39180004018DE000100200015
:10FDE000E0088800D20888000000EB00B09188008D
:10FDF000010037000000EB00000006006091800069
:10FE0000E10F50002C003A0086C0BF000038A3006C
:10FE100002003A006200E20027003A001FE1A80059
:10FE20008780A9000000EB00E0918800019280002B
:10FE30000100E0000E003200000178005016800042
:10FE40004600DE007140800000F1780087C0BF00EE
:10FE50000048A300FDFF32008780A9000201E800EE
:10FE600001928000810F5100F4FF3900E291880077
:10FE70000000EB0010038800F0088800E191880082
:10FE80000100E000090032007040800001004000E5
:10FE900070F897000E71020000000000E0918000F1
:10FEA0008000E900E1918800F7FF3A00DEFE0700DC
:10FEB00010002000010037000000EB0000000600E9
:10FEC000812221009180FB008100D10061C160008E
:10FED00080407800024078000A01070000102000EE
:10FEE00000000600802221001014A1004101200022
:10FEF00050EE2000728A02000000000000000600A0
:10FF0000802221001014A0002101200090EF200089
:10FF1000728A0200000000000000060000B4200009
:10FF20001044A00000000600802221001014A00050
:10FF3000A8C6BF0001CEB300014060007040B3000E
:10FF4000A8E6B700C9C6BF00014060007040B3001A
:10FF5000C9E6B700C8C6BF00014060000034A00079
:10FF6000C8E6B700CAC2A900C8C2A900C902A90050
:10FF7000C8E2A800C922A900D013200010128800EE
:10FF80000000EB00201288000012880041E2A80067
:10FF9000D1012000E0F12000728A02000000000080
:10FFA00000000600889FBE008A1F780000047800C9
:10FFB000806780000000E8000080FB008067880008
:10FFC000CA1E020000000000F61C02000000000033
:10FFD000800478000000EB0090678800E30F540075
:10FFE0003000320003003E000800E000080032004C
:10FFF0000C003700E60F54003E003200E70F5400BB
:020000040001F9
:100000005C003200E40F54007A003A003000370000
:100010008109200000F82000728A02000000000020
:10002000780037005100200050602000728A0200E2
:100030000000000095000700E10F5400710032003D
:100040000900E900E10F50001100360041022000D4
:1000500080012100728A0200000000008001EB0094
:10006000220020001100200020002000D01F0200EC
:1000700000000000E10F500003003A000040EB00D8
:10008000680007000200370080C0B3006500070069
:1000900041002000C0032100728A0200000000001D
:1000A0005800370011C0B3000040EB009500070076
:1000B000F00020009E890200000000005100200096
:1000C00000042100728A0200000000004D00370089
:1000D000894078000174A0000040EB00890007000F
:1000E000A100200050042100728A020000000000DC
:1000F0004400370011C0B3000040EB00810007004E
:10010000F00020009E890200000000000900E000CD
:1001100004003A00080320000905780009052000C2
:1001200009003700080320000005EB000900E0008B
:1001300005003C003300370090032000800F54007E
:1001400001003600080320008840780010C0B3008A
:100150006C000700084078000E71020000000000EB
:100160000804E8000A05E8008A8F5400F2FF3A000C
:100170002400370011C0B3000040EB00610007000D
:10018000F00020009E890200000000000900E0004D
:1001900004003A0018022000090578000905200033
:1001A00009003700180220000005EB000900E000FC
:1001B00005003C0013003700F0072000800F5400BA
:1001C00001003600180220008840780010C0B300FB
:1001D0004C000700084078000E710200000000008B
:1001E0000804E8000A05E8008A8F5400F2FF3A008C
:1001F0000400370041022000E01D2000728A020046
:10020000000000004F0578004F04BE00000006000B
:10021000B1002000600B2100728A02000000000083
:100220000000060002C2B300824040000040EB0024
:1002300034000700F00020009E890200000000004A
:1002400081C0B3000040EB002E000700F00020004A
:100250009E8902000000000011C0B3000040EB00C6
:1002600028000700F00020009E8902000000000026
:10027000E1C0B3000040EB0022000700F0002000C6
:100280009E89020000000000000006000040EB0014
:100290003A000700F00020009E89020000000000E4
:1002A00031C0B3000040EB002200070050002000E6
:1002B0009E8902000000000031C0B3000040EB0046
:1002C0001C000700000A2000C28902000000000094
:1002D00031C0B3000040EB0016000700000A200008
:1002E000C28902000000000021C0B3000040EB0002
:1002F00010000700000A2000C28902000000000070
:1003000000000600889FBE00804478000144780009
:100310008180FB00C408DE00060007006F44640013
:100320008840780009407800020007004F04BE00B2
:1003300000000600881F7800C408DD000144780032
:100340000804A000E14F500002003A000144780088
:100350003840B30008407800080007000834A000C7
:100360000840780005000700084078000034A1002C
:10037000020007004F047800000006007A4C0200DB
:1003800000000000CAC2A800CAC2A90000000600FE
:10039000889FBE008A1F780000457800814478005D
:1003A00020DA20000048EB000A04E00003003A00D5
:1003B000A08120001080A0000C0037000104E000A4
:1003C0000A003200F103200050AE2000728A0200C1
:1003D0000000000011012000A0192100728A020013
:1003E00000000000FA700200000000004100200040
:1003F00040B22000728A020000000000CB42A80038
:10040000C942A9003100200080B22000188A0200F1
:1004100000000000CBC2BF004200DE0061006000AF
:1004200011C0B300F2000700CB42A900C942A800E6
:10043000C222A800C022A90081002000B0B2200082
:10044000188A020000000000C2C2BF000000D100F4
:100450006100600011C0B300E5000700C222A900DE
:10046000C962A800CB62A9008100200030B320003F
:10047000188A020000000000CBC2BF004300DE006B
:100480006100600011C0B300D9000700CB62A90071
:10049000C962A90081002000B0B32000188A0200C0
:1004A00000000000CBC2BF004300DE00610060001E
:1004B0008040EB00CE000700C002A900C202A800E5
:1004C000200020009E890200000000004100200062
:1004D00030B42000188A020000000000C2C2BF0031
:1004E0006140600011C0B300C1000700E1002000BE
:1004F00070B42000728A02000000000021E3A8000E
:100500002100200050B52000188A020000000000E1
:1005100072352000712B200090C0B30071000700DD
:100520000904E000080032003100200070B520000E
:10053000188A02000000000072352000712B200094
:10054000B0C0B3006700070041002000A0B5200044
:10055000188A02000000000002252000011B200074
:10056000A0C0B3005F0007000904E00008003200EB
:1005700031002000E0B52000188A020000000000D1
:1005800002252000011B2000C0C0B3005500070059
:1005900021E3A9008100200010B62000728A020029
:1005A00000000000F8C32F000004FD00C822B600C0
:1005B0000004FD00003C2000CC22B70040062000D3
:1005C0009E8902000000000010C0B3006100070017
:1005D000A100200090B62000728A020000000000F6
:1005E0000004FD00CC22B6000004FD000904E00078
:1005F00002003200C962A800CB62A90040062000B8
:100600009E890200000000000040EB00510007003E
:100610000904E0000B003200A100200030B72000E8
:10062000728A020000000000003C2000C822B700CF
:10063000400620009E8902000000000010C0B300A8
:10064000440007000A04E000120032000904E00040
:1006500010003200C002A900C202A800C422A800F3
:1006600001022000D0B72000728A020000000000C2
:10067000F1002000B0182100728A02000000000082
:10068000FA70020000000000C422A900C002A90004
:10069000C202A9005688020000000000610020008C
:1006A000D0B92000188A02000000000028DA2000DB
:1006B000184078005E6F02000000000081002000FA
:1006C00030BA2000728A020000000000A0812000E1
:1006D0001080A1001880FB004F0578004F04BE0079
:1006E00000000600889FBE008A1F78000044780042
:1006F000810478000205780080C2B3000E71020008
:10070000000000000840780094880200000000000B
:10071000000478000A7002000000000090C2B300DC
:100720000E71020000000000890F54000300360023
:10073000100020008A0F5400010039000000EB0077
:1007400011C0B3002A0007004F0578004F04BE0017
:1007500000000600881F7800004478004100200057
:10076000B0BA2000188A020000000000CBC2BF000F
:100770000000D10061006000884078001C00070084
:1007800031002000F0BA2000188A020000000000AA
:10079000CBC2BF00614060008840780014000700B1
:1007A0004100200020BB2000188A02000000000049
:1007B000CAC2BF000080FB004700DE00884078000E
:1007C0000B0007002100200060BB2000188A0200F7
:1007D00000000000CAC2BF004600DE0061006000E9
:1007E00088407800020007004F04780000000600EF
:1007F000814F500005003A003100200080BB2000EE
:10080000728A02000000000006003700510020003C
:10081000B0BB2000728A02000000000020DA200035
:100820001048E8000000060020D22800826D020077
:100830000000000000000600889FBE008A9FBE00E6
:10084000794080001000200050918800F6FF0700DA
:100850008005EB00FA70020000000000E34F50003A
:100860001200320004003E00E14F5000310032001F
:1008700034003E0096003700E64F50000900320079
:1008800003003E00E54F50008B003A006300370044
:10089000E74F50003E003200E84F500086003A001B
:1008A00031003700E0FF0700EAFF370030C0B30037
:1008B000804C780080C0B3009044980021E3A800E9
:1008C000C0C0B3009488020000000000C800DE0031
:1008D000A1449800B0449800B0C0B30094880200CE
:1008E00000000000C800DE00C1449800D044980019
:1008F000A0C0B3009488020000000000C800DE0021
:10090000E1449800F044980090C0B300948802003D
:1009100000000000C800DE00814C9800904C980058
:1009200021E3A900A1002000090078008E00070043
:10093000C8FF3700FA7002000000000067000700DF
:10094000C4FF3700FA700200000000000044780085
:10095000FA70020000000000804078000840780033
:1009600091000700BBFF3700FA7002000000000092
:1009700000447800FA70020000000000C840DD006A
:100980000080FB000080700050918800B1FF3700AC
:10099000FA700200000000000085FB00E14F5000EB
:1009A00004003A0030C0B3002471020000000000CF
:1009B0000300370020C2B3002471020000000000D1
:1009C000FA7002000000000000447800FA70020093
:1009D0000000000080407800A0CAB300804F54009F
:1009E00003003A0050C5B30080CF5000040032002D
:1009F00020C2B30024710200000000000005EB00DB
:100A000070C0B300804C78009A4498002100200008
:100A100009007800540007008EFF3700FA700200CA
:100A20000000000000457800FA700200000000009D
:100A3000004178008560A900C850DD000080FB00FF
:100A40000084700000002200800F54000100360076
:100A50000004780050C0B300804C78009A4498009D
:100A6000A244980031002000090078003E000700F1
:100A70007040800000408800E7004400C308DE00AA
:100A800081804000114088002B4088004183200075
:100A900081004000314088004B4088005B40880066
:100AA0009560A8005391800008017800468D0200EF
:100AB0000000000067FF37008B4C78009B449800D3
:100AC00011002000090078002700070061FF3700AF
:100AD0004F05BE004F04BE0000000600CAC2A900B8
:100AE000CB22A900CB02A900CB42A900CA02A900CF
:100AF000E24F500006003A00CAC2A800CB02A8008C
:100B0000CB22A800CB42A800CA02A80005003700EB
:100B1000CAC2A900CB02A900CB22A900CB42A900DE
:100B2000CA02A9000040E900E14F500007003E0062
:100B3000C8C2A900C922A900C902A900C942A900C6
:100B4000C802A900C8E2A80006003700C8C2A80071
:100B5000C922A800C902A800C942A800C802A8006A
:100B6000C8E2A80000000600889FBE008A1F780027
:100B700000057800810478000100E00007003200E1
:100B80000004EB0068407D000E71020000000000D0
:100B90000804E800888F5400FAFF3A004F057800F7
:100BA0004F04BE0000000600E44F50002300320056
:100BB00005003E00E14F500008003200E24F5000B7
:100BC0002A003A000D003700E84F500021003200A3
:100BD000F04F500025003A0010003700C022A90055
:100BE000E1C0600081C04000C2C2BF000014A1008B
:100BF00001407000C2E2B7001C0037000104E000B1
:100C000003003200C002A900C202A800170037008A
:100C1000C002A900C202A900140037000104E000CC
:100C200003003200C962A800CB62A9000F003700A0
:100C3000CB62A900C962A9000C003700E1C06000C6
:100C4000CAC2BF000004A10001407000CAE2B700A0
:100C500006003700E1C06000C208DD00CBC2BF0063
:100C60000024A10001407000CBE2B70000000600A4
:100C7000F00F20005C780200000000000000060079
:100C80005C780200000000008000780000B42000C2
:100C900002C4B3001040610001003A008000EB0084
:100CA000010078000000060000B420001064A000DD
:100CB00080B42000104078006140600004003200E1
:100CC0000040EB00C679020000000000030037007E
:100CD00010C0B300C67902000000000080B42000FC
:100CE000104078006140600003003200F0C2B300A1
:100CF0000E71020000000000A100200090AB200057
:100D0000728A0200000000000000060000B420000B
:100D10001064A10080B420001040780061406000A1
:100D2000040032000040EB00C67902000000000021
:100D30000300370010C0B300C679020000000000B5
:100D400080B4200010407800614060000300320051
:100D5000F0C2B3000E71020000000000A1002000EC
:100D600090AB2000728A0200000000000000060024
:100D700000B420001064A10080B42000104078006E
:100D8000614060000400320010C0B300C679020068
:100D900000000000030037000040EB00C6790200AD
:100DA0000000000080B42000104078006140600026
:100DB00003003200F0C2B3000E7102000000000018
:100DC000B100200030AC2000728A02000000000058
:100DD0000000060046790200000000000080FB00D1
:100DE00000000600D2790200000000000080FB0035
:100DF0000000060010C0B300887902000000000067
:100E00000000060010C0B300BA7902000000000024
:100E1000000006000040EB00BA790200000000006C
:100E20000000060010C0B300AE7902000000000010
:100E3000000006000040EB00AE7902000000000058
:100E40000000060041012000E0AC2000188A0200EA
:100E500000000000E0B22000104078005E6F020049
:100E60000000000000C2B3000E710200000000008C
:100E700080B4200010407800614060005E6F020086
:100E80000000000000C2B3000E710200000000006C
:100E900000B420001080FB004400DE0061406000D0
:100EA0005E6F02000000000000C2B3000E7102007D
:100EB00000000000C0D228009A6D0200000000006F
:100EC00000000600889FBE00CA1E0200000000004D
:100ED000F61C02000000000000047800CA1E020098
:100EE00000000000F61C02000000000080047800F2
:100EF000CA1E020000000000F61C020000000000F4
:100F0000000178000800E900E30F500002003600FD
:100F10000004EB0002003700E0B220000848E900BE
:100F20000900E900E10F5000020036000004EB0068
:100F30000500370081B420000940E90061406000ED
:100F40001104A100914870000200E900E10F500077
:100F500008003E0000B42000E1406100C408DD004C
:100F6000104178000244A100014871000800E0002F
:100F70002E003A00B103200080452000728A020052
:100F8000000000008001EB00420020001100200062
:100F900010002000D01F020000000000E1B220007D
:100FA0008048E900D1012000601C2100728A020003
:100FB000000000008001EB00220020001100200052
:100FC00020002000D01F02000000000081B420009B
:100FD0000040E900614060001104A10091487000E8
:100FE000F1042000E0932000728A0200000000005B
:100FF0008001EB00220020001100200010002000E2
:10100000D01F02000000000002B420006140600018
:101010004400DD00924078000144A10000C9700046
:101020000000EB00906788000100370085FF070093
:1010300001B42000F0C9B300914860004F04BE0025
:1010400000000600E0B220009040780030C0B300FD
:101050009A77020000000000C922A900C902A90075
:10106000C8E2A80080B42000104078006140600011
:10107000C679020000000000000006000101200007
:1010800040062100728A02000000000000000600F5
:1010900001B4200011417800E0B220000048EB00CC
:1010A00000CEB3008048610000000600889FBE00AB
:1010B000C922A800C902A800C8E2A800C8C2A800A6
:1010C000C942A800C222A900C022A900CAC6BF0006
:1010D00009CEB30009406000CAE6B7000004EB0087
:1010E000A8408800EAFF0700CB62A900C962A900F6
:1010F000C002A900C202A9002D83A9002D43A900A6
:101100002D23A9002D63A900094078002063B700B2
:101110008819880020F021002019880018198800FB
:101120004F04BE00000006000080FB00401988004C
:101130002023A8002003A90020C3BF000008A300AB
:10114000FDFF3200001880000000060021E3A80027
:10115000C0C0B300F4FF07000A70020000000000E6
:1011600021E3A90000000600881F7800E1002000AC
:10117000E0352000728A020000000000F10020002B
:10118000B0182100728A020000000000F100200067
:10119000C0362000188A0200000000000000EB00AA
:1011A0000A7002000000000011002000B03720008B
:1011B000188A0200000000000F00370021E3A80099
:1011C000C0C0B300D8FF07000004780021E3A900E5
:1011D000E0D02800826D02000000000008007800C6
:1011E0000A7002000000000011002000B03720004B
:1011F000188A020000000000747002000000000065
:101200000004E000EDFF3200FA7002000000000070
:1012100040D128009A6D0200000000004F047800C1
:1012200000000600881F780000047800F0B220005B
:1012300010407800EF4F500005003E008080FB001A
:10124000EF801000F0FF27000180DE000004640042
:1012500090408000E10F500012003200050039007C
:10126000E20F50001B003200E30F500031003A0043
:101270002600370000B4200001C2B30010C0600097
:101280000400320008007800E06F02000000000057
:101290002800370008007800A46F0200000000005A
:1012A0002400370000B4200001C2B30010C0600069
:1012B0000400320008007800146F020000000000F3
:1012C0001C003700084078005E6F0200000000003C
:1012D0001800370000B4200001C2B30010C0600045
:1012E0000600320008407800BA6D020000000000DD
:1012F00000C2B3000E710200000000000840780038
:10130000BA6D0200000000000A00370000B420009F
:1013100001C2B30010C06000030032004840DE008C
:101320000E71020000000000084078000E710200FB
:10133000000000004F04780000000600889FBE00F7
:101340008A1F7800000578000000E0000A003400E1
:101350008004EB000004EB00A00F20000900070050
:101360000804E800E40F5400FBFF3A008904E80099
:10137000890F5500F7FF3A004F0578004F04BE0073
:10138000000006000000E000140034008000EB00C4
:10139000000000000000000000000000000000004D
:1013A000000000000000000000000000000000003D
:1013B000000000000000000000000000000000002D
:1013C000000000000000000000000000000000001D
:1013D0008100E800810F5000EDFF3A000000060098
:1013E000000278008001EB001100200002012000C3
:1013F0008381410001006200010032000300A0006F
:10140000818040000201E900F9FF3A00F0B22000BB
:1014100010407800F04F5000030032000080FB00C5
:10142000700010008019DE00030078000000060044
:10143000889FBE008A9FBE0081004000810F50003F
:1014400025003D0000047800390020002B4B2200CD
:1014500001057800110009000904D8000100E0002E
:1014600006003A00000040000B0040001000BA00E7
:101470000E7102000000000014003700E18F5000E0
:1014800009003A00110009000904D80000004000DA
:101490000B0040001000BA004800DE000E71020090
:1014A0000000000009003700E28F500007003A00FA
:1014B000110009000904D800000040000B004000A2
:1014C0001080BA000E710200000000000804E8005D
:1014D000880F5500DFFF3A004F05BE004F04BE00E5
:1014E00000000600D2FF070000D328009A6D02001A
:1014F000000000000000060011022000402721002B
:10150000F8FF0700C104200050292100F5FF070063
:1015100061022000102E2100F2FF0700810220004E
:1015200070302100EFFF070051012000F032210050
:10153000ECFF0700B101200040342100E9FF070063
:1015400081022000F0352100E6FF0700B1012000F4
:1015500070382100E3FF0700E1022000203A21005B
:10156000E0FF070051012000003D2100DDFF0700E2
:1015700031022000503E2100DAFF0700E102200086
:1015800080402100D7FF0700C101200060432100F7
:10159000D4FF07001102200020452100D1FF0700E1
:1015A000C101200030472100CEFF0700510220007A
:1015B000F0482100CBFF070011022000404B210022
:1015C000C8FF070091012000504D2100C5FF070012
:1015D000F1012000E04E2100C2FF0700910220002F
:1015E000D0502100BFFF07005102200060532100AE
:1015F000BCFF070061032000B0552100B9FF0700C0
:10160000E103200010592100B6FF0700000006008A
:10161000881F7800E10020007091200084FF0700FF
:10162000FA70020000000000004478000E71020011
:101630000000000000D328009A6D020000000000A6
:1016400090C7B300804F5400040032008000EB00CC
:1016500090C5B300804F540001003A0011002000F3
:10166000010078004F047800000006000400070025
:10167000320D0200000000000000EB000000060038
:101680000400FA00881F7800F0FF2F0001002000FE
:10169000D0BF9F00E1BF9F004507A9002CA3EF002A
:1016A0004227A9000080EB008080EB005FB9970023
:1016B000EFB9970061015100E0815900D2BF9F004E
:1016C000E3BF9F005FB99700EFB99700800F51000B
:1016D000818F5900F5FF3A00A4C6BF0001CEB300C8
:1016E000014060005040B300A4E6B700C4C6BF008C
:1016F000014060003040B300C4E6B70081C0B300D1
:1017000000812000014878000004EB009840880028
:1017100056880200000000004A700200000000002D
:1017200068C0A80068E0A80088007800F00F2000DA
:101730003470020000000000B0408800210020004A
:10174000F00F20003470020000000000C04088004C
:10175000501680000080FB004200DE006340600005
:10176000E34F500004003A0011C6B300A0812000EE
:10177000014878000B003700E24F500004003A00A7
:1017800021C6B300A0812000014878000500370081
:101790000004E00003003A0051C3B300A081200020
:1017A0000148780068C0A90068E0A900A081200075
:1017B0001080A10081C0B300F0B220000148780081
:1017C000703F0200000000003260EF0080D228006D
:1017D0009A6D020000000000EE20020000000000F0
:1017E0004F0478000080FA0000000600889FBE00C9
:1017F000C922A800CB22A900C922A90028022000E2
:10180000A0002000C2890200000000000804E900D6
:10181000FBFF3A00C922A80010042000C289020080
:1018200000000000CBC2BF00E204600038022000CC
:10183000A0002000C2890200000000000804E900A6
:10184000FBFF3A00CBC2BF00110020000018A3002C
:10185000010032008980FB00010078004F04BE00C7
:1018600000000600881F780000447800C922A80004
:10187000CB22A900C922A90040002000C289020091
:10188000000000000804E00001003200C922A800A6
:1018900080002000C2890200000000000804E0006F
:1018A00007003200CBC2BF000000D10061446000DD
:1018B00000022000C289020000000000080037007A
:1018C00090012000C289020000000000C922A80087
:1018D00070002000C2890200000000000044EB00FC
:1018E00050002000C2890200000000000880FB00B8
:1018F0004F04780000000600889FBE000044780076
:1019000089C0B30061406400D6FF07008880FB00F7
:101910000104D1000004E000010032000874A000BE
:101920008944E900F7FF3A0080002000C2890200E4
:10193000000000000880FB004F04BE00000006000D
:10194000E1C0600081C04000F52C20009542780085
:101950000514A10081C272008002FD00CFE2B70031
:101960008002FD00616A20009140780005CEB3003E
:1019700085C060007140B3008000FD00A6E6B7009E
:101980008000FD00916C20009140780085C06000CF
:101990005140B3008000FD00C9E6B7008000FD00A3
:1019A000C01188008002EB00851188003062A80019
:1019B00061416100C410DD0030C2BF000044A100DD
:1019C0000140700030E2B700E3C1610083C1410013
:1019D00030C2BF0091CFB3000140600003407000EF
:1019E00030E2B7006142620030C2BF000004A100D3
:1019F0000440700030E2B700951188004611DD0008
:101A000033C2BF000064A1000240700033E2B7009F
:101A10000000060031E2A8003342A80087C0A900F8
:101A2000C922A9000000060031E2A9003342A90042
:101A3000F0C1B300A666B700C9C6BF0001CEB300AF
:101A400001406000C9E6B700CF22A900C922A80062
:101A5000000006008000780033C2BF000018A30019
:101A6000FDFF3A00A11188000000060032C2BF004D
:101A70000008A300FDFF3200B01180000000060046
:101A800032C2BF006100600000000600889FBE00F7
:101A90008A9FBE008C1F78008002EB000203E900E1
:101AA000800378000104780003067800A92C200048
:101AB0009A0020006B00200010408000E482420069
:101AC0000028E600050078000408E300FEFF35006A
:101AD00037017800B70178000280FD000302690039
:101AE000F40FB20004016900848169000280FD00E6
:101AF000F00020000030E60006007800800078004A
:101B00000C800900000000001980A1000281D300B0
:101B10001950AD008381D3001958AD000C80090025
:101B2000000000001980A0001970A3000482D300F7
:101B30008100E900F2FF3100EF0010000122DE0019
:101B4000041C78004300DE000000E8000A28B4000E
:101B50009580AB0008003200404080000A08E30096
:101B6000050032008580A9009580A8000608B40011
:101B7000100078002011880070035300CEFF310060
:101B80004F0678004F05BE004F04BE0036710400BA
:101B90000000000011022000203F2000728A020095
:101BA0000000000010002000906788000000060080
:101BB00011022000203F2000728A02000000000075
:101BC0001000200090678800001020000000060030
:101BD00011022000203F2000728A02000000000055
:101BE00010002000906788000000EB000000060055
:101BF00011022000203F2000728A02000000000035
:101C000010002000906788000000060081C0B3002B
:101C1000F0B220000148780000B420001054A10068
:101C20000000060081C0B300F0B220000148780037
:101C300000B420001054A1000000060001012000A3
:101C400040062100728A0200000000000000060029
:101C5000E0D228009A6D020000000000000006009B
:101C60008080FB000138A30003003200C002A900FD
:101C7000C202A80002003700C002A900C202A900E7
:101C80000128A30003003200C962A800CB62A900AA
:101C900002003700CB62A900C962A9000118A300A5
:101CA00003003200C942A900CB42A800020037005D
:101CB000C942A900CB42A9000008A30009003200D4
:101CC00000B4200010407800704060000200320034
:101CD000C8C2A80006003700CCC2A800C8C2A9002C
:101CE00003003700F0FB2F00CC22B600C822B6005C
:101CF000000006000040DA000000FE00FFFFFF00C9
:101D0000FFFFFF00FFFFFF00FFFFFF00FFFFFF00DF
:101D1000FFFFFF00FFFFFF00FFFFFF00FFFFFF00CF
:101D2000FFFFFF00FFFFFF00FFFFFF00FFFFFF00BF
:101D3000FFFFFF00FFFFFF00FFFFFF00FFFFFF00AF
:00000001FF
